:020000021000EC
:10B0000000800020DD570300255803002758030067
:10B010000000000000000000000000000000000030
:10B02000000000000000000000000000295803009C
:10B0300000000000000000002B5803002D58030002
:10B040002F5803002F580300651703002F580300E3
:10B05000F93B030000000000291903002F580300EA
:10B060002F580300B95403002F5803002F58030032
:10B070002F5803002F5803002F5803002F580300A8
:10B080002F580300411F03002F5803002F580300BF
:10B09000C91B03002F5803006D3D03002F58030008
:10B0A0002F5803002F58030000000000000000008C
:10B0B0000000000000000000000000000000000090
:10B0C000164B002B00D1144B9D46402292029A1A37
:10B0D000924600218B460F461348144A121A00F07C
:10B0E00067F80F4B002B00D098470E4B002B00D079
:10B0F00098470020002104000D000D48002802D0D0
:10B100000C4800E000BF00F02DF82000290000F0FE
:10B1100059F800F011F8C046000008000080002037
:10B120000000000000000000781F00208C5C002060
:10B130000000000000000000084B10B50400002BC8
:10B1400002D0002100E000BF054B1868836A002B85
:10B1500000D09847200000F033F8C04600000000FF
:10B160002C7D03000E4B70B500251E000D4CE41A1B
:10B17000A410A54204D0AB00F35898470135F8E776
:10B180001CF0C8FD084B00251E00084CE41AA41052
:10B19000A54204D0AB00F35898470135F8E770BDDD
:10B1A000781F0020781F0020781F0020781F0020C3
:10B1B00003008218934202D019700133FAE77047F6
:10B1C000FEE7C046002308221800F0B5D54CD64D46
:10B1D000D1B023706370A37023716371E2705A1948
:10B1E000043300211060402BF9D18022A323D20523
:10B1F000DB00D150CD4B9960013191609A68002AF3
:10B20000FCD00023CA4A01251360962292012592A0
:10B21000FF27082225A90B728B720B330B711620A6
:10B22000023BCA714D724B718F7118F05FFFC14BB9
:10B23000C149A5605A58A120AA435A500322C00010
:10B240001D58C2262A430F251A5008301A58B60036
:10B25000AA430B3D2A43B94D1A50AA59B848024097
:10B260001000C022120210438022A851893E920091
:10B27000FF3EAA5180262A6005327602FF329E5098
:10B28000B04EAF4A330044331B781D910092002B1F
:10B290001FD11A0001332032B754202BF9D10122DB
:10B2A0000023524299007250032B02D919003C31FD
:10B2B00072540133082BF5D10321062016F0C0FB90
:10B2C0008021C123A04A9B000906D15001234436A6
:10B2D000337016F03FFC002303219C4AC520136005
:10B2E0009B4A2373117021009A4A0C311160052288
:10B2F0002100A273A275A2772200243121612100CE
:10B300001532FF322262944A9C311360934AA16144
:10B310001370934A80211370C02263732375637581
:10B3200023776377FF2449035200A95080002A58ED
:10B33000A2433F3C22432A50A12229608949D200DE
:10B340008B5004382A58009C2240C02424022243F7
:10B350002A501D9A08208958834A1160834A8449DB
:10B3600054320A604821834A1180834A834913601A
:10B3700018F04CFD002807D10122814B16301A70BD
:10B3800018F046FD002801D016F0CEFD0126022758
:10B3900042AC142200212000FFF70AFF794D7A4ABF
:10B3A0002095267227802673209B954210D0290075
:10B3B000764805F08BFB3100380005F023FE744B16
:10B3C000197F5A7F9142FBD10021022005F01AFE1D
:10B3D0002195219B34A92000349318F015FD0028F5
:10B3E00001D016F0A1FD6B4A6B4B01201A606B4A2D
:10B3F0006B4B6C491A6000226B4B1A705A706B4B86
:10B400001A705A809860DA601A619A8014330024A6
:10B410009942F5D15E4EFF27F48316F075F980232B
:10B420005B051D69624B02381C60624BADB21C604B
:10B430001C815C81604B45431C70604B35621C6015
:10B440005F4B604E1C60042333605F4B5F481C60A1
:10B450005C729C7201238372023B0381C3720722D8
:10B460002100FFF7A5FE242221005948FFF7A0FE86
:10B47000200018F09BFB574B1F550134072CF7D1C8
:10B480000423326808201A4200D1B1E080267605F4
:10B4900033699BB25F2B01D80720A9E016F034F97D
:10B4A000336901389BB25843A8239B00EB188342B1
:10B4B000F2D80022484B1C2724C33E4B474A5D600C
:10B4C0001A6060225C811A813069454B316980B213
:10B4D000C01889B21AF032FB34690123A4B2604368
:10B4E0002B4E451935620025F3833E4E3370A8B2CA
:10B4F00042A919F0D9FB041E0CD1380068433A4B1D
:10B500001C22C01842A9230014F0F8F9002804D026
:10B5100034706BE00023337068E00135072DE6D10D
:10B5200068E0C046781F002094560020FC000040D0
:10B5300000250020009000400405000000E100E02C
:10B54000FF00FFFF245700200060004084570020C8
:10B5500080570020FC5A00207C57002071570020A3
:10B5600072570020001001406C570020F820002086
:10B57000B0580020AC5800209C580020A938030087
:10B58000A0580020001F0020001E0020507D030056
:10B5900078210020E1A40200A8580020BD5003003B
:10B5A000A4580020F45B0020285B00202C5B0020C6
:10B5B000D8560020F05A0020205B0020245B002099
:10B5C000E8560020E45A0020B4250020C0250020C1
:10B5D00098260020CC250020E85A0020ED8D02009E
:10B5E0009F020000B0250020D4250020002801D0B3
:10B5F00016F09AFC8D2320A81B18052218000021A4
:10B60000FFF7D6FD0D23012642AC6371F04A063BDD
:10B61000A3710933E3711278EE4B26714293002A2D
:10B6200001D101F0DEF9EC4D2F68002F01D001F0BF
:10B63000DAF9280008C08D2320A95B18190005221B
:10B640001CF019FB022204212B7AAE72B343134380
:10B650008B432B72EB791E43E04B16438E4305332D
:10B66000EE71DF77112334A81322DD4903700EF049
:10B67000E3FE002801D016F057FC0822002120002C
:10B68000FFF796FD102323802C3363805533FF335F
:10B690002000E3800EF0D2FE002801D016F044FC1A
:10B6A0001022D0492BA81CF0E6FA0123CE4A5B42B7
:10B6B0009382CE4B1100936100232BA893750DF05C
:10B6C000FFFD041E00D0A6E00127C74B24A91B786C
:10B6D000C74A38008B700F800DF038FF041E00D071
:10B6E00099E022AD010003222800FFF761FD10233D
:10B6F0003B432B70102306223B436B70AB78210039
:10B700009343043A134342A81A32AB70FFF750FD3B
:10B710008822882120AB9B181B78783A134320AAF3
:10B7200052181370B04B66391B7820AA5218137048
:10B73000032220AB479523AD1A8421000322280061
:10B74000FFF736FD10233B432B70102306223B43AB
:10B750006B70AB7834AE9343043A13433B43210000
:10B7600012323000AB70FFF723FD28AB3493142363
:10B77000B3819D4B75603781588832009D4B42A93B
:10B780000DF0E2FE041E48D101001C2242A8FFF782
:10B790000FFD882220AB9B181A780C2388211343B5
:10B7A00020AA52181370904B66391B7820AA5218A1
:10B7B0001370022220AB1A84210003222800FFF715
:10B7C000F7FC0F222B78210093433B431340D219FF
:10B7D00013432B706B78013A93433B431340D219C8
:10B7E00013436B70AB780A3A9343043A13433B43D9
:10B7F00012323000AB70FFF7DBFC28AB349314231C
:10B80000B381794B75603781588832007A4B42A9F1
:10B810000DF09AFE0400002C02D0200016F084FBEC
:10B820000C22002128A8FFF7C3FC0122734B6D49AD
:10B83000299320AB1A840123714A5B4213801022A2
:10B840002BA889181CF017FA0E216E4B23AD2B8004
:10B8500020ABC9182BA80DF033FD42AF041E00D059
:10B86000F2E0694A290001200DF070FE0090041EEC
:10B8700000D0E9E0AC78624B01001C2238009C71DA
:10B88000FFF796FC04223B7822AD13433B7020ABBC
:10B890009C745E4B20AA1382009903222800FFF7B4
:10B8A00087FC0122102313436B70AB78053293435E
:10B8B000043A34AE1343013A134300991332300073
:10B8C000AB70FFF775FC24AB34931423B3814C4B5E
:10B8D0007560988832004E4B39000DF035FE041E1D
:10B8E00000D0B3E001001C223800FFF761FC082201
:10B8F0003B7821001343921813433B70404B20AA1E
:10B900009B7928009374434B13820322FFF750FC6A
:10B910000F226B78210093430E3A13430E321340EB
:10B92000013213436B70AB780A3A9343043A1343E2
:10B930000E3213430F3A134330001332AB70FFF74C
:10B9400037FC24AB34931723B3812D4B7560988853
:10B950003200314B39000DF0F7FD041E76D10100A5
:10B960001C223800FFF724FC02223B7821001343FD
:10B970003B70234B20AA9B7928009374274B13829A
:10B980000322FFF715FC0F222B78210093430E3A78
:10B9900013430E321340013213432B70AB780A3A33
:10B9A0009343043A1343013A134330001332AB700C
:10B9B000FFF7FEFB24AB3360022333810223B38104
:10B9C00028AB33610E4B75609888320028E0C04682
:10B9D000B0250020AD500300B425002078210020C0
:10B9E000957D0300307D030020250020C1A20200C8
:10B9F000222500202C250020242500202993020048
:10BA0000802500203015000084250020321500001C
:10BA100088250020311500009025002034150000F5
:10BA2000DC4B39000DF090FD041E0FD1299B0093D3
:10BA3000009AD94B9A622A9B002B01D0D64AD36236
:10BA40000122D64B1A7004E0002C02D0200016F020
:10BA50006BFAD34AD34BD44C1A60D44A631D127884
:10BA6000DB7F002A01D100F0C3FF002B01D000F0E2
:10BA7000BFFFCF4A1268002A01D100F0B9FFCD4ABA
:10BA80001370012600253822002134A8FFF790FB0F
:10BA9000382200213800FFF78BFBC74B24220021FE
:10BAA0002BA83E827B61FFF783FB3822C34BC4493E
:10BAB0001D70C44B1D60C44B1D6020AB9B181E70D5
:10BAC00040232F93743330930B002BAA43CA43C3F4
:10BAD00043CA43C343CA43C307222900BB48FFF7F5
:10BAE00067FB2200BA4B48349C60BA4C28322900CC
:10BAF0001A6020003822FFF75BFB02232370033318
:10BB0000E370230038AA103303CA03C3230036AA04
:10BB1000083303CA03C323003AAA183303CA03C372
:10BB20003900200018F0F8F9A84201D016F0FCF90D
:10BB300042AC1C2200212000FFF73AFBA0239B020D
:10BB40006360F0231B03A3600323A34A2373A34B67
:10BB5000A34963611300A16125CC25C325CC25C36E
:10BB6000002219609F4BA0481A7018F0D3F90028E2
:10BB700001D000F043FF01229C4B52421A809C4BA3
:10BB800018709C4B1B68002B01D100F036FF9A4BBC
:10BB900008301A7C002A01D000F030FF1A745A7461
:10BBA000964A5A6119F078FA01F05CFA1622944B21
:10BBB00001201A7002F0C6FB924B9A68012A01D14B
:10BBC00000229A60784B68331A78FF2A01D001323C
:10BBD0001A7017F0EFFB0027431E0D9300280DDCB1
:10BBE00017F0E8FB2E2800DD3CE30121142017F0BC
:10BBF0003BFB0121162017F037FB33E334AD28005F
:10BC000017F0ECFB0028EBD00121080005F0FAF951
:10BC100000223F20644B2C7868331A70784B204008
:10BC20001B78834236D10121080005F0EBF900258D
:10BC30000226A40934AB5B195878002803D15A4B6B
:10BC4000693318701EE0012802D102F01BFB19E0D5
:10BC5000042803D1002002F0AFFB13E0052802D135
:10BC600002F0EEFA0EE00300B343152B02D105F00B
:10BC700013FB07E01B2803D14B4B69331E7001E017
:10BC800002F0DAFE0135AC42D4DA0021012005F0E1
:10BC9000B9F9E4E20300113B0A2B00D90BE117F0DC
:10BCA0007BFB594B0100002218680CF04EFB0CF096
:10BCB00005FA050001F0A6F8002800D1F9E00022FD
:10BCC000524928000CF02FFC040001F09BF80028DA
:10BCD0000AD000224E4920000CF025FC01F0E1FBC7
:10BCE000C7B2FB1F022B00D90827200001F048FB38
:10BCF00015F03DFA00900490002800D1D5E0010035
:10BD0000002242A816F076FB0123BB40013BDBB2C8
:10BD10000C93002334AE34780493A40901345127E2
:10BD200020AB0134FF18341939780C9B42A8194014
:10BD3000013716F007FBBC42F6D13F2332781A4098
:10BD4000194B19006A310C7819006B31087884425C
:10BD50000DD1459801F014FB2E4E009B00223100BE
:10BD6000280023930CF0F1FA041E55D16AE00878FC
:10BD7000052141436C33CB5C3F210B409342E8D11A
:10BD8000300017F02BFB049B34780133A409049393
:10BD90000134C4E7A025002080250020A424002031
:10BDA00069A402006C1F002078210020B02500202B
:10BDB000B4250020E8240020641F0020F55B00204B
:10BDC000005C0020245C0020745C0020F65B0020F6
:10BDD0002C5C00203C5C00206425002045A402006F
:10BDE000B9A20200B4580020945800205825002021
:10BDF00062250020FC5A0020005B0020853A0300E9
:10BE0000721F0020781F00208C5A0020A97D03009B
:10BE1000B27D0300BB7D0300010023AB012228009B
:10BE200002F0FCFB00283AD1874811F019FB0421ED
:10BE3000864B28006C331A780A4331001A700CF0D4
:10BE4000CFFA2CE0824E0200310028000CF06BFB90
:10BE5000040001F039F9002805D1239A31002800A7
:10BE60000CF04CFB1EE020000FF004FB06002398B2
:10BE70000FF000FB802330189B00984205D9022167
:10BE8000724B6C331A780A431A70724B9E4206D872
:10BE900001339B1B0022239920000FF0D6F92000CC
:10BEA00001F06EFA009801F06BFA0D9B049A9B1A50
:10BEB0000D932800D1E103001C3B052B22D83F2322
:10BEC000A01F184017F068FA634B010000221868A1
:10BED0000CF03BFA0CF0F2F8040000F093FF00289D
:10BEE0000ED02B785B0603D55C49200018F0E4FDEA
:10BEF00034AB1B787F2B03D95949200018F0DCFDA7
:10BF00002000AAE101380F2800D9A8E1554B188874
:10BF100000F0E4FD109001002BA80EF004FF2B9B15
:10BF20002BA8002B00D195E10EF0EDFE00224E492A
:10BF300007000CF0F8FA05F033F84C4A8300D318E8
:10BF40000490587818F0EAF93F2334AD2C78234058
:10BF5000834201D0002573E1454B464AD158002366
:10BF60000993349B08911A0A2B791B0613438B42C1
:10BF700008D9089D099E0121002049422D184E41F3
:10BF8000089509960293099B640603930022E30F28
:10BF9000394938000C930CF0C6FA01F082FA00908F
:10BFA000002800DCBFE0354C0022210038000CF0F6
:10BFB000BAFA01F060FA16900C980FF0B4F821006C
:10BFC000020038000CF0A9FA2D4E00223100380092
:10BFD0000CF0A9FA041E59D000222A490CF0A3FA49
:10BFE00011900FF053FC050011980E0001F0C8F9F4
:10BFF0000099254B0E91C9171A685B680F9102983A
:10C000000399801A9941AD185E410E9A0F9B8018D2
:10C0100059410FF0A6F81B49020020000CF06EFAFF
:10C0200001F0AEF9039BB34203DC75D1029BAB4236
:10C0300072D90E9A0F9BAD1A9E41169B02950396DC
:10C040000C93012569E0C046C37D0300F82300205E
:10C05000F77D0300FF0100008C5A0020FC7D0300E7
:10C06000077E0300D4560020AEA30300F3B0030004
:10C070000405000000B00040117E03001A7E03009A
:10C08000207E0300287E0300F0240020052000F01D
:10C09000C6FD0400051E40D03A00AF490CF02EFA50
:10C0A00002980399AD4B1A685B68801A9941009B0E
:10C0B0001893DB171993189A199B801859410FF0A0
:10C0C00050F8A749020020000CF027FAA54D0022E5
:10C0D000290038000CF027FA2900020020000CF09B
:10C0E0001CFAA14D0022290038000CF01CFA29008E
:10C0F000020020000CF011FA04980FF026F89B497A
:10C10000020020000CF009FA200001F0DDFF2200FF
:10C11000310038000CF0F2F90025200001F030F970
:10C12000002D00D116E702980399FA22002392000D
:10C1300019F02CFCCB175B045B0C069300230A0060
:10C1400001000793069B079CC91862415304C80B62
:10C150001843D11319F07EFE0022854B1AF0BCF96A
:10C160000EF0D6FF0C990090380001F0BFFF079D3C
:10C17000002860D02A007B4938000CF0D4F9079AD7
:10C180007C49119038000CF0CEF901F074F90600EA
:10C190000400052000F043FD051E429020D0079AC0
:10C1A000714938000CF0BFF96F49020028000CF00B
:10C1B000B4F9009A6A4942980CF0A0F90498429D9B
:10C1C0000EF0C3FF6949020028000CF0A6F90C9894
:10C1D000429D0EF0A8FF6849020028000CF09DF96E
:10C1E00042AB01221199002002F018FA051E0BD172
:10C1F000002E09D0614811F033F904212C00604B66
:10C200006C331A780A431A700025429801F0B8F886
:10C21000AC420DD110992BA80DF03CFE049802F011
:10C22000C9F90135002803D12100049818F0A2F8BB
:10C23000119801F0A5F8009A4B4938000CF06DF9FF
:10C24000380001F09DF8002D00D068E62BA80EF014
:10C2500046FD64E60EF03EFD109801F091F80127CE
:10C260000D98B9E41D9A474B9B58129300231393E2
:10C270003A4B1299139A1C685D68091BAA411691E2
:10C2800017921299139A19605A603D4B169A196FBA
:10C290008A18914201D90122524208241A673A4A67
:10C2A0001388A3431380394B188800F017FC0D90B6
:10C2B000010022A80EF037FD0122354B52420492B4
:10C2C00005931F94229B002B0BD122A80EF002FD98
:10C2D0000D9801F055F80EF05FF8002800D07AE1D3
:10C2E00070E1294B1C881F9B1C40EED122A80EF048
:10C2F0000AFD22001A490C900CF015F906000FF007
:10C30000C5FA04000D00300001F03AF8169A179BA8
:10C31000A41A9D4100940195019B002B00DD31E1A1
:10C3200003D1009B002B00D02CE10121080004F078
:10C3300069FE00220B490C980CF0F5F800221090D1
:10C3400005490C980CF0EFF80023041E42939C4220
:10C3500020D10123119380E02D7E0300F0240020E2
:10C36000287E0300337E03003C7E0300AEA303005F
:10C3700000408F40457E03001A7E03004B7E030081
:10C38000F823002000B00040F824002004250020FD
:10C39000FFFFFF7F052000F042FC42900028D8D02C
:10C3A0000022B04920000CF0BEF801F07AF8009DA0
:10C3B000019EAD4BC1171A685B68521973411A9000
:10C3C0001B911A981B99121A8B411000FA2219001E
:10C3D0009200002319F0DAFACB175B045B0C0A9386
:10C3E00000230B930A9A0B9B801859410A00C00B3B
:10C3F00053041843D11319F02DFD9C4B00221AF061
:10C400006BF80EF085FE9A4D060029000B9A20006D
:10C41000429F0CF088F82900020038000CF06EF8FA
:10C4200001F029F80100200001F060FE914D11900B
:10C430000B9A29002000429F0CF075F82900020099
:10C4400038000CF06AF83200290020000CF056F891
:10C450003200894942980CF060F8002287490C9814
:10C460000CF061F8119B0500002B2AD0429E002E93
:10C4700007D042AB01221099002002F0CFF806004D
:10C480000EE032007E490C980CF04DF81099070030
:10C490000200300002F02CF90600380000F070FFB6
:10C4A000002E0ED1002D0CD0764810F0D9FF0421BB
:10C4B000754B28006C331A7835000A431A7000F067
:10C4C0005FFF429800F05CFF002C37D000226F49DC
:10C4D00020000CF013F8119B002B2CD000226C498B
:10C4E00020000CF020F800F0C6FF002823D1694B93
:10C4F000188800F0F3FA01222100060006F022F865
:10C50000071E06D0010030000BF00FFC380000F0D1
:10C5100037FF300000F034FF5F49002220000CF0AC
:10C5200002F804F03DFD060002F044F8011E02D1BD
:10C53000300017F01FFF200000F022FF002D0FD069
:10C5400028000FF0A3F906000F00280000F018FFE4
:10C55000009B019C9B197C4100930194002409E0FD
:10C560000D9922A80DF096FC01235B42DC17009385
:10C5700001940124109800F003FF019B0127002B78
:10C580000EDB00E00024059B019A934204DC07D1F6
:10C59000049B009A934203D9009A019B049205934D
:10C5A000002C0BD1009801990EF0DBFD32490200FE
:10C5B0000C980BF0B2FF22A80EF091FB0C9800F043
:10C5C000DFFE7FE6002F07D12F4B586F00F06CFB8A
:10C5D000002801D10AE001270022304B68331A708D
:10C5E000002F03D00021012004F00CFD10F08EFA82
:10C5F000002868D1244B586F00F056FB002862D009
:10C600000121080004F0FEFC1F4C656F280000F0BB
:10C610004BFB011E48D0280005F005FF0BF04EFD36
:10C6200000221F4904000BF07EFF002205001D4977
:10C6300020000BF078FF00220600114920000BF0CB
:10C6400072FF0700200000F09BFE29003A00300036
:10C6500002F04EF8380000F093FE3100280000F0A0
:10C66000C3FED1E7117E0300F024002000408F407C
:10C670001A7E03003C7E0300287E0300787E0300C0
:10C68000817E0300867E0300F8230020207E0300C5
:10C69000457E0300D4560020AEA30300782100207D
:10C6A000B67E0300BB7E0300012004F0ABFC10F05B
:10C6B0002DFA002803D1226FD24B9A4203D80122CF
:10C6C000D14B78331A70D04B78331A78002A0BD0BC
:10C6D0000820CE498A8E82438A8600221A7004F08E
:10C6E0003BFBCB4804F00CFAE023CA4C5B002288E9
:10C6F0001A4200D1BAE00121080004F083FC258829
:10C70000EB050BD5C44B2B40238005F007F804F054
:10C7100021FD00F0A7FC002001F014FE40210D4295
:10C7200000D18AE0BB4A13888B43138005F00EFDCD
:10C7300004F0F4FF04F000FD00F030FCB74804F012
:10C74000DFF9FD2025AA24A9800215F087FC002826
:10C7500000D099E10023B24FB24EB34844934297C0
:10C76000439604F0CDF9B14A42ABB149B1480AF061
:10C77000C3F8B14B439C42A900202894E41811F05F
:10C78000AAF842A9002011F0A6F842A9002011F051
:10C79000A2F8439B429A009393421CD32100A74ADC
:10C7A000A74804F093F9002400F020FC04F0DDFC1D
:10C7B00001F0B0FDA04207D0A24804F0A1F901F0B9
:10C7C000A9FD0028FBD1012404F0B6FC00F0E6FB33
:10C7D000002CB3D12BE0220095499B4804F076F958
:10C7E000FD2028A9800218F078F9984B2BA9380071
:10C7F0002B9318F072F9964804F082F90023954AB9
:10C8000043938B4942AB8B4842960AF075F8439CA0
:10C8100011F082FC002803D18F4804F071F9013433
:10C82000002C00D143E121008C4804F04FF900F0C6
:10C83000DDFB04F09AFC04F03FFD80210D4211D095
:10C84000744A13888B43138004F068FF04F074FC6F
:10C8500000F0A4FB11F072FC00F0C8FB04F085FCB2
:10C8600004F02AFD0021012004F0CCFB7C4B68334E
:10C870001B78012B23D1059B002B05DC1FD14823FE
:10C88000049AFF339A421AD921240C255E4B694E33
:10C890007A331888002812D0013C002C05D00138CA
:10C8A0006843801900F0B3F9F4E70121080004F0AF
:10C8B000A9FB05F04BFC2100012004F0A3FB684B11
:10C8C0001A0068321278012A53D91A006A32117894
:10C8D0001A006B32127891424BD11A7F5B7F9A42D9
:10C8E00047D1049805995F4B5F4AD25842AB1492E6
:10C8F00000221592149C159D0019694144924290A2
:10C9000043911A7772B6594B594A10781978159B8A
:10C9100088421DD01D2312785343564AD3185A78A3
:10C9200018781202024311009A7812040A43D97847
:10C93000090611431E915A79187912020243110017
:10C940009A79DB7912040A431B0613431C930123D3
:10C9500062B6002B08D0439B1C9A934204DB06D19D
:10C96000429B1E9A934202D242A816F087FA18F010
:10C9700033FF01F015FCC022244B1201998E1142A5
:10C980000DD0998E3C4A204C0A40E06F9A860FF0F9
:10C9900024F8002801D00023236704F07DFC374CE5
:10C9A0002378002B01D1FFF707F90023237004F04F
:10C9B000C9F9002801D1FFF7FFF83E2004F096F8EE
:10C9C000114D3A220021E86F04F02CFFED6F280092
:10C9D0000EF050FD62680100280004F0CBF8FFF76C
:10C9E000EBF8274800E0274815F09EFAFEF73AFEDC
:10C9F000234815F099FAFFF744F8082015F094FA47
:10CA0000FFF7D0F8CB0C0000F82300208C5A002050
:10CA1000C07E0300F8240020FFFEFFFFF07E03002D
:10CA2000FCFF030004F40300017F0300D7D80200D9
:10CA3000D02F0000BC260020000CFCFFFC0B0000E7
:10CA40000D7F0300407F0300AA7F0300EFBEADDE31
:10CA5000C57F0300B1D802006E7F0300897F030009
:10CA6000782100200405000000B00040B9580020E3
:10CA7000BA580020BB580020FFF3FFFF78240020A5
:10CA80000880000004800000249815F00BFB259A14
:10CA9000249B9B18084A934200D95BE6074804F0A0
:10CAA0002FF8259A249B24A9981825AA4DE6044816
:10CAB00004F026F8BBE6C046FBFF030056A60300C1
:10CAC000A27F0300020010B5643213783E2B04D815
:10CAD0005C1CC31801331470D97710BD0C2380225D
:10CAE00001385843034B9200181843899B1843811F
:10CAF0007047C046BC260020031E06D0044B054AE2
:10CB0000C31A9B10534301339BB218007047C046B1
:10CB1000BC260020ABAAAAAA4289044B4172090A8A
:10CB200013404903194341817047C046FF9FFFFFEF
:10CB3000C02243899200407A5B0913401843704732
:10CB400070B5C26F0400C36E111E00D0D15C256F9A
:10CB500001332170E366AB421CD3A06F5B1BE3661D
:10CB6000666F002810D0FFF7E3FF00280CD00C23DD
:10CB700001385843084B7519C018A067E06765670E
:10CB800004F006FF206705E000237519A367E3673B
:10CB90006567236770BDC046BC26002010B50378CA
:10CBA0004380FFF7CDFF10BD3F23C2794171090AD1
:10CBB000134089011943C17170473022C379017153
:10CBC0000909114093431943C1717047002370B59F
:10CBD0000400438172B6054D2988FFF7EEFF20005F
:10CBE000FFF78AFF288062B670BDC046722400201D
:10CBF0000323C2798171090A9A430B401343C3711D
:10CC00007047C37940799B091B0218437047C022C3
:10CC1000C379920000791B01134018437047F8B59F
:10CC2000050008261B4F3B88002B14D072B60C233E
:10CC30003C88013C5C43184BE4182000FFF7E7FFF9
:10CC4000388062B60023A3602360636080239B006A
:10CC50001D4365811BE0114C23783343237005F09D
:10CC600075FA0028DED101F055FB0028DAD12378CF
:10CC7000DB0602D40A4810F0F3FB102223780821C7
:10CC8000134323700024074A938E0B43938620009E
:10CC9000F8BDC04672240020BC2600206424002079
:10CCA000308103008C5A0020C022C3799200807921
:10CCB0001B0213401843704710B5FFF7F5FF8305BB
:10CCC00001D5024BC01880B200B210BD00FCFFFFBE
:10CCD000031E0AD03F2342891A403E3B0E2A04D04D
:10CCE00000230421103A91425B4101201840704713
:10CCF000031E0AD042893F23002013400100062270
:10CD00000E3B9BB29A4241410B00012018407047F4
:10CD1000031E0AD042893F230020134001000D2248
:10CD20000C3B9BB29A4241410B00012018407047D6
:10CD300070B506000025FFF7EBFFA8420BD03000CE
:10CD4000FFF765FF041EAC4205D03000FFF759FF26
:10CD5000201A45424541280070BD031E05D03F23DF
:10CD600040890340023B584243410120184070472C
:10CD7000031E05D07F2340890340463B5842434170
:10CD8000012018407047031E02D043895B06DB0F69
:10CD9000012018407047031E05D03F2340890340FF
:10CDA0000C3B58424341012018407047031E05D0F8
:10CDB0003F2340890340043B58424341012018402F
:10CDC000704770B50400FFF7F1FF0123051E0BD17A
:10CDD0002000FFF79DFF2B00002805D02000FFF763
:10CDE00087FF01235840C3B20120184070BD031EC5
:10CDF00005D03F2340890340033B58424341012073
:10CE000018407047031E05D03B2340890340013B77
:10CE100058424341012018407047031E07D03F236A
:10CE2000428901211A400023063A91425B410120C8
:10CE300018407047031E0AD042893F230020134048
:10CE400001000722083B9BB29A4241410B0001209E
:10CE500018407047031E05D03F2340890340223B02
:10CE600058424341012018407047F0B589B0029004
:10CE70000C210B3018F0D8FD00250124431C019330
:10CE8000434B290005A81D80FFF797FE05AB0093D3
:10CE90000C26631E03933300621E53433D4FFB1861
:10CEA00059893F2319401AD1019B0135AB4238D82B
:10CEB000E31A01339BB2013B73430198364A704336
:10CEC000DD19A9606A81029A6960DA5102000134B1
:10CED0000C3AA819FEF76CF9A4B2019638E0651B6C
:10CEE000ADB2A5420CD20C236E1E5E43294B290025
:10CEF0009E1900980135FFF760FEADB20096F0E78D
:10CF00000C23039E00255E43224B9819FFF7A2FFD6
:10CF1000A84206D0B8590C210B3018F085FD241812
:10CF2000A4B2FF230134A4B29B009C42B0D90025D7
:10CF300021E0019B661E5E43164BF7187B899B061A
:10CF40000BD121000098FFF738FE00970134A4B2FE
:10CF5000FF239B009C42ECD90DE03800FFF77AFFDD
:10CF60000028F3D00B4B0C21F0580B3018F05CFD6F
:10CF70002418A4B2EAE700210098FFF71EFE05A8D6
:10CF8000FFF745FE024B1880280009B0F0BDC046EF
:10CF900072240020BC260020220200000022F8B5E6
:10CFA00001243F270F4B1A800C23651E5D430E4E54
:10CFB000A8194189394003D11A00FEF7F9F80AE0AF
:10CFC000FFF748FF002806D0A8590C210B3018F0B5
:10CFD0002BFD2418A4B2FF230134A4B29B009C4271
:10CFE000E2D9F8BD72240020BC2600200021F0B553
:10CFF000012487B0194D03A8298003AEFFF7DDFD9A
:10D0000001950C233F22651E5D43154BEF187B896C
:10D01000134205D130002100FFF7CFFD3E000CE0A8
:10D020003800FFF717FF002807D00D4B0C21E858F8
:10D030000B3018F0F9FC2418A4B2FF230134A4B279
:10D040009B009C42DDD900213000FFF7B6FD03A80C
:10D05000FFF7DDFD019B188007B0F0BD72240020B2
:10D06000BC26002070B501240B4D28000026013499
:10D07000A4B22E800A382100FFF79FFD074B0C3524
:10D080009C42F2D131000648FFF797FD0122054B83
:10D090001A80FFF7ABFF70BDC6260020FD0300001D
:10D0A0008056002072240020031E0AD042893F23AC
:10D0B0000020134001000922243B9BB29A424141C7
:10D0C0000B00012018407047031E0AD042893F23FD
:10D0D0000020134001001322103B9BB29A424141B1
:10D0E0000B0001201840704710B50400FFF7ECFF5B
:10D0F00003000120002B02D12000FFF7D5FF012300
:10D10000184010BD70B50400FFF771FE012500281E
:10D1100012D12000FFF776FE00280DD12000FFF786
:10D120007CFE002808D12000FFF7CEFF002803D1A5
:10D130002000FFF73BFE05000120284070BD10B520
:10D140000400FFF777FE03000120002B02D120002E
:10D15000FFF7BAFF0123184010BD10B5021E06D01C
:10D16000438900225B0602D5FFF7AEFF02000123D0
:10D170001A40100010BD011E08D03F234089012134
:10D1800003400A2B02D00F3B594259410122114062
:10D1900008007047031E05D03F2340890340093B28
:10D1A00058424341012018407047031E0AD03F23D4
:10D1B00042891A4000230F2A04D8E9231B02D340D6
:10D1C00001221340012018407047031E05D03F2361
:10D1D000408903400B3B58424341012018407047AF
:10D1E00070B50400FFF7E1FF012500280DD12000F4
:10D1F000FFF7EBFF002808D12000FFF7BCFF002855
:10D2000003D12000FFF7A9FD05000120284070BDD3
:10D21000031E05D03F2340890340013B5842434150
:10D2200001201840704770B50400FFF7F6FD012596
:10D2300000280DD12000FFF7E5FD002808D12000CF
:10D24000FFF7D5FD002803D12000FFF7E1FF05001F
:10D250000120284070BDF8B5037A0400002B00D0EF
:10D260008AE0FFF721FF002800D085E063899B0654
:10D2700000D181E02000FFF73BFD002810D1200005
:10D28000FFF79FFD00280BD02000FFF70DFD0028C1
:10D2900006D0FFF723FC037A013B037200F070F81D
:10D2A0002000FFF721FF002809D12000FFF7BBFF76
:10D2B00000284DD02000FFF7F7FC060030E02000EA
:10D2C000FFF736FC0C260500002D0BD0013D754301
:10D2D0002A4FEF193800FFF72BFC05003800FFF745
:10D2E00075FCF1E72000FFF7B5FD0028DDD02068D0
:10D2F0000C210B3018F098FB05002000FFF7FCFB19
:10D300000C26401980B2013DCFD3013887B270435B
:10D310001A4B181800234381FFF758FC3800F2E736
:10D32000002E26D03000FFF7D9FB0500FFF76FFC79
:10D33000002106002800FFF737FC28000021FFF736
:10D340003CFC2B7A2800013B2B7200F019F8E7E730
:10D350002000FFF7DDFC00280BD02000FFF757FC72
:10D36000002806D000F01EF82000FFF74AFC00F06D
:10D3700019F82000FFF72AFCF8BDC046BC260020A3
:10D3800010B500280AD04389054A9B18F0229BB2A9
:10D3900052014381134201D1FFF75DFF10BDC0462A
:10D3A00000FEFFFF10B5FFF799FB037A013B037204
:10D3B000FFF7E6FF002010BD70B504000D00002C43
:10D3C00005D0013CA300E858FFF7DAFFF7E770BD8E
:10D3D00070B50D001400FFF7D3FF2800FFF7D0FF52
:10D3E0002000FFF7CDFF70BD10B50C00FFF7C8FFA0
:10D3F0002000FFF7C5FF10BDF8B500200C250C4E2E
:10D40000441C68438019A7B2FFF702FF002803D02D
:10D410003800FFF763FB0AE0FF2320009B009C42DB
:10D42000EED10120FFF7FBFB037A01330372F8BD55
:10D43000BC26002070B504680500002C0DD020002B
:10D44000FFF7E5FB06002000FFF79AFF0020864269
:10D4500002D03000FFF742FB286070BD10B5040019
:10D460000800FFF721FC0023984202D0FFF736FBAB
:10D470000300236010BD70B504000EF01EF8050017
:10D480002000FFF77DFF280070BDD0B504000AF032
:10D490004AFE06000F002000FFF772FF300039003F
:10D4A000D0BD70B504000EF099F905002000FFF71B
:10D4B00067FF280070BD0300F0B5213BC3B0050035
:10D4C0000C0016005E2B06D827230B7060708B7043
:10D4D0000023CB7050E00223FF33984213D006DCC8
:10D4E00000280ED0013B984211D1244921E081232C
:10D4F0005B00984209D00423FF33984207D12049AA
:10D5000017E0204915E0204913E0204911E0AF1F42
:10D51000FF3F342F20D8812201AD52001C49280042
:10D520001AF0A9FB812200215200002F05D1320000
:10D53000691820001AF0DAFB1EE00223FF3399423B
:10D54000F5D8685C4B1C002802D11900013FECE7BC
:10D550009142FAD01900F4E732000E4920001AF087
:10D56000C5FBA11C012228000A230FF0FBFB32009F
:10D57000094920001AF0A6FB43B0F0BD4381030027
:10D58000508103003F810300468103004A8103006C
:10D59000D27F0300578103007FAC0300002310B546
:10D5A0004380836F0400002B04D080215A898900B6
:10D5B00052185A81A06FFFF7E3FE206E002803D0B7
:10D5C000FFF7DEFE00232366A06EFFF7D9FE0023DF
:10D5D0002361237610BDF0B5040089B025782800BA
:10D5E00013F014FF002803D02000FFF7A9FAF5E795
:10D5F0002F2D26D1E36F002B23D0E26E9B5C2F2BC7
:10D6000008D12378002BEFD00A2BEDD02000FFF7B4
:10D6100097FAF6E72A2B14D12378002B00D195E353
:10D620002A2B03D02000FFF78BFAF5E7E36F002BDE
:10D63000F8D0E26E9B5C2F2BF4D12000FFF780FA2C
:10D64000D2E723000025643365801D70206EA84258
:10D6500002D0FFF795FE2566E26863689B182200FA
:10D66000013BE3616C32231D23CA23C303CA03C3F6
:10D6700026783300213B26765B2B00D962E3BF4B33
:10D680009B191F3B18780F2800D962E318F0C2F9E4
:10D6900010003201FE015A03AA02BD02CA02D702DB
:10D6A000E3020703F702EF02FF0220030F03340334
:10D6B000202521780B00AB43413B192B06D82000D5
:10D6C000FFF700FA2000FFF73BFAF2E75F29F6D0F8
:10D6D0000B00303B092BF2D92429F0D080235B00CA
:10D6E0006380631CD87F6238152800D931E318F0B5
:10D6F00091F916001F003700570060003003300317
:10D700007E003003300330033003950030033003D4
:10D710003003A600AE00B600DE00F000E700984936
:10D72000200017F043FC9123002800D00FE310E302
:10D730009449200017F03AFC9A23002800D006E311
:10D740009149200017F032FC9523002800D0FEE21A
:10D750008E49200017F02AFC2423002807D1F8E284
:10D760008B49200017F022FC002802D03623FF331B
:10D77000EEE28849200017F019FC9B23002800D016
:10D78000E5E28549200017F011FC20230028EED1A6
:10D790008249200017F00AFC3A230028E7D1D8E29A
:10D7A0007F49200017F002FC8F23002800D0CEE232
:10D7B000CFE27C49200017F0F9FB2E230028D6D1B8
:10D7C0007949200017F0F2FB2C230028CFD17749AC
:10D7D000200017F0EBFB22230028C8D17449200059
:10D7E00017F0E4FB9223002800D0B0E2B1E27149C7
:10D7F000200017F0DBFB1E230028B8D16E49200063
:10D8000017F0D4FB32230028B1D16C49200017F067
:10D81000CDFB9923002800D099E29AE268492000C4
:10D8200017F0C4FB9823002800D090E2654920003F
:10D8300017F0BCFB9723002800D088E289E26249F8
:10D84000200017F0B3FB2623002890D181E25F4926
:10D85000200017F0ABFB3423002888D179E25C4923
:10D86000200017F0A3FB2823002880D1594920006D
:10D8700017F09CFB9423002800D068E25649200052
:10D8800017F094FB9623002800D060E25349200053
:10D8900017F08CFB2A23002800D068E750492000AD
:10D8A00017F084FB3823002800D060E751E24D498F
:10D8B000200017F07BFB3023002800D057E748E218
:10D8C0004949200017F072FB9023002800D03EE267
:10D8D0003FE24649200017F069FB9323002800D05F
:10D8E00035E24349200017F061FB9C23002800D05B
:10D8F0002DE22EE22E2E11D12000FFF721F9237800
:10D90000303B092B08D881235B0063803100200065
:10D91000FFF7D8F8012582E066801AE2302E01D0A8
:10D9200001251AE031002000FFF7CCF82000FFF7B6
:10D9300007F9217820230A009A431300423BDBB207
:10D94000162BEDD82B4A0125DA409543E8D120006B
:10D95000FFF7B8F82000FFF7F3F802232026FF3383
:10D96000638021780B00303B092B45D82000FFF75E
:10D97000A9F82000FFF7E4F8F3E7C046D2800300DF
:10D980005A81030060810300658103006B810300FD
:10D99000748103007C81030083810300868103007E
:10D9A0008F810300948103009A810300A281030008
:10D9B000D5AA0300A6810300EA9F0300A981030002
:10D9C000B4810300B8810300BD810300C48103005A
:10D9D000BB7E0300CB810300D1810300D68103000D
:10D9E000DA81030073B00300E1810300E7810300E3
:10D9F000EB81030001204000002D05D10B00B34353
:10DA0000413B052BB2D90AE02E2908D181235B00C6
:10DA100020006380FFF756F82000FFF791F80223FB
:10DA2000E25E81235B009A4202D0002D0CD190E18E
:10DA300021780B00303B092BF7D82000FFF742F884
:10DA40002000FFF77DF8F3E7217820230A009A43AE
:10DA5000131E452B00D07CE1BD3363802000FFF70F
:10DA600031F82000FFF76CF82178FD230A002B3AEB
:10DA70001A4205D12000FFF725F82000FFF760F8D3
:10DA800021780B00303B092BF4D962E113F06FFBD6
:10DA9000011E206601D160805BE1002203A814F022
:10DAA000A9FC2000FFF74CF82178002900D191E073
:10DAB0008E4200D18EE020005C2900D083E0FFF789
:10DAC0003FF8257828006238162847D817F098FFC5
:10DAD0001146464616464646464646460C46464685
:10DAE0001B46202A25462A002000FFF729F80A2590
:10DAF00060E02000FFF724F808255BE02000FFF736
:10DB00001FF80C2556E02000FFF71AF80D2551E00C
:10DB10002000FFF715F809254CE02000FFF710F86A
:10DB20000B2547E001AF05228B4938001AF0A3F816
:10DB3000752D05D12000FFF703F82000FFF700F84E
:10DB40002000FEF7FDFF23782000BB70FEF7F8FFF2
:10DB500023782000FB70FEF7F3FF23E02B00303B1F
:10DB6000072B24D830230193002301AF20003B7101
:10DB70007D70FEF7E5FF2278022311003039072976
:10DB80000ED82000BA70FEF7DBFF227803231100C5
:10DB90003039072904D82000FA70FEF7D1FF04239A
:10DBA0000022FA5438000FF0C3FDC5B202E0200095
:10DBB000FEF7C6FF29002000FEF784FF290003A816
:10DBC00014F0C0FB70E7FEF77DFF217803A814F086
:10DBD000B9FB66E70698FFF7D3FB2000FEF7B0FF1E
:10DBE0000423C4E52000FEF7D9FF23783D2B00D0A5
:10DBF000AFE00823FF3363802000FEF7A1FF237806
:10DC00003D2B00D0A5E0CB3395E02000FEF7C6FF0A
:10DC100023783D2B01D1122382E02B2B00D098E0FA
:10DC200014237DE02000FEF7B9FF23783D2B01D1BE
:10DC3000D53380E02D2B00D08BE0E7337BE0200054
:10DC4000FEF7ACFF23783D2B01D1DB3373E0262BAD
:10DC50007FD11A2364E02000FEF7A0FF23783D2B3C
:10DC600001D1DD3367E07C2B73D11C2358E0200009
:10DC7000FEF794FF23783D2B6BD1DF335BE0200070
:10DC8000FEF78CFF23783D2B63D1162348E020005C
:10DC9000FEF784FF23783D2B5BD1D9334BE0200086
:10DCA000FEF77CFF23783D2B53D1182338E020006A
:10DCB000FEF774FF23783D2B4BD10623FF3363809F
:10DCC0002000FEF73DFF23783D2B42D1C93332E0DF
:10DCD0002000FEF763FF23783D2B01D10A231FE0CC
:10DCE0003C2B36D1CE3363802000FEF729FF23780A
:10DCF0003D2B2ED10C2313E02000FEF74FFF23789D
:10DD00003D2B01D1CF3316E03E2B22D10E23FF3322
:10DD100063802000FEF714FF23783D2B02D11023EF
:10DD2000FF3308E03E2B14D12000FEF709FF2378D3
:10DD30003D2B05D1D33363802000FEF701FF08E0BF
:10DD4000872304E02000FEF729FF02E082235B0026
:10DD5000638009B0F0BDC046F081030030B5040017
:10DD60000223C05E89B00D0088424BD080235B0047
:10DD7000984212D110222649684619F0B7FF2300B5
:10DD80000022210064331B782031E3180133DA7755
:10DD90006846103219F096FF1DE00423FF3310226D
:10DDA000984215D11B49684619F0A0FF23000022B4
:10DDB000210064331B782031E3180133DA77684699
:10DDC000103219F07FFF1449684619F05DFF02E038
:10DDD0006946FFF770FB2800102204A9FFF76BFBD0
:10DDE0006268E368E5699B18013BE3616A4604AB3E
:10DDF0000A4902200FF012FA2000E561FFF7EBFB61
:10DE0000002003E02000FFF7E6FB012009B030BD51
:10DE1000F5810300F9810300008203000282030000
:10DE200070B5836F86B005000E00002B04D08021F2
:10DE30005A89890052185A81A86FFFF7A1FA310058
:10DE4000684614F058FC2B006C466C3307CC07C3B3
:10DE500006CC06C3A86FFFF793FA337D28002B701A
:10DE600000232B612B76FFF7B6FB06B070BD802236
:10DE70004B8992009B184B810300002210B50400CF
:10DE800064338166428002610276C2611A70026662
:10DE90005A806C3014F0AEFAA06FFFF771FA2000D0
:10DEA000FEF74EFE2000FFF796FB10BD70B50D008B
:10DEB000040014F020FC2B7D2000237570BD10B5EC
:10DEC000C068FFF75DFA10BDF8B506001A20FEF72E
:10DED000A6FE051E03D122480FF0A4FA3EE08022E0
:10DEE0000400438992009B18438133782000002B63
:10DEF00032D0FFF7D9F80921002806D12000FEF71B
:10DF000007FF0421002800D1033100233278002AC2
:10DF100005D0E254013301368B42F7D100E01900FD
:10DF200020000A3014F088F93378002BDDD024204B
:10DF3000FEF775FE071E04D10A480FF073FA2000A1
:10DF40000AE0FEF7D9FD01002000FEF7E5FD200004
:10DF5000FFF716FA3C00C8E7FFF712FA2800F8BDF1
:10DF6000158203004282030010B50300006E0028F2
:10DF700005D08022438992009B18438109E01A0052
:10DF8000643212789A1801322033D0771800FFF7E4
:10DF90009BFF10BD70B50B4B040000220A49586866
:10DFA0000AF0C1FA051E0BD02100012204F0CAFAC2
:10DFB0000400631E9C412900E4B2FFF715FA20001B
:10DFC00070BDC0468C5A0020698203007FB5114C99
:10DFD000114D060003AB02AA216828680DF0A3F9D1
:10DFE000002E01D1266003E028680DF043FA20607E
:10DFF000039B28680193029B6A460093216801AB4A
:10E000000DF091F9009B019A0299039802F088FDA6
:10E010007FBDC0467C24002074240020F0B5194C3C
:10E0200085B0070020680DF0D4F9174D03AB02AAA4
:10E030000600296820680DF076F9029B039AF8180B
:10E040000192002801D0009001E001230093009B81
:10E050009E4200D20096009920680DF02FF901AB86
:10E06000010028606A4620680DF05DF902F0D0FEDC
:10E07000002805D0009B019A0299039802F050FDF8
:10E0800005B0F0BD742400207C24002070B50C4B3A
:10E090001A78002A12D000220A4C1A702068FFF762
:10E0A00079FF00280AD020680AF0D0FA051E05D0B2
:10E0B00002F036FE2068FFF763F9256070BDC046A8
:10E0C000802400207424002070B5074B04001888B9
:10E0D000FEF704FD2100050016F034FC04002800C2
:10E0E000FFF74EF9601E70BD0425002010B5002218
:10E0F0000C0008490AF017FAFFF7D3F901230028AA
:10E1000005D0C30F002C02D0C3171B1ADB0F180059
:10E1100010BDC04671820300F7B5070005200D0051
:10E1200001920093FEF77BFD041E2FD0184A2900B0
:10E1300009F00BFFFFF724F9009B002B18D00320F8
:10E14000FEF76DFD0026051E12D0009BB34207DDD1
:10E15000019AB300D158280004F0CBF90136F4E756
:10E1600029000C4A200009F0F0FE2900FFF73CF9D5
:10E17000002F06D0084A3900200009F0E6FEFFF71C
:10E18000FFF8064B2100186804F0D2F9F7BDC0462D
:10E19000B67E0300817E0300BB7E03006C2400205A
:10E1A00070B5224C0022224960680AF0CEF8051EA4
:10E1B00012D009F02BFF29000600606809F0B5FDB8
:10E1C0002800FFF7DDF8002E06D01A48310002F0D3
:10E1D0007DFC3000FFF7D4F80EF098FC002808D042
:10E1E00002F0BAFD144802F08BFC0822A38E934380
:10E1F000A3860022114960680AF0A7F8051E13D013
:10E2000009F004FF29000600606809F08EFD28006F
:10E21000FFF7B6F8002E07D000223000110003F0FF
:10E2200001FB3000FFF7ACF870BDC0468C5A0020EF
:10E23000768203007D8203008A820300A1820300AC
:10E2400070B50E4C20680DF015F906000C4D2968CC
:10E250008E4212D920680CF0DFFF0A280DD002F0A0
:10E26000D7FD002805D0296820680CF0D5FF02F002
:10E270003DFC2B6801332B60E8E770BD742400205F
:10E280007C24002010B50B4C2168002911D00A4BCA
:10E29000013918680CF0C0FF0A280AD002F0B8FD56
:10E2A000002802D0082002F021FC2368013B2360F3
:10E2B000E9E710BD7C2400207424002070B5040020
:10E2C00002F0A6FD114D124E00280FD028680DF067
:10E2D000D1F831680200286802F04CFC286802F08E
:10E2E000C5FC3A220021200003F09CFA02F018FD40
:10E2F0002868FFF745F88022638992009B186381A4
:10E3000020002C600DF0B6F8306070BD7424002041
:10E310007C24002070B5094B0022094958680AF096
:10E3200002F9051E09D004F07EF80400631E9C412A
:10E330002900E4B2FFF758F8200070BD8C5A002085
:10E340006982030070B50024050002F00EFFFF2271
:10E35000134B1C70134B1C80134B1A70A5420DD02D
:10E360000FF0DAFE041E09D002F0E6FEFEF716FEFC
:10E370000FF0E4FEFEF73AFE02F0F7FE02F09CFF1B
:10E3800002F0E0FC00280AD0002C02D1074802F07D
:10E39000B7FB074802F0B4FB0122064B1A7070BDB0
:10E3A00070240020F8240020711F0020A8820300A0
:10E3B000A87F030078240020F0B5494C85B0019077
:10E3C00020680DF057F8474D019B02902968002BFB
:10E3D00002D0002904D181E0029B8B4269D87DE004
:10E3E000013920680CF018FF03000A3B5A425A41D9
:10E3F00003920A2868D102F00BFD002812D00122F6
:10E400002968206802F0CEFB019B002B61D03648C2
:10E4100002F076FB2B6820685A1E190002F0AAFB56
:10E4200002F07EFC12F0A3FE2E4B07001E68019B3B
:10E43000002B00D0013E002E05D0330000222168C1
:10E4400038000CF002FF029B721C934204D9274B48
:10E45000216838000CF0F9FE02F062FC2068FEF73B
:10E460008FFF019B2760002B02D02B68013B2B60A4
:10E4700002F0CEFC002831D0039B002B0ED029687F
:10E480003A22380003F0CEF9246820000CF0F2FFA5
:10E490002A680100200002F06DFB1FE0019B002BA9
:10E4A00002D0082002F022FB2968206816F050FDF7
:10E4B00014E020680CF0B0FE03000A3B5A425A41B7
:10E4C00003920A2805D196E712F051FE2E68070044
:10E4D000B0E712F04CFE2E680700ACE705B0F0BDC7
:10E4E000742400207C24002075830300FFFFFF7F3D
:10E4F000F8B52B4B070000222A4958680AF013F898
:10E50000051E36D0284B0122196804F01BF8061EA0
:10E5100015D0002F05D0FEF774FB0024A0420AD0CE
:10E5200004E0FEF774FB3C00002804D0FEF7D6FAA6
:10E5300009F0C4FD04003000FEF722FF0AE00400E9
:10E54000002F07D02B682800591E04F034F809F07A
:10E55000B5FD04002800FEF713FF002C09D02000B1
:10E56000FFF7ACFE2000FEF70BFF01220F4B1A70E5
:10E5700014E0002F12D102F04BFC0B4C002802D00B
:10E58000206802F073FB02F0CBFB2068FEF7F8FE78
:10E5900012F0EDFD0022064B20601A60F8BDC04667
:10E5A0008C5A0020698203007424002080240020FB
:10E5B0007C240020F0B5174B85B001901888FEF739
:10E5C0008DFA0100050003A80CF0ADFB0024039BAD
:10E5D00003A8002B15D00CF096FB00220E49070073
:10E5E00009F0A1FF060002F0C2FC019B984200D195
:10E5F000012430003900FEF7F7FE03A80CF06FFB92
:10E60000E5E70CF067FB2800FEF7BAFE200005B036
:10E61000F0BDC046D4560020AEA30300F0B585B0CF
:10E620000190080016001F0009F0F0FC051E04D13F
:10E630000EF06CFA002846D14AE0FEF7D8FB00281D
:10E640001FD0290003A80CF06EFB039B002B13D0F6
:10E6500003A80CF058FB3B00010000903200019829
:10E66000FFF7DCFF04000098FEF78AFE03A80CF019
:10E6700036FB002CE9D100E0012403A80CF02AFBB2
:10E680001CE02800FEF7C9FB041E06D03B00320048
:10E690000199280002F0ECFC09E02800FEF714FDC7
:10E6A000002807D022002100280002F00DFDFEF70F
:10E6B00067FE02E00A480EF0D3FE01242800FEF7B0
:10E6C0005FFE002CB4D10122064B00201A7005E039
:10E6D000054B01201A68054B9A42F4D905B0F0BDEC
:10E6E000788303007024002068240020CB0C0000F5
:10E6F000F0B587B000AFB8607960002A31D000264D
:10E700001568B5422FD06946AB000E33DB08DB003D
:10E71000CB1A9D4614231100F8186E46FEF79EFE94
:10E7200000247B69FB60002B10D0A54209D9631C33
:10E73000FB601423F8180CF0E6FAA40034192060EA
:10E74000FC681423F818FEF775FEEAE71433F8188E
:10E750000CF0C0FAFB68A54205D9A200B350013401
:10E76000F9E71600150033002A007968B868FFF74A
:10E7700055FF040031002800FEF71EFE2000BD46B4
:10E7800007B0F0BDF0B5A14CABB0A14D0290206830
:10E790002E680CF06FFE0190019BB3420AD9310044
:10E7A00020680CF039FD12F031FE071E00D1E9E0BF
:10E7B0000136F1E7029B002B00D1D6E00AAF2168B9
:10E7C0003800FFF754FB00267B88002B19D08221EC
:10E7D0001AB249008A4212D020218B431BB25B2B14
:10E7E00001D0282A00D101365D2B01D0292A02D17F
:10E7F000013E00D204E13800FEF7EDFEE4E7FA2620
:10E80000B6003800FEF7CAFE002E00D0ADE002F0E0
:10E81000FFFA002802D07F4802F072F97E4B1A8876
:10E820000393930702D401227C4B1A70236801934F
:10E8300012F09DFC06000022019905A813F0DAFDF4
:10E8400000223100380013F0D5FD00230193069B10
:10E850000293029A059B934224D205A812F080FCF1
:10E86000029005A813F086FE029B202B02D1019B8B
:10E870000133EBE7029B0A2B04D11900380013F097
:10E8800061FDE2E7019B002B07D02021380013F047
:10E8900059FD019B013B0193F4E70299380013F005
:10E8A00051FDD4E70898FEF76BFD0D98FEF768FD63
:10E8B00002F036FA2068FEF763FD12F058FC0027DC
:10E8C0002060574C3900628830002F6002F0FCFB5A
:10E8D00001940500BE4221D030000CF0CBFDB842BF
:10E8E0001CD0504B03225049586809F01CFE041EEE
:10E8F000BC4213D03A00310003F024FE071E06D0BC
:10E900000100200009F011FA3800FEF739FD31004E
:10E91000200003F0EEFD2000FEF732FD3000FEF790
:10E920002FFD0023019A538002F00CFA002810D02A
:10E930003C4B9C8E38231C400BD13D2002F0D6F876
:10E9400028002300394A172110F046F9314802F017
:10E95000D7F82800FEF714FDFFF722FC0222039BE4
:10E960001B889343039A13804EE002F051FA00286B
:10E9700002D02F4802F0C4F8FFF788FB254802F0C8
:10E98000ADF939E0FFF782FB02F042FA002804D02B
:10E990003A002968206802F005F912F0E8FB2B68BC
:10E9A0000600002B03D0002221680CF04EFC0A2345
:10E9B0000AA930000B7015F0B1FF1E4B2A682168C0
:10E9C00030000CF042FC02F0ABF92068FEF7D8FCF6
:10E9D000266002F01DFA00280ED03A222968300085
:10E9E00002F020FF246820000CF044FD2B68010099
:10E9F0005A1C200002F0BEF82B6801332B6003E0A4
:10EA00003800FEF7CBFD02E72BB0F0BD74240020E8
:10EA10007C240020A87F0300F82400207824002014
:10EA2000802400208C5A002069820300010B020020
:10EA3000A0830300FFFFFF7FF0B5984B85B01A78E5
:10EA400005001C00022A0DD10020013218704F2D44
:10EA500002D05B2D02D104221A7062E10A2D00D08F
:10EA60005FE1F0E0032A1FD100221A70462802D18C
:10EA7000FFF7E6FB55E1482802D1FFF703FC50E120
:10EA80002F206F2D02D06A2D03D12A20FFF7D4FF4B
:10EA900047E12D206D2DF9D02B206B2DF6D00D20C8
:10EAA0004D2D00D03DE1F1E7042A70D100221A700B
:10EAB0000200303AD1B2092903D879498A80052267
:10EAC000CAE7442816D1774C2168002900D128E1F3
:10EAD000754B013918680CF09FFB0A2800D120E122
:10EAE0002368013B236002F093F9002800D118E16C
:10EAF0006E4814E1432818D16B4D28680CF0BAFC1D
:10EB0000684C2168884200D80BE128680CF084FB2F
:10EB10000A2800D105E123680133236002F078F967
:10EB2000002800D1FDE06248F9E0412813D15E4C95
:10EB300020680CF09FFC051E05D15A4B1B689D42B6
:10EB400006D101201CE02068FFF724FA0028F4D148
:10EB50000120404218E0422800D0E2E0524C2068F8
:10EB60000CF088FC051E05D14E4B1B689D420AD156
:10EB7000002005E02068FFF70DFA0028F4D102E03C
:10EB8000FFF7B6FCCDE00120FFF748FAC9E0052AFF
:10EB900039D10300303B092B07D80A23404A91881A
:10EBA0004B43303B1D189580BBE0642803D13C4BA0
:10EBB0009A885A8024E0482806D1394B9B88022B3A
:10EBC0001ED102F069FB1BE07E2819D1344B9B88D3
:10EBD000012B02D1FFF756FB12E0032B03D10020DB
:10EBE000FFF7EAFB0CE0042B02D1FFF729FB07E05B
:10EBF0000020052B02D0062B02D10120FFF7E6F9F9
:10EC0000002323708DE010280BD1274B18680CF0DF
:10EC100031FC002805D10221264A13880B431380BA
:10EC20007FE000232370082D01D07F2D03D1012028
:10EC3000FFF7C2FB75E00D2D02D00A2D06D101E0D1
:10EC4000012323700120FFF79DFD6AE01F2D01D8ED
:10EC5000092D66D1002303AC25706370092D00D106
:10EC6000154CFFF713FA631C1A1B013301925A1E4D
:10EC70001278002AF8D1114E3368002B04DA0A4BBF
:10EC800018680CF0F7FB3060064D33682A689A422A
:10EC900016DB200002F022F836E0C046E121002019
:10ECA000802400207C24002074240020A8830300FA
:10ECB000AC830300F8240020A3830300681F002016
:10ECC00012F055FA2B680600002B04D016490022DA
:10ECD00009680CF0BAFA210030000CF06BF9124F01
:10ECE000124B2A68396830000CF0AFFA02F018F8BD
:10ECF0003868FEF745FB3E6002F08AF8002803D032
:10ED00002968300016F024F9094A019B11688C46E5
:10ED10006344136002F07CF8002802D0200001F068
:10ED2000EFFE05B0F0BDC04674240020FFFFFF7F5A
:10ED30007C24002010B5042206F0B6FB06F056FC39
:10ED40000422524206F0B0FB10BD10B51B4A1378E6
:10ED50001100012B19D11A4B1B681B0715D1194B38
:10ED6000E0241A68F0231000184022420BD1164A02
:10ED700012681A4209D1154A154B1A608022154BA8
:10ED800012021A6001E03028F1D00B68DBB2012BCF
:10ED900012D10B4A126812070ED1F021094A1268EB
:10EDA0000A40402A08D1084A12680A4204D1C12206
:10EDB0008021D200C9058B5010BDC046E00F00F085
:10EDC000E40F00F0E80F00F0EC0F00F0DFFF07C0E9
:10EDD00004050040186C0040F7B500230022040031
:10EDE0000D0016F0C3FF002847D101AA200029001A
:10EDF00006F0C8FB234A244B17F092FF234A244B0A
:10EE000017F03EF8019EF30703D5224A224B17F074
:10EE100087FF721006F048FB06000F0002000B008F
:10EE20002000290017F058FB32003B0017F028F8AB
:10EE300000221A4B17F074FF06000F0002000B00AF
:10EE40002000290017F048FB32003B0017F018F8AB
:10EE50000022124B17F064FF06000F0002000B00A7
:10EE60002000290017F038FB32003B0017F008F8AB
:10EE700000220A4B17F054FF01E00020002103B0EC
:10EE8000F0BDC04679CF2F8F9BE2E23F528E34EF28
:10EE90002AB5DA3FCD3B7F669EA0F63F0000E03FFB
:10EEA000F8B506000F0006F0A1FB02000B000400FD
:10EEB0000D003000390018F0ADF90022184B0600A3
:10EEC0000F0016F05DFF00281FD10022144B300008
:10EED000390016F03BFF00281FD00022104B200005
:10EEE000290017F01DFF06F081FB02000B0016F051
:10EEF000C7FF02000B002000290018F08BF9002248
:10EF0000084B16F023FF002807D02000290000221C
:10EF1000044B16F0B5FF04000D0029002000F8BDD9
:10EF20000000E03F0000F03FF8B514001D000CCCDD
:10EF300006000F0016F0A4FF013D32003B0017F061
:10EF4000EFFE0CCC013D16F09BFF002DF5D1F8BD76
:10EF5000F8B514001D0006000F0003CC32003B0082
:10EF600017F0DEFE0CCC013D16F08AFF002DF5D126
:10EF7000F8BDF7B5284B002206000F0016F080FF01
:10EF8000264A274B04000D0016F0E6FE002807D1A4
:10EF9000224A244B2000290016F0F2FE002804D05B
:10EFA0002000290000F0ACF934E032003B003000D2
:10EFB000390017F0B5FE00221B4B04000D0017F0BE
:10EFC000AFFE062300900191184A30003900FFF788
:10EFD000BFFF02000B002000290017F0A1FE134A1A
:10EFE00004000D003832062330003900FFF79CFF83
:10EFF00002000B002000290017F06EFA32003B00DF
:10F0000017F08EFE009A019B16F03AFF32003B008B
:10F0100016F036FF03B0F0BD0000F03FCD3B7F6639
:10F020009EA0E63F9EA0F63F0000E0BFB083030035
:10F03000F7B50023002204000D0016F087FE061E1F
:10F0400076D16F007F083C4A3C4B2000390016F017
:10F0500097FE0022002809D000232000290016F086
:10F060008FFE002862D10400354D61E0354B200051
:10F07000390016F08FFE2200002828D03B00200027
:10F08000390016F0FDFE06F071FB00222E4B16F043
:10F09000F7FE0B0080210200C905002017F01CFAC2
:10F0A00002000B000020284918F0B4F800220600E6
:10F0B000009120000F000023290016F04DFE3400BF
:10F0C000009D002834D080231B06FD1830E02B0063
:10F0D0002000290017F024FE1C4A02236832009009
:10F0E0000191FFF735FF032306000F0000980199F7
:10F0F000174AFFF719FF02000B003000390017F024
:10F10000EBF9009A019B06000F002000290017F080
:10F1100007FE32003B0017F003FE02000B00200048
:10F12000290016F0ADFE04000D0001E03400064D8C
:10F130002000290003B0F0BDEF39FAFE422E7640E0
:10F140000000F0BF0000E43F0000F03FB083030088
:10F1500030840300F0B5070087B00191002200233E
:10F160003800019916F0F2FD002800D0A9E0594AB4
:10F17000594B3800019916F003FE002807D1574A71
:10F18000574B3800019916F0FBFD00280BD00022E8
:10F1900000233800019916F0F3FD002800D093E019
:10F1A0000400504D92E0019B00225C0064084E4B2D
:10F1B0003800210016F0E4FD002850D04B4A4C4B9B
:10F1C0003800210016F0E6FD002821D00022494B2E
:10F1D0002100380017F0A4FD06F0C8FA0022454BC4
:10F1E00004000D0017F09CFD02000B002000290018
:10F1F00017F096FD00220D0004000023380001994D
:10F2000016F0AAFD002861D080231B06ED185DE0F2
:10F210002100380006F0AAFA0022364B04000D0047
:10F2200017F07EFD2200029003912B00002031494F
:10F2300017F052F902000B000298039917F0EAFF49
:10F2400000220E0004000D0000233800019916F082
:10F2500083FD00283AD080231B06F51836E02300F2
:10F260003A002100380017F05BFD05000E00020097
:10F270000B003800019917F053FD1F4C04900591C5
:10F2800022000323183228003100FFF761FE22001C
:10F29000029003913832032328003100FFF744FE27
:10F2A00002000B000298039917F016F9049A059BC7
:10F2B00017F036FD3A00019B16F0E2FD04000D0048
:10F2C00004E03C00019D01E000240C4D20002900D9
:10F2D00007B0F0BD7DF8B98FCE338640E0EEEC6527
:10F2E0009C4E87400000F0FF0000F03F617B3A6ECB
:10F2F000B72886400000E03F308403000000F07F24
:10F30000F0B5020087B00B0006000F0018F0D6FA27
:10F3100034003D00002800D010E10122894B524208
:10F320003000390016F02CFD002800D006E1002244
:10F3300000233000390016F019FD00280BD0002200
:10F3400000233000390016F001FD0024002800D110
:10F35000F3E07D4DF2E005AA3000390006F012F925
:10F36000059E0400B31C0D00784A042B71D9784B1C
:10F3700016F0F2FC00280CD0013E0022754B200054
:10F380002900059617F046FF002206000F00714B7A
:10F390000FE000226F4B2000290017F03BFF0022F6
:10F3A0006C4B17F037FF002206000F0020002900E9
:10F3B000684B17F0B5FC0022664B16F061FD0200A9
:10F3C0000B003000390017F087F802000B00040032
:10F3D0000D0017F0A5FC604A0223503206000F0012
:10F3E000FFF7B6FD02000B003000390017F098FC63
:10F3F000594A009001916832032330003900FFF729
:10F4000093FD02000B000098019917F065F82200A7
:10F410002B0017F085FC00900191059818F0A4FAD4
:10F420004E4A4F4B06000F0017F07AFC02000B000B
:10F430000098019917F0EEFE02000B002000290051
:10F4400016F01EFD002204000D00464B300039006E
:10F450006AE03F4B16F080FC002809D00122013EF3
:10F4600020002900059606F01FF800223E4B03E01D
:10F470000022200029003C4B17F0CCFE02000B00BC
:10F4800006000F0017F04CFC052302900391374A49
:10F4900030003900FFF75CFD02000B000298039971
:10F4A00017F03EFC314A04000D00303205233000D5
:10F4B0003900FFF739FD02000B002000290017F08A
:10F4C0000BF83B00320017F02BFC059B04000D00ED
:10F4D0000093002B0ED0180018F046FA1F4A204B5C
:10F4E00017F01EFC02000B002000290017F092FE0E
:10F4F00004000D00029803990122524205F0D4FF46
:10F5000002000B002000290017F084FE3B003200AF
:10F5100016F0B6FC009B04000D00002B0ED0180066
:10F5200018F022FA00220F4B17F0FAFB22002B00F2
:10F5300016F0A6FC04000D0000E00D4D200029008F
:10F5400007B0F0BDFFFFEF7F0000F0FFCD3B7F660F
:10F550009EA0E63F0000E03F30840300A80C615C01
:10F5600010D02B3F0030E63F0000F03FB084030096
:10F570000000F87FF0B5020087B00B0004000D001A
:10F5800018F09CF926002F00002800D0F4E001229A
:10F590007B4B52422000290016F0F2FB002800D0DD
:10F5A000EAE0002200232000290016F0DFFB0028FB
:10F5B0000BD0002200232000290016F0C7FB0026F4
:10F5C000002800D1D7E06F4FD6E005AA200029001F
:10F5D00005F0D8FF059E0400B31C0D006A4A042BF9
:10F5E00054D96A4B16F0B8FB00280CD0013E00221B
:10F5F000674B20002900059617F00CFE002206003C
:10F600000F00634B0FE00022614B2000290017F030
:10F6100001FE00225E4B17F0FDFD002206000F00E8
:10F62000200029005A4B17F07BFB0022584B16F0A4
:10F6300027FC02000B003000390016F04DFF0200DD
:10F640000B0006000F0017F06BFB524A02235832E2
:10F6500004000D00FFF77CFC02000B0020002900D5
:10F6600017F05EFB4B4A009001917032032320009B
:10F670002900FFF759FC02000B000098019916F0D1
:10F680002BFF32003B0017F04BFB4AE03F4B16F0DC
:10F6900063FB002809D00122013E200029000596C5
:10F6A00005F002FF00223C4B03E00022200029006D
:10F6B000394B17F0AFFD02000B0006000F0017F0EA
:10F6C0002FFB364A04000D000832052330003900B4
:10F6D000FFF73EFC02000B002000290017F020FB82
:10F6E0002E4A029003910523383230003900FFF78B
:10F6F0001BFC01220090019152422000290005F0DC
:10F70000D3FE009A019B04000D000298039916F0A5
:10F71000E3FE32003B0017F003FB22002B0017F042
:10F7200079FD1F4A1F4B04000D0017F0F9FA1C4A1F
:10F73000009001911B4B3000390017F0F1FA009A4C
:10F74000019B16F09DFB02000B002000290016F023
:10F7500097FB02000B003000390016F091FB04000B
:10F760000D00059818F000F922002B0016F088FB18
:10F7700006000F0000E00C4F3000390007B0F0BD6C
:10F78000FFFFEF7F0000F0FFCD3B7F669EA0E63FCE
:10F790000000E03FB08403000000F03F308503002C
:10F7A000F80BAE941D55DC3F0000F87FF0B5020069
:10F7B00085B00B0004000D0018F080F826002F0023
:10F7C000002800D0B4E001225B4B52422000290007
:10F7D00016F0D6FA002800D0AAE00022002320006C
:10F7E000290016F0C3FA00280BD0002200232000C5
:10F7F000290016F0ABFA0026002800D197E04F4F01
:10F8000096E003AA2000290005F0BCFE4C4A4D4BAF
:10F8100004000D0016F0A0FA00280AD0039B012274
:10F82000013B20002900039305F03EFE0022464BD9
:10F8300003E0002220002900434B17F0EBFC0200FC
:10F840000B0006000F0017F06BFA404A0090019180
:10F850000623603230003900FFF77AFB02000B000C
:10F860000098019917F05CFA394A04000D0006234C
:10F87000183230003900FFF757FB02000B00200060
:10F88000290016F029FE3B00320017F049FA012248
:10F8900004000D0000980199524205F005FE020097
:10F8A0000B002000290017F0B5FC04000D00020039
:10F8B0000B003000390016F0E3FA264A264B17F009
:10F8C0002FFA002200900191244B2000290017F00C
:10F8D00027FA009A019B16F0D3FA04000D000022CB
:10F8E0001E4B3000390017F01BFA22002B0016F0D7
:10F8F000C7FA060003980F0018F036F8184A194B9B
:10F9000004000D0017F00CFA32003B0016F0B8FAB4
:10F9100006000F000022144B2000290017F000FA07
:10F9200032003B0016F0ACFA06000F0000E00F4F6B
:10F930003000390005B0F0BDFFFFEF7F0000F0FFA1
:10F94000CD3B7F669EA0E63F0000F03F3085030080
:10F95000B0850300651CCA4D2AF6463F00C0DB3F58
:10F96000CCFBE77D424D303F0040D33F0000F87FA5
:10F970000348044B0840C018411E88417047C046E8
:10F980000000F07F00001080F0B5002285B0002359
:10F9900005000C0016F0DAF9002800D0C8E02A00B3
:10F9A00023002800210017F089FF002800D0BFE0C5
:10F9B00028002100FFF7DCFF002800D1B3E000237E
:10F9C00000222800210016F0C7F90123002804D0E6
:10F9D00080231B06E41801235B4201930022564B4F
:10F9E0002800210016F0CCF9002800D09EE0534BEF
:10F9F000534A2800210016F06FFD05F0F7FD0322A1
:10FA0000524206000F0005F04FFD05F0EFFD032206
:10FA100005F04AFD0B0002003900300017F0FAFB38
:10FA200017F06CFF03000090DB070AD503000133D9
:10FA30000093300039000022424B16F021FA0600F4
:10FA40000F00A0223D4BD2053000390017F068F9B5
:10FA500002000B002800210017F0DCFBC02204008C
:10FA60000D00D205384B3000390017F059F902006B
:10FA70000B002000290017F0CDFB344A04000D00D4
:10FA8000334B3000390017F04BF902000B00200017
:10FA9000290017F0BFFB02000B0005000C0017F057
:10FAA0003FF92C4A2C4B06000F0016F069F900288C
:10FAB00027D02A4A0223483230003900FFF748FA9B
:10FAC00002000B003000390017F02AF9234A029097
:10FAD00003916032042330003900FFF725FA020059
:10FAE0000B000298039916F0F7FC2A00230017F088
:10FAF00017F902000B002800210016F0C1F90500DB
:10FB00000C00009B9B0707D52A0023000020144906
:10FB100016F0E2FC05000C00019B013308D18023A4
:10FB20001B06E41804E005000E4C01E000252C0043
:10FB30002800210005B0F0BD0000D041FB21E93FC5
:10FB4000182D44540000F03FB410413E075C1433BC
:10FB500026A6813C9B2BA1869B84063DB085030095
:10FB60000000F0BF0000F87FF0B5020085B00B0088
:10FB700006000D0017F0A2FE002800D0D3E03000F0
:10FB80002900FFF7F5FE002800D1C7E0002200237E
:10FB90003000290016F0E0F8002802D080231B0670
:10FBA000ED180022624B3000290016F0E9F8002819
:10FBB00000D0B6E05F4B604A3000290016F08CFCA4
:10FBC00005F014FD042252420090019105F06CFCF6
:10FBD00005F00CFD042205F067FC02000B00009804
:10FBE000019917F017FB17F089FE0400C30708D529
:10FBF000009801990022514B16F042F900900191B2
:10FC0000013407231C40063B0393032C02DD023B17
:10FC1000043C0393012C02DD039B5B42039380228F
:10FC200000980199D205434B17F07AF802000B00B7
:10FC30003000290017F0EEFA002206000F000098AD
:10FC400001993F4B17F06CF802000B0030003900AF
:10FC500017F0E0FA3B4A06000F00009801993A4B72
:10FC600017F05EF802000B003000390017F0D2FAEE
:10FC700002000B000090019117F052F8013C0600C1
:10FC80000F00012C16D802000B000098019917F004
:10FC900047F8052304000D002C4A30003900FFF717
:10FCA00057F902000B002000290017F039F8009ADC
:10FCB000019B28E00122524205F0F6FB32000400CD
:10FCC0000D003B003000390017F02AF81F4A009061
:10FCD00001910523303230003900FFF739F9220055
:10FCE0002B0006000F000020144917F093FA320091
:10FCF00004000D00009801993B0017F011F8020074
:10FD00000B002000290016F0BBF8039B06000D0035
:10FD1000013308D180231B06CD1804E006000C4DEA
:10FD200001E0002635003000290005B0F0BDC046D6
:10FD30000000D041FB21E93F182D44540000F03F62
:10FD40002D44643E7051CC989846E83C30860300C0
:10FD50000000F87FF0B5002285B0002306000D00FA
:10FD600015F0F4FF002800D0DAE032002B0030005C
:10FD7000290017F0A3FD002800D0D1E030002900B1
:10FD8000FFF7F6FD002800D1C5E000230022300077
:10FD9000290015F0E1FF0123002804D080231B0671
:10FDA000ED1801235B42039300225F4B30002900D2
:10FDB00015F0E6FF002800D0B0E05C4B5C4A300054
:10FDC000290016F089FB05F011FC04225242009034
:10FDD000019105F069FB05F009FC042205F064FBC4
:10FDE00002000B000098019917F014FA17F086FD35
:10FDF0000400C30708D50098019900224D4B16F066
:10FE00003FF800900191013407231C40032C03DDCF
:10FE1000039B043C5B420393802200980199D20526
:10FE2000424B16F07DFF02000B003000290017F056
:10FE3000F1F9002206000F00009801993E4B16F0E0
:10FE40006FFF02000B003000390017F0E3F93B4A66
:10FE500006000F0000980199394B16F061FF02006F
:10FE60000B003000390017F0D5F902000B000090AC
:10FE7000019116F055FF013C06000F00012C29D816
:10FE80000122524205F010FB320004000D003B003D
:10FE90003000390016F044FF2A4A009001910523F2
:10FEA000303230003900FFF753F822002B000600F3
:10FEB0000F0000201F4917F0ADF9320004000D00BB
:10FEC000009801993B0016F02BFF02000B00200068
:10FED000290015E002000B000098019916F020FFA0
:10FEE000052304000D00174A30003900FFF730F8F1
:10FEF00002000B002000290016F012FF009A019B5F
:10FF000015F0BEFF039B06000D00013308D18023CE
:10FF10001B06CD1804E006000B4D01E0002635005D
:10FF20003000290005B0F0BD0000D041FB21E93FC1
:10FF3000182D44540000F03F2D44643E7051CC987D
:10FF40009846E83C308603000000F87FF0B51600C4
:10FF500091B0009307000C000022002330000099AC
:10FF600015F0F4FE002801D000F0C4FC3A00230094
:10FF70003800210017F0A2FC002801D000F0BFFCDF
:10FF80003200009B3000009917F098FC002801D047
:10FF900000F0B2FC0022B94B3000009915F0D6FEFB
:10FFA000051E01D000F0ABFC30000099FFF7E0FC2B
:10FFB00000220390002812D1B04B3800210015F028
:10FFC000C5FE051E01D000F09DFC0022AC4B3800A0
:10FFD000210015F0BBFE00280AD000F094FCA74BCE
:10FFE0003800210015F0B2FE002801D000F08DFC91
:10FFF0000122A44B52423000009915F0CBFE00289C
:020000022000DC
:1000000033D000229D4B3800210015F0B9FE0028A6
:1000100075D1002200233800210015F0B1FE002820
:100020000BD00022954B3800210015F095FE0028DA
:1000300003D00025290000F0ADFC0022904B3800D1
:10004000210015F089FE002859D100228C4B380080
:10005000210015F095FE002807D00022002338006B
:10006000210015F079FE0028E3D10122864B52428F
:100070003000009915F07AFE00282FD000227F4B27
:100080003800210015F07CFE0028D2D10022002388
:100090003800210015F074FE002807D00022774BAD
:1000A0003800210015F058FE002828D10022744B9A
:1000B0003800210015F050FE0028BAD10022704B04
:1000C0003800210015F05CFE002807D00022002334
:1000D0003800210015F040FE002810D10122694BA4
:1000E00052423800210015F055FE00280AD00022A7
:1000F00000233000009915F043FE002899D0002518
:1001000000F047FC3000009905F070FA03900A9166
:1001100002000B003000009915F018FE002801D0F5
:1001200000F0F5FB050003900122574B52423800C6
:10013000210015F01BFE00281BD0002200233000F8
:10014000009915F01DFE002806D0039B002BD6D089
:1001500000254E4900F01EFC0022002330000099CB
:1001600015F0FAFD002804D0039B002B00D160E7B6
:10017000BCE3002200233800210015F0F7FD002821
:1001800024D0002200233800210015F0DFFD0028D4
:1001900016D0002200233000009915F0DDFD002864
:1001A00002D0002CD1DBAAE7002200233000009906
:1001B00015F0E6FD002800D196E3002CD4DB38E7EB
:1001C000002D00D19FE301230A9303E0002D00D10D
:1001D000BEE30A903800210005F008FA02000B0087
:1001E0003800210015F0B2FD002800D114E1009B79
:1001F00000225D003000264B690815F0ADFD002897
:1002000000D109E10099300017F078FB00220500C9
:1002100000233800210015F099FD002808D0002D9A
:1002200000D172E300DA6AE7EB0700D567E300E785
:10023000002D00D169E36B1C07D13A002300002098
:100240000E4916F049F90500A4E300220023380006
:10025000210015F081FD002806D080231B06E4183C
:1002600001235B42009300E000900120002D11DA91
:100270006B42039301235B420A930DE00000F03FC1
:100280000000F0BFFFFFEF7FFFFFEFFF0000F0FF78
:100290000000E04003950A90039B009A03400493FA
:1002A0005B421A40009238000FAA210005F06AF95B
:1002B0000F9E039B06900791701E5843002803D0A1
:1002C00003004033802B32D906980799AD4AAE4BD4
:1002D00016F0A0FFAB4A0890099106980799AA4B1F
:1002E00015F0CEFD02000B000898099916F0F4F8FD
:1002F000A64AA74B16F014FD0022A64B16F08AFF63
:1003000006900791300017F02FFB02000B000698B3
:10031000079915F0B5FD06900791280017F024FB0A
:1003200002000B000698079916F0FAFC01E017F09E
:100330001BFB994A994B16F0F3FC974A984B050022
:100340000E0015F01DFD069000285BD1954A964BD6
:100350002800310015F000FD002843D18E4A934B50
:100360002800310015F0F8FC00280CD00A9B01335E
:1003700009D123003A0000208D4916F0ADF8012381
:1003800007000C000A93049B002B02D03D002600BE
:1003900016E0049D864E13E03A0023003800210049
:1003A00016F0BEFC0122039B07000C00134207D08D
:1003B00002000B002800310016F0B2FC05000E0010
:1003C000039B5B100393039B002BE5D10A9B013336
:1003D0000AD12A0033000020754916F07DF8050087
:1003E0000E0001E0069D2E00009B3100002B00D185
:1003F000D0E2002200232800310015F0A7FC0028DD
:1004000006D073E2009B002B00D1C1E20025694EAB
:1004100080231B06F118BDE20A9B002B03D00123A9
:10042000640064080A930022614B3800210016F032
:10043000F1FE009B02005B005B080D00049006913A
:100440000B9330000B00009916F06AFC0C914900E8
:100450004B086D0008900D93574A584B0498690853
:1004600015F084FC002807D00022514B30000B9976
:1004700015F07CFC002811D14F4A504B08980D997B
:1004800015F074FC002800D1ACE00022484B30008D
:100490000B9915F07FFC002800D1A3E00099002201
:1004A000474B300016F0B6FE049A069B16F038FC57
:1004B0000022444B16F010F8434A444B15F0E0FC80
:1004C000049A069B16F02CFC002204000D00404B01
:1004D0000099300016F09EFE02000B00200029005B
:1004E00016F01EFC3B4A3C4B15F0CAFC049A069BD6
:1004F00016F016FC002204000D00384B0099300065
:1005000016F088FE02000B002000290016F008FCFF
:10051000304A334B15F0B4FC049A069B16F000FCED
:10052000802304000D0000220099DB05300016F046
:1005300071FE02000B002000290016F0F1FB0022E2
:10054000144B15F09DFC049A069B16F0E9FB002263
:1005500004000D00164B3000009916F05BFE0200FF
:100560000B002000290016F0DBFB089A0C9B16F00C
:10057000D7FB089A0C9B15F083FC00220C4B15F05E
:100580007FFC9FE1CD3B7F669EA0E63FE69D3F332B
:100590004F5007400000E03FEF39FAFE422EE63FA1
:1005A000422E864052302DD5104987C0421E86C04B
:1005B0000000F03F0000F07FFCA9F1D24D62503FF7
:1005C0000000144000808640111111111111813F6B
:1005D00000001040555555555555A53F00000840A1
:1005E0005555C53F0FAA2100380004F0CBFFD94A6A
:1005F000D94B0490059115F0B9FB0924002800D1CE
:10060000083C271DD54DFB00EB181A6E5B6E049855
:10061000059915F0ABFB002800D03C000498059923
:10062000A71CFB00ED182A6E6B6E15F09FFB0028CF
:1006300000D03C0004980599C94ACA4B15F0AAFBA2
:10064000002801D001246442671CC44AFB00D3186F
:100650001C6E5D6E0498059922002B0016F0DAFDE1
:10066000C14A7B10DB00D3189A6EDB6E16F0D2FD08
:1006700022002B0015F030FF02000B0004900591C2
:1006800016F04EFBB94A069007910498059930324E
:100690000323FEF75DFC02000B000698079916F095
:1006A0003FFBB24A04000D00049805995032042320
:1006B000FEF73AFC02000B002000290015F00CFFA9
:1006C000049A059B16F02CFB012204000D000698ED
:1006D0000799524204F0E8FE02000B0020002900B6
:1006E00016F098FDA24AA34B04000D0016F018FB6B
:1006F00002000B002000290015F0C2FB9C4A0400F8
:100700000D00049805999B4B16F00AFB02000B00A4
:100710002000290015F0B4FB0B0002000498059995
:1007200015F0AEFB08900991784217F01DF90422EC
:10073000524204F0B9FE04000D000F9817F014F9AE
:1007400022002B0015F09CFB0690079130000099C9
:10075000FEF7F0FA0490059102000B0030000099BA
:1007600016F058FD069A079B16F0DAFA089A099BCC
:1007700004000D003000009916F0D2FA02000B00C0
:100780002000290015F07CFB04000D00FEF7D2FAD2
:1007900006000F0002000B002000290016F03AFDB1
:1007A000049A059B009001910698079916F0B8FAF3
:1007B00032003B0015F064FB04000D00FEF7BAFAAE
:1007C00002000B0006000F002000290016F022FD99
:1007D00002000B000098019915F052FB049005915E
:1007E000FEF7A8FA0B0000900191020039003000DA
:1007F00015F046FB042204F057FE00225E4B040075
:100800000D0015F0BDFA002804D00A9B002B00D083
:100810009BE474E40022594B2000290015F09CFA57
:10082000002805D00A9B002B00D09DE4FFF701FCB7
:100830002000290017F062F8009A019B0400049838
:10084000059916F0E7FC0022002306000F0015F0C2
:1008500097FA002801D10F9409E0300039000134E3
:100860000022474B0F9416F0D5FC06000F003F4ABC
:100870000623703230003900FEF76AFB0F9A0F230F
:10088000D443E50FD4171C40A41824112B1900934E
:100890001B019A1A314BD2009A18146E556E0B0038
:1008A00002003900300016F03BFA22002B0016F04F
:1008B00037FA02000B002000290015F0E1FA009A37
:1008C00004F0F2FD0A9B05000C00002B18D0039BDE
:1008D000002B15D00022002315F038FA002805D18E
:1008E00080231B06E11855E005000EE0802100255D
:1008F00009064FE0002508E0350000994AE03D0078
:10090000210047E0039D1F4944E01F4942E0009B4E
:1009100000225D0069081D4B300016F001FA04F05A
:1009200065FE0A9B049005915D000022174B039819
:10093000690816F0F5F9049A059B15F007FA434289
:10094000584101234042034003930125FFF7ECFB8C
:100950000A9568E5295448DD07ABE53F308603007A
:10096000DA90A4A2AFA4EE3FB08603003087030064
:10097000F80BAE941D55DC3F80FFCF4000C8D0C0BF
:100980000000B03F0000F87F0000F03F0000E03FB3
:100990001D000249280011B0F0BDC0460000F07FE4
:1009A000F7B5154B019206000F0000220199186857
:1009B00007F0B9FD051E1DD00022104907F0B3FD58
:1009C000041E13D03000019B0D4A39000CF050FB7F
:1009D0002000FCF717FA002805D03B003200102158
:1009E00020000EF0F9F839000648B0472900200031
:1009F000FCF7FAFCF7BDC0468C5A0020A97D030025
:100A0000188803000389030070B50A4B0100032214
:100A1000586807F088FD0400051E05D0037A0133ED
:100A20000372FCF769F805002000FCF7A9FC280018
:100A300070BDC0468C5A0020F7B5150001930F4BCE
:100A400006000F0001222900186801F07BFD041E3A
:100A50000DD0FCF739FB002809D0019B9C4206D041
:100A60002300074A390030000CF002FB05E03B0090
:100A70003200132128000EF0AFF8F7BD8C5A002089
:100A8000E2A90300F7B50D000400170003210C4A8A
:100A900018000AF0BFFC06003B0029000090094A3C
:100AA00020000CF0E5FA3000FCF76AFC2900002376
:100AB000089A2000FFF7C0FF29000348A047F7BDB0
:100AC000FFFFFF7F22880300038903000FB407B5EF
:100AD00004AB04CB0021044801930CF073F903B07C
:100AE00008BC04B01847C046010B020010B5034B08
:100AF0000100187812F08CFD10BDC046721F002056
:100B000010B504002378002B09D00A2B02D10D2048
:100B1000FFF7ECFF2078FFF7E9FF0134F2E710BDA3
:100B2000F8B505000C0017001E00BD4204D20D48A8
:100B3000FFF7E6FF0135F8E7BD4204D90A48FFF7A1
:100B4000DFFF013DF8E7B44204D20848FFF7D8FFC1
:100B50000134F8E7B44204D90548FFF7D1FF013C5E
:100B6000F8E7F8BDAC830300A88303002D880300D9
:100B70003188030030B5040085B0150091420FD0D4
:100B80006B4601AA0AF0CFFB02AB03AA29002000A2
:100B90000AF0C9FB039B029A01990098FFF7C0FF76
:100BA00005B030BDF0B5050085B0019202AB03AAD7
:100BB0000AF0B9FB039928000AF0E2FB0600029C48
:100BC000B44204D82020FFF791FF0134F8E7002455
:100BD000B44204D00820FFF789FF0134F8E7280069
:100BE0000AF0F7FB039B00905C1C009B9C421FD803
:100BF0001A48FFF785FF210028000AF0C1FB0026F4
:100C00000700BE4204D02020FFF770FF0136F8E74E
:100C10000026BE4204D00820FFF768FF0136F8E73F
:100C2000019B002B02D00E48FFF76AFF0134DCE77E
:100C3000039B5C1C009B9C4204D80A48FFF760FFA2
:100C40000134F7E70124029B9C4204D20648FFF7D7
:100C500057FF0134F7E705B0F0BDC0462D8803000B
:100C60007583030031880300AC830300F7B50700E8
:100C70000AF0AFFB04000190002C2AD021003800BC
:100C80000AF07EFB019B050000269C4201D0002655
:100C900006E0AE42FBD00820FFF728FF0136F8E758
:100CA000AE4204D02020FFF721FF0136F8E70026EE
:100CB000AE4204D00820FFF719FF0136F8E7012CF7
:100CC00005D90448FFF71CFF0348FFF719FF013C53
:100CD000D2E7F7BD758303003188030070B50D4C72
:100CE0000500E268002A07D10B4B2000196811F0BB
:100CF00081FB200011F05FFB2978002908D020003B
:100D000011F020FB054A0135136801331360F3E746
:100D100070BDC0468824002074240020681F002075
:100D200010B5064CE068002803D0FCF729FB00232F
:100D3000E3600122024B52421A6010BD8824002059
:100D4000681F0020034B1888032318404342584172
:100D5000C0B27047F824002070B50E4B1C78002CF0
:100D600016D101261E70FFF7EDFF002810D00A4DA6
:100D7000286800280CD0094B22001968FFF7FAFEFA
:100D8000286832002100FFF70DFF0820FFF7AEFEB4
:100D900070BDC04678240020742400207C240020EC
:100DA0007FB5184C0500237883422AD096239B01F7
:100DB0000193FF2301A90B714B718B71F73BCB7131
:100DC000012200234A720B728B7213F08FF9FFF726
:100DD000C3FFFFF7B7FF002806D0280012F0DCFAA7
:100DE00001000948FFF772FE26782570FFF7AAFF79
:100DF000002806D0300012F0CFFA01000348FFF7B8
:100E000065FE7FBD721F0020358803003C8803000B
:100E100010B5FFF797FF0023984203D00120034B42
:100E20001B7843400120184010BDC04678240020A4
:100E3000036804491B021B0A00228B4200D1C278BE
:100E400010007047444556001F2342090349920091
:100E500003405058D840012318407047FC2400201C
:100E6000002310B50C1E03701F2C08D844330370E8
:100E7000411C3A3B012220000BF074FF03E00822E2
:100E8000014916F0F8FE10BD73B0030030B50578C7
:100E90000300422D1AD14278542A37D182784E2A43
:100EA00034D1C2781120002A60D0312A1CD0322AD5
:100EB00002D11A79122027E0332A02D11A7913209D
:100EC00022E0342A22D11A7914201DE04C2D1DD1A4
:100ED0004278452A1AD18278442A17D1C27815203F
:100EE000002A43D0312A01D11A790DE0322A02D1E9
:100EF0001A79162008E0332A02D11A79172003E064
:100F0000342A03D118201A79002A2FD02A00413A16
:100F1000FF20072A2AD85C78303CE2B2092A25D87B
:100F20009978002903D12300442D1FD11DE03039C9
:100F3000CAB2092A1AD8DA78002A04D10A32130070
:100F400063435B180CE01B79002B0FD1303AD3B20E
:100F5000092B0BD864230A20634341435B189B1879
:100F6000FF20442D02D11F2B00DCD8B230BD10B5BC
:100F70000400FCF7A9F8002806D06379002B03D100
:100F80002000FFF783FF0AE02000FCF70EF90300C2
:100F9000FF20002B03D020000AF020FCC0B210BDBF
:100FA00070B50400FFF7E3FF05002000FCF7E8F947
:100FB000280070BD00231F2804D8034B8000C35CA9
:100FC000581E834118007047F3B0030070B5040049
:100FD0000D00FFF7EFFF00280DD02000FFF734FFD2
:100FE000002803D10121200013F056FB2900200026
:100FF00013F0B8FB03E0024901200CF00FF970BDBB
:101000004388030010B50A4B1A7D002902D0104313
:10101000187501E082431A75064A1078FF2805D03A
:10102000197D4B1E9941C9B2FFF7D0FF10BDC046D4
:1010300088240020711F002070B50500FFF7BAFF5B
:10104000041E0CD02800FFF7FFFE002803D1032167
:10105000280013F021FB280013F074FB04E00120AA
:1010600002490CF0DBF8200070BDC0464388030045
:10107000F0B5382695B0134C06AD070003910492E5
:10108000210032002800059316F0F5FD0123002110
:10109000A386059BA160E16221630193049B039AEF
:1010A000009338000B0006F00FF80700A38E320003
:1010B0009BB229002000AB8616F0DDFD380015B08C
:1010C000F0BDC0468C5A0020F0B5AFB00EAD0E009A
:1010D000010028001400FCF7CAFE9E236B441C800C
:1010E000144C38222100684616F0C5FD0123A56086
:1010F000A386371E05D000233000E3620CF01CF9F4
:10110000070003F0A5F80600002F01D00CF0FAF854
:101110002800FCF743FA6A46A38E69469BB2938681
:101120002000382216F0A7FD301E01D006F0C6FFC1
:101130002FB0F0BD8C5A002070B50025044C6068BB
:10114000FCF71EF920686560FCF71AF9256070BD90
:101150008C5A002010B5FFF7EFFFFCF74DF9037A2A
:10116000013B0372FCF70CF910BD10B5FCF744F914
:10117000044C05220449206007F0D5F90123606082
:10118000A38610BD8C5A00205088030010B5084B70
:1011900004000022186807F0C6F9031E06D0041BDD
:1011A00063425C41E4B2FCF7EBF82300180010BD89
:1011B0008C5A002070B5154B0100060001221868FA
:1011C00007F0C3F8051E20D006F020FF041E0DD145
:1011D000310001F0ADFE041E04D12800FCF7D0F868
:1011E000200012E00100280007F009F90122084957
:1011F000200007F0AAF806000100200003F0E8FA3A
:1012000020002900FCF7F0F8300070BD8C5A002057
:1012100090880300F8B505000800FFF7CBFF060033
:101220000520FBF7FCFC041E04D13000FCF7A8F8F5
:1012300020002CE0002D0BD0280012F035F80028FB
:1012400006D044232370013363701133A370E07020
:10125000300006F0DBFE070001000D4A200006F01A
:1012600074FE32003900FCF7B3F82000002D0ED0D8
:10127000084B29000122186807F067F8051E02D004
:10128000210007F0BCF82000FCF77AF82800F8BD30
:10129000528803008C5A002010B5FFF75DFDFFF760
:1012A0003FFD044C2068FCF76BF80FF060FF2060F6
:1012B00010BDC04674240020F0B50024514B85B009
:1012C00003201C70FBF7ABFC4F4B18600FF04FFF77
:1012D0004E4B18604E4B1C604E4B1C80FFF720FDA0
:1012E00004214D4A4D4B4E48DC6013888B431380DC
:1012F000FF234C4A13704C4A1370FFF785FB4B4B8E
:1013000018804B48FFF780FB4A4B4B4A18804B4BE9
:101310004B4FD2584B4B4C4D14C301224B4B5242B6
:101320001A6039002200686807F0FDF8414B061E7C
:101330000193A6420AD022002100FFF7C5FE31002A
:10134000FCF752F83900686807F04AF8019B1888E2
:10135000002824D0FBF7C2FB0400010003A809F019
:10136000E2FC039B03A8002B14D009F0CCFC002264
:101370003749070007F0D7F80600FFF7F8FD01210D
:1013800012F0F8FF30003900FCF72EF803A809F03E
:10139000A6FCE6E709F09EFC2000FBF7F1FF002227
:1013A0002C49286807F0BFF8041E0FD0FFF7CAFCCD
:1013B000002802D02848FFF7A3FB002321001A00D1
:1013C0001800FDF72BF92000FBF7DAFF0022234974
:1013D000286807F0A8F8041E11D00022204907F061
:1013E000A2F8051E08D0002301001A001800FDF71E
:1013F00015F92800FBF7C4FF2000FBF7C1FF05B07B
:10140000F0BDC046642400206C2400207424002019
:101410007C24002082240020F8240020882400203E
:101420005C880300711F0020701F0020042500202D
:1014300063880300D456002000B00040040500007B
:101440008A880300F02400208C5A002068240020A1
:10145000AEA303006B88030072880300C0A70300DB
:1014600087880300F0B589B0039018000E001C00B7
:10147000049200F055FE2100059006A809F053FCE7
:10148000069B06A8002B78D009F044FC050006A8AE
:1014900009F039FC059B0400002B06D139492800CE
:1014A00006F04EFF002806D119E02800059B98475A
:1014B0000028F3D059E0344A0021049809F0AAFF2B
:1014C000071E52D0314909F075FD039823003A00F8
:1014D0003100FFF7C7FF3800FBF752FF45E001225C
:1014E0002B49280006F0EAFE002828D02000FBF750
:1014F0007EFC00281BD0210007A809F014FC079BE4
:1015000007A8002B10D009F0FEFB070000902B006D
:10151000049A31000398FFF7B5FA3800FBF730FF63
:1015200007A809F0DCFBEAE709F0D4FB1DE0009412
:101530002B00049A31000398FFF7A4FA15E020006D
:10154000FBF721FC071E10D1049B124A31000398BF
:1015500000950BF08DFD3B00310003982200FFF752
:101560006BFA31000C48039B984720002900FBF7D9
:101570003BFF06A809F0B3FB82E709F0ABFB09B01B
:10158000F0BDC04690880300FFFFFF7F8F880300F7
:101590009A8803009E88030004890300F0B51E00AA
:1015A00087B0284B05920400002218680D000599A9
:1015B00006F0CBFE039006F029FD071E3CD0002E5E
:1015C00005D00300039A29002000FFF74BFF0022FB
:1015D0001D49380006F0A7FF002204901B4938007F
:1015E00006F0A1FF049B0600002B01D100281ED0AD
:1015F00004980AF0F3F8002801DC9620800100909E
:10160000059B2000124A29000BF032FD3000FBF749
:10161000F9FB002808D029000E48A0472B00220023
:10162000102130000DF0D8FA29000B48A0473A00ED
:1016300031000498FBF7CCFE0398FBF7A1FE07B03E
:10164000F0BDC0468C5A0020A7880300A97D030086
:10165000B18803002A88030003890300F8B5274EE8
:10166000040033880D001700DB0701D52448A0478C
:10167000244B1B78FF2B04D0234A290020000BF0B9
:10168000F7FC224B1B78FF2B04D0214A29002000B5
:101690000BF0EEFC33885B0702D529001D48A047FC
:1016A0003B001D4A29002000FFF778FF162011F0AB
:1016B00073FE3B00020029002000FFF76FFF222687
:1016C000300011F069FE0136020029002000F6B258
:1016D000FFF766F9252EF3D1300011F05DFE2900E9
:1016E00002002000FFF75CF9262011F055FE2900CA
:1016F00002002000FFF754F9F8BDC046F82400208E
:10170000BD880300711F0020C6880300701F0020E1
:10171000DD880300F588030007890300F0B5002485
:10172000344B87B01C60FFF7FBFA334D2868FBF79A
:1017300027FE0122314B2C601A60314D314B286855
:101740001C70314B1C70A04202D0FBF719FE2C60BC
:101750002E4C2088002803D0FBF724FE0023238092
:101760002B4C2088002828D0FBF7B8F90500010091
:1017700001A809F0D8FA019E01A8002E14D009F0A2
:10178000C2FA00222349070006F0CDFE0600FFF74B
:10179000EEFB002112F0EEFD30003900FBF724FED5
:1017A00001A809F09CFAE6E709F094FA2B7A2800E0
:1017B000013B2B72FBF7E4FD26800FF0D8FC041EE2
:1017C00015D00100002201A810F014FE002201A98A
:1017D0001148FFF743FF0498FBF7D2FD0F4B22009F
:1017E0000F49586806F08AFE2000FBF7C9FD07B0D4
:1017F000F0BDC0467C2400207424002004900040EA
:101800006C240020B9580020BA580020042500207C
:10181000D4560020AEA3030061AF02008C5A002012
:101820008A88030030B589B015000A00010003A8BA
:1018300010F0E0FD039B0093049B0193019A009B31
:10184000934216D203A80FF08BFC041E0A2C02D17F
:101850000D20FFF74BF92000FFF748F90A2C04D1BF
:10186000002D02D02800FFF741F903A810F082FEF6
:10187000E0E70698FBF784FD09B030BD10B5040021
:10188000FBF722FC0300002083420ED02378FF2BBD
:1018900001D1012009E00649200006F051FD002891
:1018A000F7D10449200006F04BFD0123184010BD7C
:1018B000528803005BAA030010B50400FBF704FC88
:1018C000002803D023780120FF2B02D02000FBF753
:1018D00044FC0123184010BDF8B5040080250C26F7
:1018E000214F63892000AB436381FBF7FDFB002898
:1018F00005D12000FBF765FA00280CD118E0200084
:10190000FBF716F90028F4D00138704338184389E2
:10191000AB434381F4E72000FBF7C6F9002821D050
:10192000441E7443104BE41863892B42D9D119E04B
:101930002000FBF778FC002814D02000FBF7B4F956
:101940000C24802500280DD001386043064E8619EE
:1019500073892B4202D03000FFF7BEFF3000FBF747
:1019600056F9EFE7F8BDC046BC26002010B50C00C4
:1019700088B069462022FBF79EFD22006946034895
:101980000BF06EFD002008B010BDC0460B890300AF
:101990003F2342891340222B01D1006810E0232B02
:1019A00001D180880CE0181E192804D81538142B92
:1019B00006D8103B03E02438212B01D81A3B18002D
:1019C000704710B50400FBF76FFB0923002806D110
:1019D0002000FBF79DF90423002800D103331800F1
:1019E00010BDF7B5012306000D00141E262C0ED0E5
:1019F0007C2A0CD05E2A0AD085211A0049008C422C
:101A000005D0210000230E39FF398A425B410122B3
:101A10001F001740002B07D1210025390A2904D8BF
:101A2000B24BCB40134000E013000122A11F134032
:101A3000FF390093072903D89523CB409A4304D05C
:101A4000022322009A433C2A2AD13000FBF7F2F904
:101A500000280CD02800FBF737FB002807D0300007
:101A6000FBF7BEFB0021884215D0280010E02800BB
:101A7000FBF7E0F9002813D03000FBF725FB002826
:101A80000ED02800FBF7ACFB0021884203D03000C9
:101A900009F077FB010001270F40002E2ED15AE2FA
:101AA000002E0ED1002D0CD10623FF3301209C42C5
:101AB00000D148E20823FF3300209C4200D142E2DB
:101AC0004DE2009B002B19D13000FBF7B3F9002841
:101AD00007D1002E05D03000FBF73FF9002800D1D8
:101AE0007EE12800FBF7A6F9002807D1002D05D0DC
:101AF0002800FBF732F9002800D171E1002F0BD14B
:101B00003000FBF76DFB002800D1CAE02800FBF78E
:101B100067FB002800D1C4E0300009F05FFE0090B0
:101B2000280009F05BFE07005E2C68D01EDC2B2C21
:101B300045D007DC262C5FD02A2C46D0252C00D09F
:101B4000ADE05FE02F2C4AD009DC2D2C00D0A6E0C0
:101B50003A000098FB17C117801A99413CE03C2CD1
:101B600000D181E03E2C00D18BE098E00A23FF33C6
:101B70009C4200D17EE00DDC0623FF339C4253D013
:101B80000823FF339C425FD07C2C00D087E0009874
:101B9000384346E086235B009C4279D005DC023B5B
:101BA0009C427CD10098B8403BE00E23FF339C421E
:101BB00035D001339C4272D10098F84031E0009A50
:101BC000C117D3178018594106E0009B0200D917AE
:101BD000C317009813F0DAFE09F0C3FABFE10098CA
:101BE00015F0C2FE040038000D0015F0BDFE020025
:101BF0000B0020002900A6E00098384011E0009872
:101C000078400EE0002805D00100009814F07CF820
:101C1000080006E0002200231000190093E000985D
:101C2000384109F089FA9AE1009B0022834209D1E8
:101C30003000FBF792F804002800FBF78EF8201A1A
:101C40004242424110007EE1009B0120BB4208D18C
:101C50003000FBF782F804002800FBF77EF86040B4
:101C6000C0B2012318406EE1009B0120BB4200DAA4
:101C700060E10BE0009B009AD80FFB179742584198
:101C800058E1009B0120BB4200DD53E1002051E1FF
:101C9000009B009AD817FB0FBA4258414AE11449F9
:101CA00055E1300006F03FFA00900191280006F05F
:101CB0003AFA3C2C00D175E01CDC2B2C35D00BDC27
:101CC000252C43D02A2C00D088E002000B0000987D
:101CD000019915F025F83FE02D2C2DD02F2C00D0A8
:101CE0007CE002000B00009801992CE02105000027
:101CF000408903000823FF339C4230D006DC3E2C91
:101D000060D00623FF339C4229D067E00A23FF33CB
:101D10009C424FD003339C4260D102000B000098DC
:101D20000199012414F036F853E002000B000098EA
:101D3000019914F0A5F80FE002000B00009801993A
:101D400015F068FA08E014F0C7FB05E002000B008C
:101D50000098019908F0F4FF09F0DAF9FFE00200B9
:101D60000B0000980199012713F0F0FF002800D123
:101D7000071C3000FFB2FAF7F0FF002801D0002D59
:101D800006D02800FAF7E9FF002802D0002E00D183
:101D900001270623FF3338009C4200D1D3E0012005
:101DA0007840D0E002000B0000980199012413F064
:101DB000D3FF0EE002000B0000980199012413F0FC
:101DC000D5FF06E002000B0000980199012413F0F2
:101DD000D7FF002800D1041CE0B2B4E06049B6E0AF
:101DE0003000FBF704F8071E18D13000FBF70AF8A3
:101DF000002813D13000FBF710F800280ED128007E
:101E0000FAF7F5FF002809D12800FAF7FBFF0028B0
:101E100004D12800FBF701F800283FD02800FAF78A
:101E2000E6FF87423AD1022322009A43130006229A
:101E3000FF32934232D13000FAF79AFF002809D1DD
:101E40002800FAF795FF002804D1701B4342434154
:101E5000D8B213E033682A68002193420DD1B288CA
:101E6000AB889A4209D13000FAF71EFF060028001D
:101E7000FAF71AFF301A4142414108000623FF33A6
:101E80009C4260D00823FF339C4202D1012670405F
:101E900059E03449002F5AD0334958E0002130002E
:101EA00009F06AFB00210600280009F065FB050027
:101EB000002E01D0002805D130002900FBF794FA4C
:101EC00000204CE02B2C0DD1300006F0BFFB041E8F
:101ED00002D0290009F0E9F930002900FBF784FA63
:101EE00020003CE0002301001A00300012F04EFCFC
:101EF000290007003000FBF777FA0623FF339C42E6
:101F000016D006DC3C2C17D03E2C1FD1F817C01B76
:101F100018E00A23FF339C4210D003339C4210D0B8
:101F20000823FF339C4211D1781E8741F8B20AE0A2
:101F300078427841C0B206E0F80F04E0781E3843DA
:101F400000E0F843C00F09F0EEF808E00749200070
:101F5000FFF70CFD03E0002D00D0CFE5A4E5FEBDAA
:101F6000488903003989030000A00300CDA50300C0
:101F700070B50400631E9C414B424B4105000E00AE
:101F80005C4000281CD000291AD0FBF70EF900286D
:101F900004D12800FBF7FEF800280AD03000FBF738
:101FA00004F9012400280BD13000FBF7F3F80028D6
:101FB00006D173896C895C403F231C4063425C41BD
:101FC000002C0CD006223100FF322800FFF709FD5B
:101FD000050009F072FA04002800FBF7D1F920008F
:101FE00070BD70B50400080009F0A6F8051E0AD0FF
:101FF000002301001A00200007F0BDF804002800AB
:10200000FBF7BEF9200070BDF0B587B00500029166
:1020100003920124002800D17AE0FAF7F3FE041EAF
:1020200004D13D4901200BF0F9F871E0290005A821
:10203000FBF714FA059E002E66D080227389920069
:102040009B18738100231D00029C0193039B019A3E
:10205000934247DD2168300006F072F900283CD039
:10206000A3680125002B38D005A808F04CFE050018
:10207000A088033817282CD813F0C2FC0C2B0C0CAA
:102080002B1F2519142B2B2B2B2B2B2B2B2B2B2BDB
:102090002B2B2B0C80216B89A26889005B186B812C
:1020A000156016E02800A768FEF761FF03E028002E
:1020B000A76809F002FA38700BE02800A76809F059
:1020C0008DFB386005E02800A76806F02CF8386022
:1020D00079602800FBF754F90125019B0C3401338A
:1020E0000193B3E70124002D05D1200032000B49F4
:1020F0000BF094F82C003000FBF742F905A8FBF731
:1021000099F9002C96D100E0012405A808F0E2FD21
:10211000200007B0F0BDC0464F890300718903005D
:1021200010B50400FAF779FE064A002808D120000D
:10213000FAF768FE0300581E8341034A5B421A40C7
:10214000100010BDB91802007D180200F0B501247E
:10215000802789B00C233F22651E5D43654E7019B0
:10216000438913420CD03B434381FAF773FE0028A6
:1021700006D070590C210B3013F056FC2418A4B271
:10218000FF230134A4B29B009C42E3D901240C2715
:102190003D008022661E7543564B5D196B891342C4
:1021A00005D0DB041B0F02D02800FFF795FB2800A9
:1021B000FAF750FE002808D07E434E4B0C21985968
:1021C0000B3013F031FC2418A4B2FF230134A4B265
:1021D0009B009C42DCD900250126474B290005A81D
:1021E0001D8005ACFAF7E9FC01950C23721E5343E0
:1021F0008022404F0293DD196B892800039313421C
:1022000051D0FAF727FE002827D0029B0C21D8597D
:102210000B3013F009FC002302906B8120002C008E
:1022200035003100FAF7C9FC029B0193019B5A1E4D
:1022300001920ED30C230135ADB26F1E5F432D4BBF
:102240002000FF18002329007B81FAF7B6FC3C0030
:10225000ECE7029BF618B6B222E02800FAF7B1FDCF
:10226000002811D02800FAF71FFD00280CD00C23FD
:102270000138584338184389002B05D08022134277
:1022800002D1037A013B03720C22731E5343194A95
:102290002000D318002231005A81FAF78EFC2C005E
:1022A0000123019314E0FAF7D5FD002808D0029B22
:1022B0000C21D8590B3013F0B7FB301886B207E069
:1022C000039B002B04D120003100FAF776FC2C0090
:1022D000FF230136B6B29B009E4286D90021200022
:1022E000FAF76BFC05A8FAF792FC034B18800198EB
:1022F00009B0F0BDBC26002072240020F0B58FB0DC
:10230000009000200E0001921F00824250DD0099D3
:1023100003A810F0FDF803A80FF0F2FF040003A8D3
:10232000002C42D010F0A5FA041EB4420AD1009B42
:10233000BB4207D003A80FF099FF012109F01CF957
:1023400004002CE02000FAF75DFD002809D12000F0
:10235000FAF74DFD002804D12000FAF75EFD0028B1
:102360001FD0019B31005A1E20003B00FFF7C6FF23
:10237000051E16D003A80FF079FF06002000FAF71B
:1023800041FD0C4B002800D10B4B31002A001800F6
:1023900009F04FF8290004003000FBF725F803A8E6
:1023A00003E003A810F02EF9B5E70FF083FF20003B
:1023B0000FB0F0BD8389030089890300F7B50C00D5
:1023C000160005F023FE0190200005F01FFE070017
:1023D000019808F011FE0400380008F00DFE3900E5
:1023E00005000198FBF700F80222F31FFF3B93431F
:1023F0000DD129002000FFF7BBFD83235B009E4227
:1024000002D001235840C0B208F08DFE04E0320033
:1024100029002000FFF7E5FA060029002000FAF75E
:10242000E3FF3000FEBD70B50500FAF73DFC041E69
:102430002BD0FAF753FB04002800FAF735FC06000E
:102440002800FAF775FB864203D100212800FAF72D
:1024500063FB2000FAF7DBFB01002800FAF7C8FB5A
:10246000237A2000013B2372FAF7D1FB002808D021
:10247000FAF734FB05000021FAF796FB2800FAF77B
:102480007FFF00212000FAF798FB200070BDF8B50F
:102490000500041E2BD000240668A64227DD013E5D
:1024A000FAF746FBA04215D0FAF718FB041E11D02C
:1024B000FAF77BFE002810D12000FAF7A2FB0700F4
:1024C0002000FAF75DFF002F04D03800ECE7200071
:1024D000FAF756FF00242E6009E0200009F07EF98B
:1024E0008642F4D12100280005F01FFCF3E720000C
:1024F000F8BD70B505000C00002800D0006808F099
:102500001BFE210009F078FA041E04D107480AF0E6
:1025100089FF200009E00100280005F06FFC200081
:10252000FAF72EFF281E00D0286870BD908903009E
:1025300070B50C00FFF7DDFF05002000FAF720FF63
:10254000280070BDF8B50D001700FAF7ADFB0400C8
:10255000201E1FD0FAF7C2FA060005F057FD041E30
:10256000AC4207D0002F0AD12900FFF701FD002857
:1025700005D025002800FAF703FF30000AE020000C
:10258000FAF7FEFE3000FAF742FB04003000FAF7DB
:10259000F7FEDDE7F8BD70B5002204000D00FFF77F
:1025A000D1FF002804D129002000FFF7A2FF01E09D
:1025B000FAF7E6FE70BDF7B50F000190FAF7B8FA2A
:1025C0000500002D16D02800FAF788FA0600FAF761
:1025D000ECFD002806D034683000BC4229D0FAF760
:1025E000CFFE08E03000FAF70CFB05003000FAF7E8
:1025F000C7FEE6E72C00BC4201DA00202CE0E30F26
:102600001C196410A7420FDD002DF6D02800FAF740
:1026100065FA036804009F420BD0FAF7F2FA05004E
:102620002000FAF7ADFEEFE70198FAF73DFB050051
:102630000FE005F043FD0FE02800FAF74FFA0368BA
:1026400004009F42F5D0FAF7E2FA05002000FAF7FD
:1026500097FE002DF0D1D0E7FEBDF7B58022050032
:102660000E0043895200002905D0002413426AD08D
:10267000364A134003E00C00134264D113436B81CC
:102680002800FAF79EFB002804D12800FAF7CBFDBA
:1026900000281CD02800FAF707FB01240700002FB0
:1026A00021D03800FAF71AFA31000190FFF7D5FF70
:1026B00024182800FAF7B7FD0027B84203D0019884
:1026C000FAF7A5FA07000198FAF75AFEE7E728009B
:1026D000FAF7C0FB0124002805D028680C210B3034
:1026E00013F0A2F904192800FAF7FEFC002811D013
:1026F0002800FAF71DFA0700002F0BD03800FAF770
:10270000EDF90190FAF714FA070001980134FAF78D
:1027100037FEF1E72800FAF7FBFA002813D028006B
:10272000FAF7E6FA00280ED12800FAF7BDFA0028D9
:1027300009D0FAF7D3F931000500FFF78EFF04192D
:102740002800FAF71DFE2000FEBDC046FFFEFFFF79
:10275000F0B591B0050002910EF009FD041E60D0A5
:10276000290005A80FF0D4FE002705A80FF0C8FD2A
:1027700000283DD005A80FF079FD0390FAF715FD6C
:10278000012600282BD0039809F028F8029B0600A8
:10279000002B07D0B74205DA02992000013708F074
:1027A00084FDF7E705A810F064F8012600900028E2
:1027B00012D0FAF7D2FA011E0ED1009808F0DCFE12
:1027C0000190002807D00100200008F06EFD01985C
:1027D000FAF7D6FD00E0019E0098FAF7D1FD0398C4
:1027E000FAF7CEFD05A80FF00DFF002EBDD100E0D9
:1027F000012605A80FF05EFD002E12D0029B002BD3
:102800000FD02800FAF7F3FA00280AD02E1E00D0C5
:102810002E680137BE4204DD0299200008F045FD14
:10282000F7E7200011B0F0BD014802497047C046EB
:10283000CD3B7F669EA0E63F014802497047C046F7
:10284000CD3B7F669EA0F63F014802497047C046D7
:102850000EE526157BCBDB3F014802497047C04699
:10286000FE822B654715F73F014802497047C04675
:102870001655B5BBB16B0240014802497047C046CE
:10288000EF39FAFE422EE63F014802497047C04642
:10289000182D4454FB210940014802497047C046A5
:1028A0006957148B0ABF054000207047002070470D
:1028B00000207047002070470120704710B50022AB
:1028C00000230020014913F007FE10BD0000F03F77
:1028D00010B5002200230020014913F0FDFD10BDBA
:1028E0000000F03F10B5002200230020044913F03F
:1028F000F3FD0200802000060B181900100010BD27
:102900000000F03F80210020490370470120014969
:1029100040427047FFFFEF7F0022002310B51000F8
:10292000190013F0D9FD10BD0022002310B51000CE
:10293000190013F0D1FD10BD10B5064B064A002159
:10294000D05813F087FAFC2300229B0514F0E8F915
:1029500010BDC0460405000000B000408021034ABD
:10296000490013880B4313807047C046F8240020A9
:102970004021024A13880B4313807047F82400203B
:102980008021024A13880B4313807047F8240020EB
:10299000F8B50D000400FDF7DDF9084A06000F0048
:1029A000074B2900200013F06BFAFDF7D3F9020062
:1029B0000B003000390013F08FFDF8BD182D445482
:1029C000FB21F93F10B5034A034B13F059FAFDF709
:1029D000C1F910BD182D4454FB21F93F10B5052055
:1029E000FAF71DF910BD10B5FFF7F8FF10BD10B5CF
:1029F000FFF7F4FF10BD10B5FFF7F0FF10BD10B5E5
:102A0000FFF7ECFF10BD10B5FFF7E8FF10BD10B5E4
:102A1000FFF7E4FF10BD10B5FFF7E0FF10BD10B5E4
:102A2000FFF7DCFF10BD10B5FFF7D8FF10BD10B5E4
:102A300002490348FEF7EEFB10BDC0464D9A030065
:102A4000549A030010B502490248FEF7E3FB10BD9B
:102A50005E9A0300629A030010B502490248FEF72D
:102A6000D9FB10BD5E9A0300679A030010B50249B6
:102A70000248FEF7CFFB10BD76B203006C9A03004C
:102A800010B502490248FEF7C5FB10BD76B203003F
:102A9000719A030010B502490248FEF7BBFB10BD56
:102AA00076B20300769A030010B502490248FEF799
:102AB000B1FB10BD4D9A03007B9A030010B502498B
:102AC0000248FEF7A7FB10BD4D9A0300859A03004C
:102AD00010B502490248FEF79DFB10BD4D9A030058
:102AE0008F9A030010B502490248FEF793FB10BD10
:102AF0004D9A03000789030010B512F099FE14F0F7
:102B000033FF024A024B13F0E7FC10BD0000C0FF88
:102B1000FFFFDF4110B501210EF02EFB10BD10B5F7
:102B200000210EF029FB10BD10B501230EF081FA33
:102B300010BD10B500230EF07CFA10BD10B5FEF7E5
:102B400077F9FEF72DF910BD10B50248FBF7BCF977
:102B500010BDC046979A030070B505000320FAF730
:102B60005EF8041E04D002000121280011F0E4FFE9
:102B7000200070BD70B505000320FAF750F8041E60
:102B800004D002000021280011F0D6FF200070BD03
:102B900010B5042207F0F4F810BD10B5022207F0BA
:102BA000EFF810BD10B5012207F0EAF810BD10B51E
:102BB000042207F024F910BD10B5022207F01FF916
:102BC00010BD10B5012207F01AF910BDF8B50600C6
:102BD000FAF7CEF84C4D00281DD02C0033684B4A34
:102BE0002D34934200D18CE0494A9034934200D175
:102BF00087E0484A1234934200D182E0464A0934C1
:102C000093427ED0454AAC1DFF34934279D0444A6A
:102C10001234934275D03000FAF7F4F8002807D147
:102C200030002C00FAF750FA2D34002869D13AE030
:102C300000223C49300005F088FB05F03FFA041EF5
:102C4000EED0FAF795F80028EAD0276820002C008B
:102C5000FAF796FB344B12349F4252D0334B09346F
:102C60009F424ED0324B1B349F424AD0314B1234DC
:102C70009F4246D0304B24349F4242D02F4B1234D7
:102C80009F423ED02E4B24349F423AD02D4B0934E4
:102C90009F4236D02C4B3F349F4232D02B4B1234C4
:102CA0009F42BDD12DE030002C00FAF7B6F8BD34BC
:102CB000002826D130002C00FAF777FACF3400280C
:102CC0001FD13000FAF766FA00281AD130002C0024
:102CD000FAF77BFAD834002813D13000FAF766F8F7
:102CE000002804D03379AC1DFF34812B09D130008A
:102CF0002C00FAF77CF81834FF34002801D12C009E
:102D0000B4342000F8BDC046B78903007113030036
:102D10005DA002006504030091050300E72902009D
:102D2000678D02005BAA0300EF290200FBDE0200B0
:102D30002DC2020085DA0200C5DA0200F72902007E
:102D400095DA0200A5DA0200FDBC0200B5DA020045
:102D500010B50400FAF70CF800282ED02368304A8A
:102D6000304893425BD0304A93422ED02F4A934250
:102D70002ED02F4A93422ED02E4A93422ED02E4A46
:102D800093422ED02D4A93422ED02D4A93422ED0DC
:102D90002C4A93422ED02C4A93422ED02B4A934257
:102DA0002ED02B4A93422ED02A4A93422ED02A4A22
:102DB00093422ED0294A93422ED0294B00201B68E3
:102DC0009C422CD117485A3029E01648093026E099
:102DD0001448243023E013483F3020E0114851309C
:102DE0001DE0104863301AE00E48753017E00D48BA
:102DF000873014E00B48903011E00A4899300EE01B
:102E00000848C6300BE00748E13008E00548F330D9
:102E100005E004480F3001E002482130FF3010BDCA
:102E2000FDBC0200B7890300F1030300FF29020083
:102E3000F7290200072A02000F2A0200172A0200BF
:102E4000678D0200650403001F2A0200FBDE0200FA
:102E5000EF29020071130300272A0200DD29020076
:102E60008C5A0020F0B50500002787B00491059228
:102E70000379013B0393039B9F4256DC039B297814
:102E8000FE186B78AC781B020B4324041A00230055
:102E9000EC781343761024061C43AA79F300E41857
:102EA0006979EB7912020A431B0413431A002B7A47
:102EB00061781B06134322780902114359180598BB
:102EC00014F0EFFE031E29D1E579A2792D02FC2032
:102ED0001543A778E27826796179E024C00128407B
:102EE000E401A0420CD11002020030043A43024334
:102EF000080610430093049A29000AF0CFFA15E05F
:102F0000120234043A43224346200C061443F9F7D4
:102F100086FE00280AD00460858007E0002802DAD7
:102F2000731E0393A7E7771CA5E7002007B0F0BD49
:102F3000F7B504000D00002800D145E1FAF768F963
:102F4000002800D040E12000F9F712FFA64E00282B
:102F500005D12000FAF7B8F8002864D16CE02368A6
:102F6000A24A934203D12A00210030004FE0A04A38
:102F7000934202D13000093047E09E4A934202D189
:102F80003000243041E09C4A934202D130003F306F
:102F90003BE09A4A934202D13000513035E0984AE2
:102FA000934202D1300063302FE0964A934202D11F
:102FB0003000753029E0944A934202D130008730C6
:102FC00023E0924A934202D1300090301DE0904AB3
:102FD000934202D13000993017E08E4A934202D1D9
:102FE0003000C63011E08C4A934202D13000E1300B
:102FF0000BE08A4A934202D13000F33005E0884A60
:1030000093420AD130000F30FF302A002100FFF731
:1030100029FF002800D0E5E09BE7824A934298D13F
:1030200030002130F0E730002A002D302100FFF77A
:1030300019FF002800D0D5E02000F9F7EEFE0028A7
:1030400008D030002A00BD302100FFF70BFF002818
:1030500000D0C7E02000FAF7A8F800280AD1200025
:10306000FAF798F8002805D12000FAF7AEF8002802
:103070000AD112E030002A00CF302100FFF7F2FE23
:10308000002800D0AEE0EFE730002A00D830210061
:10309000FFF7E8FE002800D0A4E02000F9F786FE44
:1030A000002802D02379812B05D12000F9F79FFE5B
:1030B00000280AD113E0B01DFF302A002100FFF7DD
:1030C000D1FE002800D08DE0EFE730001830FF304F
:1030D0002A002100FFF7C6FE002800D082E0200071
:1030E000F9F790FE002806D000224F49200005F095
:1030F0002CF904F0E3FF0700F9F784FE00230193A5
:10310000984207D01A004949380005F01EF904F02A
:10311000D5FF01903800FAF733F9019B002B4BD013
:103120001800F9F725FE002846D0019B18001F68FB
:10313000FAF726F9384B9F4202D13000123034E0C2
:10314000344B9F4202D130001B302EE0384B9F425F
:1031500002D13000363028E0364B9F4202D1300099
:10316000483022E0344B9F4202D130006C301CE0EA
:10317000214B9F4202D130007E3016E02F4B9F4200
:1031800002D13000A23010E02D4B9F4202D130001E
:10319000AB300AE0154B9F4202D13000EA3004E028
:1031A000284B9F420BD13000FC302A002100FFF752
:1031B00059FE002816D102E00198FAF7E1F8300034
:1031C0002A00B43021000BE02800FDF75FFEFF2845
:1031D00002D007F0BAFF05E02A00210002485A3069
:1031E000FFF740FEFEBDC046B7890300FDBC0200EC
:1031F000F1030300FF290200F7290200072A020059
:103200000F2A0200172A0200678D020065040300DE
:103210001F2A0200FBDE0200EF29020071130300E7
:10322000272A0200DD290200528803005BAA03005E
:103230002DC2020085DA0200C5DA020095DA02002A
:10324000A5DA0200B5DA0200F7B500230600002275
:103250000020184913F040F980231B060500CC1804
:1032600001A8310007F05FFD019B01A8002B1BD0D6
:1032700007F049FDFAF709F92A00230007000E00BC
:1032800012F07EFD002809D13A00330038003100E9
:1032900014F014FB002801D12F00260001A807F02C
:1032A0001EFD3D003400DFE707F014FD280021007B
:1032B00003B0F0BD0000F03FF7B50023040000228A
:1032C0000020174913F008F906000F0001A821009B
:1032D00007F029FD019B01A8002B1BD007F013FD6F
:1032E000FAF7D3F832003B0004000D0012F034FD71
:1032F000002809D122002B002000290014F0DEFA5A
:10330000002801D134003D0001A807F0E8FC2600A8
:103310002F00DFE707F0DEFC3000390003B0F0BD1E
:103320000000F03FF0B5C54C9BB0216809A807F03C
:10333000FAFC0694099B09A8002B79D007F0EAFC57
:10334000070009A807F0DFFC402204000AA93800A2
:1033500008F0C6F90AA803F07DFB002804D023007A
:103360003A000021B64859E0B649380004F0E8FFB9
:10337000002855D1B449380004F0E2FF00284FD1AD
:103380003B78FF2B4CD00AA80FF08EFF002847D1C6
:103390002000F9F7F8FC061E42D12000F9F73DFDA8
:1033A000A74D0390002813D03B00A84A3100280005
:1033B00009F05EFE33002A00102120000BF058FBBC
:1033C0003100A348FDF79CFB23003A00310024E0C4
:1033D00028003B009F4A039909F04AFE2000F9F7B4
:1033E00011FD002800D11EE19B49039A200005F041
:1033F0009AF8011E00D116E1069823000422006805
:10340000FEF77CFF031E00D10DE1944A0021280045
:1034100009F02EFE23003A0000212800FEF722F8D2
:1034200020003900F9F7E0FF09A807F058FC81E710
:1034300007F050FC8A4B1888F9F750FB0400010094
:1034400009A807F070FC2000F9F79AFF099B09A86A
:10345000002B5DD007F057FC00228249060004F0E3
:1034600074FF040004F082FD03902000F9F788FF48
:1034700000227D49300005F056F8041E7B4800D13B
:103480007B480021FDF73CFB00236D4D039A19009A
:103490002800FDF7D1FA0695002C03D0200008F093
:1034A000F5F90EE022007349300005F03CF8070002
:1034B00008F0ECF90D0007903800F9F761FF2900DA
:1034C0000798FA220023920012F060FACB175B04EF
:1034D0005B0C049300230593049A059B80185941C3
:1034E0004B04C00B1843C91312F0B4FC624A00909D
:1034F00001910599069809F0BBFD03992000F9F7A1
:1035000073FF3000F9F73CFF09A807F0E8FB9DE7DF
:1035100007F0E0FB594B1888F9F7E0FA04000100C6
:1035200009A807F000FC2000F9F72AFF099C09A868
:10353000002C6FD007F0E7FB00224A49040004F09A
:1035400004FF050004F012FD04902800F9F718FFAD
:1035500000224B49200004F0E6FFF9F78CFF00221F
:1035600048490690200004F0DEFFF9F79AFF002298
:1035700003904549200004F0D6FF0022434907008C
:10358000200004F0D0FFF9F78CFF0021060040482E
:10359000FDF7B6FA00232A4D049A19002800FDF71A
:1035A0004BFA069B3B4A002B00D13B4A03993B4B0D
:1035B000002902DB3A4B00D13A4B019300923B00C9
:1035C000394A0021280009F053FD002E13DDFA22AC
:1035D00000239200F117300012F0D8F94B04C00B11
:1035E0001843C91312F036FC304A009001910021B3
:1035F000280009F03DFD00212D48FDF781FA0499CE
:103600003800F9F7F1FE2000F9F7BAFE09A807F033
:1036100066FB8BE707F05EFB012221000848FEF7FE
:103620001DF81BB0F0BD28003B0022000021FDF773
:1036300003FA00211F48FDF763FAF1E68C5A0020D7
:10364000010B02005C88030063880300CD9A03002D
:10365000A87F0300D99A030052880300E39A03006D
:1036600004250020337E0300787E0300A09A030027
:10367000AD9A0300287E0300F79A0300D456002079
:10368000457E030071820300AEA30300117E030098
:10369000FF9A0300D181030094810300B99A0300CB
:1036A000C19A0300C89A0300099B0300269B0300EC
:1036B000369B030004890300F7B54F4C0026A06831
:1036C000F9F789FF1F23A28E1A40009201F050F8EB
:1036D000009B012B02D1A68E36091E40A068002552
:1036E0000223C25E95235B009A425FD1F9F773FF14
:1036F0002821A068FAF732FBA84200D17AE0AE4256
:103700000BD0A0680121030064331B78C318013378
:10371000DD77203009F0E6F905008021A068490036
:10372000FAF71CFB002865D02921A068FAF716FBE0
:1037300000285FD0002D22D000223049606804F0BC
:1037400004FE071E14D004F061FC01000190280063
:1037500004F055FE0198F9F713FE3900606804F093
:10376000E4FA3800F9F70CFE2549606804F038FEE9
:103770005022A38E28009343A386F9F701FE009BF5
:10378000012B10D1002E0ED1A38E9DB209F0DAF8D4
:1037900000F0EEFFA28E1B4B1A401B4B2B40134335
:1037A000A386009D02E000F0E3FF0125A06802234C
:1037B000C25E2C23FF339A4206D0002D1AD1043B5F
:1037C000A28EFF3B1A4215D12C21FF31FAF7C6FA1F
:1037D00000280FD0002E03D01022A38E9343A3867F
:1037E00000F0C6FF002E05D0002D03D11022A38EBD
:1037F0001343A3860020FEBD8C5A0020768203006E
:10380000A1820300C0FCFFFF3F030000F8B53C4D60
:103810000026A868F9F7DFFEAB6802229B5E8022D3
:10382000520093426AD109F071F9002866D11F2332
:10383000A98E0400194001292ED1AB681A00643208
:1038400012789A1801322033D077180009F04AF91B
:10385000041E21D110F0DCFF50E0A8680223C15EF5
:103860002E2921D1FAF77AFA002823D01F23AA8E15
:103870001A40012A10D1A96800200B0064331B787C
:10388000CB180133D8772031200004F05EFD07000B
:103890002000F9F775FD3C008021A8684900FAF77F
:1038A0005DFA0028D9D105E03D2918D1FAF756FA7A
:1038B000002803D12000F9F763FD1FE001F04CFA66
:1038C00004F0FCFB1F22AB8E07001340012B03D139
:1038D0000100200009F04EFD3800F9F751FD3000DD
:1038E000F9F74EFDA8680223C15E2C2905D1FAF72D
:1038F00035FA260000288FD100E026003000F8BD00
:103900008C5A0020F0B5854C9DB00600A068F9F7F0
:1039100062FEA38E9BB20293002E2DD02821A068B8
:10392000FAF71CFA002800D1F5E0A36804AD191DD0
:10393000280016AFFAF7BAFA3B0007CD07C307CD48
:1039400007C301F009FA1F23A28E050013400020CF
:10395000012B04D1280004F059FBF9F78CFD012359
:10396000184001902800F9F70BFD2921A068FAF70B
:10397000F5F9002802D1CBE001230193A36810A838
:10398000191DFAF793FAA58E019BADB2002B01D158
:1039900008F0D8FF8022029B520013400393A38EAD
:1039A0001343A38600F0FAFEF9F7EAFC039B002B11
:1039B00003D1A28E5A4B1340A3860423A28E134038
:1039C00003D00123A386002305E0A28E0293930770
:1039D00002D50123A3860293019B002B06D1A28E60
:1039E000504B1A40504B1D401543A586002E39D12F
:1039F0009021A0684900FAF7B1F9002801D110A878
:103A000087E02821A068FAF7A9F90028F7D0A36871
:103A100004AF191D380016ADFAF748FA2B0007CF8E
:103A200007C307CF07C301F097F91F23A28E070032
:103A300013403000012B04D1380004F0E7FAF9F705
:103A40001AFD0126304001903800F9F799FC292130
:103A5000A068FAF783F9002804D110A8FAF72FFA22
:103A6000280056E0A36804AD191D28000AAFFAF734
:103A70001DFA3B0007CD07C307CD07C3029B002BF0
:103A80003CD1019B002B39D016A9A068FAF7C8F9E0
:103A900001F062F91F22A38E06001340029D012B44
:103AA00004D104F0B3FAF9F7E6FC05003000F9F7A9
:103AB00067FC002D20D010A9A068FAF7B1F9802288
:103AC000A38E52001343A38600F068FEF9F758FC5A
:103AD000039B002B03D1A28E114B1340A386A38E10
:103AE0005B0702D50123A386C8E7A38E9B07C5D534
:103AF0000123A3860293C1E70195BFE73900A068BF
:103B0000FAF78EF916A8FAF7DAF910A8FAF7D7F942
:103B10003800FAF7D4F900201DB0F0BD8C5A00200F
:103B2000FFFEFFFFC0FCFFFF3F03000070B52B4C02
:103B3000A068F9F750FD2821A068FAF70FF90028CE
:103B400049D001F014F92823A58E06001D4043D169
:103B50002921A068FAF702F900283CD01F23A28E81
:103B60001340012B05D1300004F050FAF9F783FC23
:103B700005003000F9F704FCA38E9EB2002D01D1A0
:103B800008F0E0FE00F00AFEF9F7FAFB002D06D17E
:103B9000A28E134B1A40134B33401343A386A068E5
:103BA0000223C25E8F235B009A4214D1F9F713FD02
:103BB000A38E9EB2002D01D008F0C4FE00F0EEFDF1
:103BC000F9F7DEFB002D06D0A28E054B1A40054BFF
:103BD00033401343A386002070BDC0468C5A00209A
:103BE000C0FCFFFF3F03000070B55B4DA868438831
:103BF0009AB2511EFF39032918D93639022915D92D
:103C0000233189B21D2904D8544CCC402100C90766
:103C10000CD4213A92B20C2A00D997E05049D140F5
:103C20000A00D20702D41BB25B2B02D101F09FF82D
:103C300090E07B2B02D100F09BFD85E03B2B00D177
:103C40007CE093225200934202D1FFF7DFFD81E036
:103C50001E22FF32934202D1FFF768FF7AE0202252
:103C6000FF32934201D1002004E09022520093429F
:103C700003D10120FFF746FE6CE02222FF3293427F
:103C800002D100F073F865E02A22FF32934202D19C
:103C9000FFF712FD5EE02622FF32934202D100F0D0
:103CA0005FFB57E094225200934202D100F040FBA8
:103CB00050E092225200934202D100F0DDFA49E036
:103CC0002422FF32934211D1F9F785FC1F22AB8EDB
:103CD0001340012B38D18023A88E5B001840041EAE
:103CE000204915D0AB8E9343042219E09122520053
:103CF000934218D1F9F76FFC1F22AB8E1340012BB2
:103D000022D1C023A88E9B001840041E05D116495D
:103D1000022009F083FA20001CE0AB8E93430222BC
:103D20001343AB8610E03422FF32934202D100F0FD
:103D30004DFB0FE03A22FF32934202D1F9F74BFCE0
:103D400002E00021FAF70AF8002003E07E2B00D001
:103D500069E76BE770BDC0468C5A00200300103E37
:103D600081140000669B0300969B0300F0B5C34CD2
:103D7000A5B0A068F9F72FFC2821A068F9F7EEFF9D
:103D8000002800D15CE28023A28E5B001A400192E1
:103D90008022A38E00251343A386A36802229B5E84
:103DA0003B2B02D0FFF720FF050008F0AFFE071EF7
:103DB00035D18022A38E9343A386A36802229A5E04
:103DC0003223FF339A4200D0C2E0A68E133BFF3B62
:103DD0001E40012E0DD12800F8F79AFF002808D1C7
:103DE0002800F9F7CDFA2A00A549300009F016FAA3
:103DF00026E21F23A68E1E4000230293012E07D128
:103E00002B7A002B04D12900206803F0F7FF0296DB
:103E10003221A068FF31F9F7A1FF002803D1280063
:103E2000F9F7AEFA0CE200F0A2FF04F047F92921FD
:103E30000600A068F9F792FF002800D183E0A3688C
:103E40000DA8191DFAF732F8A78E08F07BFD802225
:103E5000A38E52001343A38600F0A0FCF9F790FA5A
:103E6000A36813A8191DFAF721F8019BBFB2002B14
:103E700003D1A28E834B1340A386A28E824B1A409D
:103E8000824B1F401743A786A78E1F242740012F70
:103E900047D13000F9F736F900283BD03000FEF763
:103EA0003FF93100049019A80EF032FB002305946D
:103EB00003930093714B059A9B8E1340012B25D1E0
:103EC00019A80EF01DFA002820D0039B002B1DD14D
:103ED00019A80EF0CBF9049B0400002B00D151E18E
:103EE0009847002800D14DE12000F9F7EDF80028AF
:103EF00000D19AE16649200004F022FA002800D19E
:103F000093E1200004F082F800908EE119A80EF0F1
:103F1000D1F906E0002E04D032005E49380009F0E5
:103F20007DF9564C13A9A068F9F77AFF0DA8F9F7A7
:103F3000C6FF13A8F9F7C3FF029B002B03D029008B
:103F4000206803F0F2FE31002800F9F74DFA77E11E
:103F50002800F9F715FA3B21A068F9F7FFFE0028C1
:103F600000D16DE1A36807A8191DF9F79FFFA368A9
:103F7000012602229B5E3B2B12D000F0EDFE1F2398
:103F8000A28E050013403800B34204D1280004F08B
:103F90003DF8F9F770FA012606402800F9F7F0F924
:103FA0003B21A068F9F7DAFE002801D107A8E6E076
:103FB000A3680DA8191DF9F779FFA36802229B5E7B
:103FC000292B0ED0A38E9DB208F0BCFC00F0CFFED2
:103FD000F9F7D6F9A28E2C4B1A402C4B2B401343E9
:103FE000A3862921A068F9F7B9FE002804D107A803
:103FF000F9F765FF0DA8C2E0A36813A8191DF9F72A
:1040000055FFA78EBFB2002E01D108F09BFC802285
:10401000A38E52001343A38600F0C0FBF9F7B0F95A
:10402000A36819A8191DF9F741FF019B002B03D1C3
:10403000A28E144B1340A386002E04D11F23A28E00
:104040001340012B0FD00423A58E1D4003D0033B4A
:10405000A386002504E0A38E9B0701D50125A58634
:10406000002E19D100E03500A28E074B00261A4021
:10407000064B1F401743A7861BE0C0468C5A002002
:10408000CB9B0300FFFEFFFFC0FCFFFF3F030000D0
:1040900052880300FC9B03000DA9A068F9F7C0FE3D
:1040A000A36802229B5E292B03D000F060FEF9F783
:1040B00067F91F27002D54D1A38E3B40012B50D10F
:1040C000002E4ED007A9A068F9F7AAFEA368022225
:1040D0009B5E3B2B0AD000F03FFE009003F096FF62
:1040E000F9F7C9F906000098F9F74AF9A38E3B40A1
:1040F000012B20D1002E1ED013A9A068F9F790FE45
:104100008022A38E52001343A38600F047FBF9F7E9
:1041100037F9019B002B03D1A28E4B4B1340A38692
:10412000A38E5B0702D50123A38604E0A38E9B0721
:1041300001D50125A586A38E3B40012BBAD1002EC7
:10414000B8D0002DB6D10DA9A068F9F769FEA36813
:1041500002229B5E292BAFD000F009FEF9F710F97F
:10416000AAE719A9A068F9F75BFE07A8F9F7A7FE67
:104170000DA8F9F7A4FE13A8F9F7A1FE19A8F9F7FD
:104180009EFE5DE02000F8F7C3FD002851D000221C
:104190002000110004F0F4F9071E2DD001002800C2
:1041A00004F02DF9BC4202D03800F9F7E9F819A85B
:1041B0000EF028FA254F0DA9B868F9F731FE8022D4
:1041C000BB8E52001343BB8600F0E8FAF9F7D8F82B
:1041D000019B002B03D1BA8E1B4B1340BB861B4B9C
:1041E0009A8E520702D501229A8605E09A8E92078E
:1041F00002D501229A8603922000F9F7C1F819A886
:104200000EF07EF8041E00D054E6009B002B00D177
:1042100050E619A80EF04EF8009919A80EF078F99A
:104220000098F9F7ADF8009444E619A80EF0EAF901
:10423000E2E7002CE0D02100280004F0E0F8B6E727
:10424000002025B0F0BDC046FFFEFFFF8C5A0020C5
:1042500010B500202824074B9A8E224209D19B6872
:1042600002229B5E002B04D0F9F78AF800F096FA40
:10427000F1E710BD8C5A0020F8B52C4E0024B06830
:10428000F9F7A9F91F23B58E37001D40012D0AD17A
:10429000B068F9F769FE210007F0AEFB041E02D1F9
:1042A00010F0B6FA3FE08021B8684900F9F756FDF2
:1042B000061E04D12000F9F763F8300034E0002036
:1042C00003F04AFB0600012D2AD1FB6A002B06DD14
:1042D00001339B00FF182A002100786802E02A00C1
:1042E0002100386804F05CFA050003F08FFE070037
:1042F000F8F793FD002808D0300003F0DFFE060039
:10430000010038000CF0DAF903E03100280009F070
:1043100031F82000F9F734F83800F9F731F82C00BB
:104320003000F9F72DF82000F8BDC0468C5A002067
:1043300070B50A4DA868F9F74EF900F018FD03F0C2
:10434000BDFE1F23AA8E04001340012B01D108F0EB
:1043500031FF2000F9F714F8002070BD8C5A0020BE
:1043600070B5174C0025A068F9F735F9A36802224B
:104370009B5E3B2B06D07D2B04D000F0F8FC03F0B5
:104380009DFE05001F23A28E1340012B12D1002198
:104390000C4808F0A7FB041E08D0290008F0EAFF2B
:1043A0002000F8F7EDFF08F0CDFA03E006490220FF
:1043B00008F034FF2800F8F7E3FF002070BDC04686
:1043C0008C5A0020BD8103003C9B0300F0B56C4E6D
:1043D00085B0B068F9F7FFF82821B068F9F7BEFC9E
:1043E0003400002800D1C7E000F0C1FC29210500FD
:1043F000B068F9F7B3FC00282DD07B21B068F9F73D
:10440000ADFC002827D0B38E9BB203931F23B28E3E
:104410001A40171E012F02D1E233FF33B386002367
:1044200001930BE0012F32D000260298F8F7A8FF85
:10443000002E38D12826A38E33423AD0A06802221B
:10444000835E9A225200934243D19A214900F9F7A0
:1044500085FC002803D12800F8F792FF8CE0A68E97
:10446000B6B2012F01D1474BA38600F075FC802323
:104470009B0002901E433A21A068A686F9F76EFCC5
:104480000028CFD102992800F8F7AEFF74E083220C
:10449000029952002800FDF791FFF8F7ECFF061E85
:1044A000C2D00197C1E7A38EDB06C3D1354BA386EB
:1044B000C0E7A3685B88002BC0D01A00353AFF3AEA
:1044C000012ABBD97D2BB9D000F068F9F8F758FF65
:1044D000B1E72800F8F754FF012F06D11F23A28E61
:1044E0001340022B01D1274BA386A38E264E274DC6
:1044F000039A2B4032401343A068A3860223C25E76
:104500003623FF3302969A4232D1F9F764F83A2102
:10451000A068F9F723FC00282ED0A68E019BB6B226
:10452000002B02D008F00EFA0FE08022A38E92003A
:104530001343A38609E0A3685B88002B09D07D2B79
:1045400007D000F02BF9F8F71BFF2822A38E1342A7
:10455000F1D0012F06D1019B002B03D10222A38EA3
:104560009343A386A38E1D40029B1E402E43A68626
:104570007D21A068F9F7F2FB002005B0F0BDC04630
:104580008C5A0020010200003F030000C0FCFFFF26
:10459000842203005200904222DC0622FF320620D1
:1045A00093424EDA2D2B47D00BDC0138262B48D016
:1045B00002DC252B42D043E02A2B3FD02B2B3BD0D3
:1045C0003EE03E2B2DD004DC2F2B37D03C2B28D0C7
:1045D00036E004205E2B34D001387C2B31D02FE024
:1045E00087225200904209DC0E22FF32904221DAEB
:1045F000033A90421ED014DB023210E01C22FF323C
:10460000012093421DD005DC1A22FF32001893428C
:1046100017D015E03222FF32934204D00132934288
:104620000ED107200DE0074B00209B8E1B0608D4FF
:10463000073006E0082004E0092002E00A2000E03C
:10464000002070478C5A0020F7B504001D4DA86863
:1046500043880193143BFF3B012B30D8F8F7BBFF95
:104660001F23A88E18400128F0D106F065FD060032
:10467000200003F0CBFC070003F0C2FD050038006A
:10468000F8F77EFE6B460421595E1423FF332B227C
:10469000994200D0023231002800FDF78FFE07005A
:1046A0003000F8F76DFE3900200008F063FE380096
:1046B000F8F766FE2000F8F763FE2C00C6E720003E
:1046C000FEBDC0468C5A0020F8B51F23254C00259E
:1046D000A28E1340012B34D138274026A3685B8873
:1046E000002B3DD07D2B3BD0FFF77EFAF8F748FE3C
:1046F000A38E3B4218D0A368002B15D0A38E334263
:1047000012D1A38E1A22334317496068A38603F09F
:104710000AFF051E08D0154906F02EFC280008F0F7
:10472000B2FC2800F8F72CFE2823A28E1A42D5D01E
:1047300016E01BB2002D0ED07B2B07D10135F8F708
:104740004AFFA0684388002BF3D109E07D3B594222
:1047500059416D1AF3E77D2B02D07B2BEFD1EDE7AA
:10476000F8BDC0468C5A0020A182030048A803006F
:1047700010B5094C7B21A068F9F7F0FA002809D0A0
:10478000FFF7A2FF2823A28E1A4203D17D21A06841
:10479000F9F7E4FA10BDC0468C5A002070B50B4DF5
:1047A000AB6802229B5E7B2B03D1FFF7E1FF002465
:1047B00009E0FFF719FA0400A8680222835E3B2B88
:1047C00001D1F8F708FF200070BDC0468C5A0020C8
:1047D000F8B506000C1E41D0080003F017FC0500D8
:1047E000F8F710FB00282BD1002D02D01C4808F050
:1047F00019FE2800F8F7C4FD0520F8F710FA80220A
:104800000500638992009B1863812000F8F74CFA39
:1048100000280ED0F8F762F90700F8F779FA0028B7
:1048200004D02000F8F7ACFD3C00EEE73800F8F7C4
:10483000A7FD2900200003F0E2FD2000F8F7A0FD0D
:1048400001220849280003F080FD041E02D0310037
:1048500003F0D5FD29002000F8F7C6FDF8BDC046DD
:104860003E9C03005BAA0300F0B585B005000291F1
:104870000392F8F7D2FA041E05D12A001A49012042
:1048800008F0CCFC2DE00520F8F7C9F9041E29D06A
:1048900001221649280003F058FD060001002800F7
:1048A000FFF796FF300003F0B1FB07000100104A4C
:1048B000200003F04AFB32003900F8F789FD00239D
:1048C0002800019300932200039B029902F0FCFB55
:1048D000051E04D02000F8F753FD280002E0F8F789
:1048E0004FFD200005B0F0BD6E9C030090880300D2
:1048F00052880300F0B5334C87B0A068250002232E
:10490000C65E982300275B009E420FD1F8F763FE36
:10491000A368013702229B5EB34207D138002A49BF
:1049200008F07CFC0FF074FF002049E000230593A1
:1049300000F0E8FB05A902F0B5FAAB68040002221A
:104940009B5E282B0BD0002F04D10598F8F718FD9B
:10495000200035E01F22AB8E1340012BF5D108F06B
:10496000D5F803900028F0D1200003F04FFB06009B
:10497000002F11D01F22AB8E1340012B0CD1AB683E
:1049800002229A5E283A51425141CAB22100FFF7F1
:104990006BFF039F029009E00023059A01930093A7
:1049A00021000133300002F08FFB02903100200023
:1049B000059AF8F70DFD002305A905930298BAE7BB
:1049C00007B0F0BD8C5A00209A9C030070B5194EB8
:1049D000B06845882B00143BFF3B012B23D8F8F728
:1049E000FAFDFFF7F3FF1F230400B08E18400128E3
:1049F0001CD106F0A1FB14232DB2FF3306002B229D
:104A00009D4200D0023231002000FDF7D7FC0500A6
:104A10003000F8F7B5FC2000290008F0ABFC2800B6
:104A2000F8F7AEFC02E0FFF765FF04002000FFF797
:104A30000BFE70BD8C5A0020F8B502271F26294DA9
:104A4000A86843881CB2212C06D07E2C04D02B3BB6
:104A5000BB439BB2002B42D1F8F7BDFDA88E30407E
:104A6000051E012DEBD1212C0AD1FFF7E5FF03F044
:104A700025FBF8F700FD6840C0B206F054FB30E0BB
:104A80007E2C09D1FFF7D8FF03F018FBF8F709FDDA
:104A9000C04306F051FB24E02D2C10D1FFF7CCFFD2
:104AA0000600002006F048FB220031000500FDF75B
:104AB00085FC310004002800F8F796FC0DE000208A
:104AC0002B2C0ED1FFF7B8FF03F0F8FA050003F026
:104AD00097FB04002800F8F753FC200001E0FFF7E3
:104AE00075FFF8BD8C5A0020F0B5934C87B0A368D1
:104AF000059106000220185EFFF74AFD05000394A9
:104B0000002D00D115E1059B9D4200D811E18A4F8F
:104B1000BB68B8685C8823B20093F8F75CFD022399
:104B20009C431A2324B2FF339C422FD1300003F060
:104B30006DFAF8F7A0FC002803D1009BA3421BD11B
:104B400004E01C23009AFF339A4215D1039B9C8EEC
:104B500007F0F8FEFFF770FF2900FFF7C5FFF8F731
:104B60000FFC039BA4B29A8E744B1A40744B1C40EA
:104B7000039B14439C86D4E03000F8F701FCFFF758
:104B80005BFF2900FFF7B0FF0600CAE0FFF754FF04
:104B90002900FFF7A9FF1F230190BF8E3B4002931E
:104BA000012B00D0BAE03223009AFF339A4236D16B
:104BB000300003F02BFA0500019803F027FA0400F7
:104BC000F8F715F9002804D12000F8F71BF9071EA3
:104BD00017D0280006F0DAFE0022010005002000B0
:104BE00003F0DEFD07003000F8F7CAFB3800431E73
:104BF0009841C0B206F097FA06003800F8F7C0FBFB
:104C000008E022004F49029808F008FB3000F8F74E
:104C1000B7FB3E0021002800F8F7E6FB7EE0992371
:104C2000009A5B009A426FD1300003F0EFF9050063
:104C3000019803F0EBF90700F8F7EFF8041E05D12F
:104C40003A004149029808F0E9FA53E02800F8F7E1
:104C5000D9F800280AD12800F8F7DFF8002805D194
:104C6000280001F07DFE011E30D134E000223749DA
:104C7000380002F0DFF8002202903549280003F0E6
:104C800052FC002304000093002C0FD0029B9C4296
:104C900001D10123009300222D49200003F043FCA1
:104CA00004902000F8F76CFB049CEDE729493800DC
:104CB000FCF76CFA002801D0012300930298F8F762
:104CC0005FFB009B002BCBD0012413E03800FCF7E6
:104CD0005DFA0028F8D12800F8F789F8041E04D1FD
:104CE0002800F8F763F8002804D01A493800FCF7C8
:104CF0004DFA0400320039002800F8F769FB200063
:104D000006F011FA060009E0009A01993000FDF75B
:104D100055FB04003000F8F733FB26000198F8F744
:104D20002FFB054B9B680220185EFFF731FC050046
:104D3000E6E6300007B0F0BD8C5A0020C0FCFFFF53
:104D40003F030000C19C0300E99C0300908803001E
:104D5000528803003989030010B5FFF76DFE00216A
:104D6000FFF7C2FE00F0DCF800F018F810BD70B5D7
:104D70002825094CA38E2B420CD1FFF7EDFFA36829
:104D800002229B5E2C2B06D1F8F7FAFAA068F8F7FE
:104D900022FCEEE7002070BD8C5A0020F7B55E4A79
:104DA00005009068438801921EB23D2E0BD00C3B4B
:104DB000FF3B9BB2112B00D9ABE0584ADA401300FD
:104DC000DB0700D4A5E0F8F706FCFFF7C5FF03F00A
:104DD00075F9019B07009A8E1F231340012B7ED18A
:104DE000002D7CD0341E3D2C1BD12B7A002B13D1EF
:104DF0002800F7F78DFF00280ED02800F7F7CBFF2B
:104E0000002809D12800F7F793FF002804D1019B5F
:104E10002900186802F0F2FF3900280008F0AAFA09
:104E20005DE01223FF339E4223D001339E425AD0CD
:104E30001623FF339E4258D001339E4257D0182389
:104E4000FF339E4255D001339E4254D002339E42DE
:104E500053D002339E4252D01023FF339E4250D093
:104E60000C23FF339E424FD005339E424ED02B2E53
:104E700026D12800F7F74CFF2B24002822D0280049
:104E800003F0C4F80600F8F71FF9002815D0300029
:104E9000F7F7E0FF019000280FD1337A012B0CD1F6
:104EA0000100380006F068FB04000100300006F045
:104EB000FCF92000F8F764FA019C3000F8F760FA7A
:104EC000002C0CD0220039002800FDF777FA0400EE
:104ED0000100280008F04EFA2000F8F751FA3800D7
:104EE000F8F74EFA15E02D24ECE72A24EAE72F2400
:104EF000E8E72524E6E72624E4E77C24E2E75E24CD
:104F0000E0E70E24FF34DDE7852400E08724640019
:104F1000D8E72800FEBDC0468C5A0020F1BC020034
:104F200070B52F4C0500A36802215A5E3F2A54D168
:104F30001800F8F750FB1F23A28E1340012B10D04E
:104F4000FFF70AFFF8F71CFA3A21A068F8F706FF06
:104F5000002801D1002540E0FFF7FEFEF8F710FA27
:104F60003BE0280003F052F8F8F785FA0600280025
:104F7000F8F706FA002E18D0FFF7EEFE3A210500EA
:104F8000A068F8F7EBFE0028E4D0A38E9EB207F0ED
:104F9000D9FCFFF7E1FEF8F7F3F9A28E114B1A40A6
:104FA000114B33401343A38617E0A38E9DB207F045
:104FB000C9FCFFF7D1FEF8F7E3F9A28E094B3A21BD
:104FC0001A40094BA0682B401343A386F8F7C6FE8E
:104FD0000028BFD0FFF7C0FE0500280070BDC04606
:104FE0008C5A0020C0FCFFFF3F0300001F23F7B5D1
:104FF0002B4C0026A28E1340012B07D10320F7F77C
:105000000EFE061E02D10FF003FC46E05B21A068F5
:10501000F8F7A4FE002700283FD02823A58E1D40C6
:1050200003D0002E35D0376033E0A36802229A5EA9
:105030005D2AF6D01F21A38E0B40012B18D12C2AFC
:1050400014D0FFF789FE03F039F80500380006F0A8
:1050500073F8290006F0D0FC0190002806D001006A
:10506000300002F0CBFE0198F8F78AF9280001E041
:10507000FFF772FEF8F784F9A0680222835E5D2BC9
:1050800001D10137C9E72C21F8F768FE0028F8D1D3
:1050900003E05D21A068F8F761FE3000FEBDC04668
:1050A0008C5A002070B5154DA868F8F794FAFFF7F0
:1050B000C3FC1F23AA8E040013400025012B18D126
:1050C000F7F726FEA8420BD02000F7F711FEA84202
:1050D00006D12000F7F7E8FDA84201D1084805E015
:1050E000200002F0EBFF040005F0B8FFF8F7ECFE3B
:1050F00005002000F8F744F9280070BD8C5A002004
:1051000073B00300F8B56E4FB8683D000223C65E69
:1051100080235B009E420CD10300002264331B7885
:10512000C3180133DA77203001F07CFF0400B8683F
:1051300016E00223FF339E4215D1BA8EE23B1340A4
:105140000024012B0BD1030064331B78C3180133F7
:10515000DC77203008F0ECFA06F003F80400A868C9
:10516000F8F739FAA9E081235B009E4211D1BA8E8B
:10517000E33B13400024012BF1D1030064331B787F
:10518000C3180133DC7720300FF00EFE05F0C0FFAE
:10519000E4E7282E12D1F8F71EFA08F097F8002855
:1051A00000D189E0FFF7E3FDBB8E0400334200D05D
:1051B00083E02921B868F8F7D1FD7EE096235B00F3
:1051C0009E4207D1F8F707FA1F23B88E184001282E
:1051D0000CD071E02E23FF339E420AD1F8F7FBF981
:1051E0001F23BA8E1340012B66D1002005F09BFFD0
:1051F00052E097235B009E420AD1F8F7ECF91F2397
:10520000BA8E1340012B57D10220F7F708FD43E077
:105210003023FF339E420BD00423FF339E420AD13A
:10522000BA8EE43B1340012B02D1F8F79DFE95E7BF
:10523000F8F7D1F940E07B2E02D100F09DF82BE089
:105240005B2E02D1FFF7D2FE26E092235B009E4246
:1052500005D1F8F7C0F9012002F07EFB1CE02823FD
:10526000FF339E420BD1F8F7B6F93C6B002C00D10E
:105270003C688022638992009B1863811DE09B2318
:105280005B009E4202D100F01DF805E03823FF3399
:105290009E4203D1FFF706FF04000EE09C235B0053
:1052A0009E4206D1F8F797F9FFF72CFFF8F768F858
:1052B00002E00021F8F752FD00242000F8BDC046AE
:1052C0008C5A0020F0B500262A4C85B0A068F8F76B
:1052D00082F90396FFF716FF03A901F0E3FD1F23F0
:1052E000A28E05001340012B3DD1F7F711FDB0420E
:1052F00001D1002034E02800F7F71AFD0028F8D18A
:10530000039E002E22D12800F7F7F6FB26680190B5
:105310003000F7F7C9FC0600002E14D0019BB34201
:105320000AD03000F7F7DAFB0700F7F770FC060049
:105330003800F8F725F8EFE78021236889005A89BB
:10534000039352185A81039E002ED2D03000F7F7F3
:1053500064FD0028CDD13000290002F0E6FC0120D8
:1053600005F0E1FE060028000399F8F73DF830004B
:1053700005B0F0BD8C5A00201F23F7B53F4DAA8E13
:105380002E001340012B72D10520F7F748FC041EB4
:1053900002D10FF03DFA6EE07B21A868F8F7DEFC41
:1053A000002868D02823B58E1D405BD1B0684388A3
:1053B0001AB27D2A56D0802149008A4202D01C317F
:1053C0008A420CDD1F23B28E00251340012B02D12F
:1053D000F8F7CAFD0500B068F8F7FDF812E09BB2D7
:1053E0009A1EFF3A022A03D92D3BFF3B032B03D819
:1053F000FFF788FE050005E080214900F8F7AEFCC4
:10540000002838D03A21B068F8F7A8FC002803D16A
:105410002800F7F7B5FF2EE01F23B78E1F40012F9E
:1054200016D1280006F0B2FA3A000100050020006B
:1054300003F0B6F9071E0BD0FFF78EFC02F03EFE1C
:1054400001000190380002F0DAFF0199F7F7CCFF74
:105450002800F7F795FFB0680222835E7D2BA1D06C
:105460002C219BE77D21B068F8F778FC03E0FFF77B
:105470007FF9002000E02000FEBDC0468C5A0020CD
:10548000074A10B5140000230C40944206D10903CA
:105490000133002902D10300581E8341180010BDBA
:1054A0000000F07FC80F704773B5160004000D00B0
:1054B0002B0C5A04520D26D1002200232000290073
:1054C0000094019510F042FC00284BD1002E09DD1C
:1054D000009A019B1000190010F0D2FC013E04005C
:1054E0000D000DE0002E3AD0330035333ADB009842
:1054F000019900221D4B11F013FC04000D00013630
:10550000002ED5D12BE0B618194A964206DD0122AD
:1055100080215242174B0020C90513E0002E14DCF5
:10552000320035321EDB10221349A8B20B40134360
:10553000934018430500721E00201049FFF7B4FF86
:1055400022002B0011F0ECFB0EE032010A490C4E58
:105550000B4016401E43A8B236043043050020001D
:10556000290001E0002000217CBDC0460000E03F92
:10557000FE070000FFFFEF7F0F80FFFF0000F03FFE
:10558000F07F0000F8B54C00150006000F00640D18
:1055900017D10022002310F0D9FB002803D02C6083
:1055A000002000211AE004003000390032003B00E6
:1055B00010F066FC060048000F00013C400DF3D0DF
:1055C0000419074B3A14E418064B30001340064AFE
:1055D0002C6013431B04BAB21A431100F8BDC04635
:1055E00002FCFFFF0F80FFFFE03F0000F7B50B005C
:1055F000020006000F0012F061F934003D0000289F
:105600004FD130003900FAF7B3F9002849D0002211
:1056100000233000390010F099FB002841D16B467F
:1056200000940195DB88214A5B045B0D9B180BD528
:10563000002200233000390010F08EFB00240025EA
:1056400000282ED01A4D2CE03422D31A6A460F2B94
:1056500003DD1080103B0232F9E7002B05DD154811
:105660005B0011881B5A0B4013800022002330007E
:10567000390010F071FB002811D0009C019D300012
:1056800022002B00390010F061FB002807D1002216
:10569000094B2000290011F0BDFD00900191009CF4
:1056A000019D2000290003B0F0BDC04601FCFFFFB2
:1056B0000000F0BF289D03000000F03FF8B5020095
:1056C0000B0004000D0012F0F9F826002F0000284E
:1056D0002ED120002900FAF74BF9002828D020000D
:1056E0002900FFF783FF06000F0002000B002000D7
:1056F000290010F045FB002807D0300039000022B7
:105700000D4B10F0BDFB06000F00002200233000FF
:10571000390010F01BFB00280AD0002200232000D3
:10572000290010F019FB002802D0802700263F0630
:1057300030003900F8BDC0460000F03FD0B506008B
:105740004C00640C23040C04240C1C430022002392
:1057500030002100270010F0FFFA002803D080213C
:10576000090663181F0030003900D0BDF7B50B00E3
:10577000020004000D0012F0A1F822002B00002806
:1057800076D13D4A3D4B2000290010F0F9FA00285F
:1057900069D13B4A3B4B2000290010F0DDFA00287C
:1057A00064D1394A394B2000290011F0B9FA00229E
:1057B000374B10F065FBFFF719FF0022354B0090C7
:1057C000019111F0ADFA02000B002000290011F048
:1057D00021FD314A04000D00009801992F4B11F072
:1057E0009FFA02000B002000290011F013FD0200B7
:1057F0000B0006000F0011F093FA294A0223283209
:1058000004000D00F9F7A4FB02000B003000390082
:1058100011F086FA06000F00214A032340322000CF
:105820002900F9F795FB32003B0011F0F3FC020070
:105830000B003000390010F04FFE02000B0010F09A
:105840001FFB184B002210F01BFB04000D000098FA
:10585000019912F053F8290002002000FFF724FEFE
:1058600002000B0004E000220F4B01E000220023A5
:105870001000190003B0F0BDEF39FAFE422E864049
:1058800052302DD5104987C0FE822B654715F73F52
:105890000000E03F402EE63FCAAB79CFD1F7B73EDC
:1058A000289D03000000F03F0000F07FF7B50B00DB
:1058B000020004000D0012F001F822002B00002865
:1058C0005CD100222F4B2000290010F059FA002251
:1058D000002852D12C4B2000290010F03DFA002264
:1058E000002300284AD1294B2000290010F0C8FAD3
:1058F000FFF77CFE0090019102000B0020002900C0
:1059000011F088FC02000B0006000F0011F008FAED
:105910001F4A0223603204000D00F9F719FB020050
:105920000B003000390011F0FBF906000F00184A97
:105930000223783220002900F9F7F6FA32003B0002
:1059400011F068FC0B0002003900300010F0C4FDBB
:105950000122FFF7A9FD0F4B002210F091FA04007D
:105960000D000098019911F0C9FF290002B2200032
:10597000FFF79AFD02000B0000E0074B1000190032
:1059800003B0F0BD00009040000090C00000E03F78
:10599000289D03000000F03F0000F07FF7B50B00EA
:1059A000020004000D0011F089FF22002B000028E6
:1059B00075D13D4A3D4B2000290010F0E1F9002847
:1059C00068D1394A3A4B2000290010F0C5F9002867
:1059D00063D1384A384B2000290011F0A1F9002288
:1059E000364B10F04DFAFFF701FE0022344B0090C9
:1059F000019111F095F902000B002000290011F02F
:105A000009FC304A04000D00009801992E4B11F05A
:105A100087F902000B002000290011F0FBFB0200B7
:105A20000B0006000F0011F07BF9284A032308320F
:105A300004000D00F9F78CFA02000B003000390069
:105A400011F06EF906000F00204A032328322000CF
:105A50002900F9F769FA32003B0011F0DBFB0B007B
:105A600002003900300010F037FD0122FFF71CFD65
:105A7000174B002210F004FA04000D000098019961
:105A800011F03CFF290002B22000FFF70DFD0200DB
:105A90000B0004E000220F4B01E000220023100065
:105AA000190003B0F0BDC046FE799F501344734007
:105AB000134473C071A379094F930A400000E03F7B
:105AC0000044D33F12F3FE799F50D33EA89D0300BC
:105AD0000000F03F0000F07F70B50B0002000C00EA
:105AE000050011F0EBFE2100002845D10022002323
:105AF0002800210010F030F9002802D080231B0676
:105B0000E4181E4A1E4B2800210010F039F9002825
:105B100030D11C4A1C4B2800210010F03BF9002812
:105B200012D00022194B2800210011F0F9F8FFF7DC
:105B30001DFE0022154B04000D0011F0F1F80200CB
:105B40000B002000290011E028002100FFF70EFEC5
:105B500004000D0002000B0000200D4910F0BCFCF9
:105B600022002B0010F08CF90022084B11F0D8F81D
:105B7000050001E000250749280070BD7DF8B98FB8
:105B8000CE338640617B3A6EB72886400000E03F06
:105B90000000F03F0000F07FF0B51600012285B054
:105BA0001F005242524B05000C0010F0E9F800288B
:105BB00002D000264F4C97E001224D4B524230005C
:105BC000390010F0DDF80028F3D101224A4B52428F
:105BD0002800210010F0C0F80028EAD10122464B2D
:105BE00052423000390010F0B7F80028E1D12A0005
:105BF00023002800210011F061FE00286ED1320040
:105C00003B003000390011F059FE002868D16400D3
:105C100064087F0000220023280021007F0810F084
:105C200095F800285CD1002200233000390010F0E4
:105C30008DF8002852D102AA28002100FFF7A2FC0B
:105C400003AA30003900FFF79DFC029A039BD11A8A
:105C50001B2943DC1B3143DBD3185B1000935B42F1
:105C60001A00280021000193FFF71EFC019A04008E
:105C70000D0030003900FFF717FC220006000F006E
:105C80002B002000290011F04BF8320004000D0019
:105C90003B003000390011F043F80B0002002900EE
:105CA000200010F0EDF8F9F797F803AA04000D00B2
:105CB000FFF768FC039A009B9B1880220393D20095
:105CC000934200DD75E70D4A93420BDB2000009AFA
:105CD0002900FFF7E9FB06000C0005E02E0003E0B9
:105CE0003C0001E0002634003000210005B0F0BD8A
:105CF000FFFFEF7F0000F07FFFFFEFFFCBFBFFFF19
:105D0000F0B587B0019002000B0001980E0011F071
:105D1000D5FD002800D0C3E001983100F9F728FE36
:105D2000002800D1BCE0002200230198310010F0CF
:105D30000DF8002800D0B3E00023002201983100C4
:105D400010F01EF801230393002805D180231B06C1
:105D5000F61801235B42039305AA01983100FFF76F
:105D600011FC04000D00514A514B10F0D9FF514A6B
:105D7000514B10F085F822002B0010F0D1FF4F4A54
:105D80004F4B11F047FA22002B0010F0C9FF4D4A8B
:105D90004D4B10F075F822002B0010F0C1FF4B4A5C
:105DA0004B4B10F06DF8059F04000D00002F17DB22
:105DB000380003210FF0C2FE83000590C01AC719F6
:105DC000012F02D1434A444B03E0022F23D1434A1F
:105DD000434B2000290010F0A3FF04000D001AE03F
:105DE000784203210FF0AAFE030002908000181AE7
:105DF000C71B012F02D1394A3A4B03E0022F07D1CA
:105E0000344A394B2000290010F08AFF04000D00AD
:105E1000029B5B420593059A20002900FFF744FB93
:105E200002000B0004000D0010F07AFF02000B00CE
:105E30000198310010F050FB02000B0020002900F7
:105E400011F0E8F9294A2A4B10F06AFF02000B0012
:105E50002000290011F0DEF902000B0004000D0003
:105E600010F05EFF02000B000198310010F034FBCF
:105E700002000B002000290011F0CCF91B4A1C4B3A
:105E800010F04EFF0B0002002900200011F0C2F9B3
:105E900003000398013005D180221206891801E021
:105EA0003100019B180007B0F0BDC046F6DF6F3827
:105EB000933CC1BF589DE5C71F7EE13FB837BAA3E9
:105EC0004C8AEE3F3A8705E56E3DF23FFEA4222163
:105ED000C1C0D93F8B728DF9A228F43F3D6E3DA51C
:105EE000FE65F93FFE65E93FA228E43F555555554B
:105EF0005555D53FF0B5002285B0002304000D00B4
:105F00000FF024FF071E00D07DE06E00760800220F
:105F10003F4B200031000FF03DFF002812D000223F
:105F20003B4B200029000FF011FF061E66D1002216
:105F3000384B200029000FF009FF002861D0340001
:105F4000354D60E0354A364B200031000FF004FF3C
:105F5000002858D10022334B200031000FF0FCFE06
:105F600000282ED022002B002000290010F0D8FE9F
:105F700006000F0002000B002000290010F0D0FEE8
:105F8000294A029003914032042330003900F8F787
:105F9000DFFF254A00900191683205233000390067
:105FA000F8F7C2FF02000B000098019910F094FA74
:105FB000029A039B10F0B4FE22002B000FF060FF4A
:105FC00019E00022124B200029000FF059FF220097
:105FD00006000F002B0000200D4911F01BF90200F4
:105FE0000B003000390010F077FAF9F789F9002238
:105FF0000C4B10F095FE04000D0004E03C000B4D2E
:1060000001E004000A4D2000290005B0F0BDC046A3
:106010000000F03F0000F0BF0000F0FF48AFBC9A66
:10602000F2D77A3E0000E03FA89D03000000F07F19
:106030000000F87FF0B5002287B000230D000400B7
:106040000FF084FE2900002800D0AFE00122594B58
:106050005242200029000FF093FE002800D0A0E05B
:106060000122554B5242200029000FF075FE0028F6
:1060700000D099E000230022200029000FF06CFEE0
:106080000123002803D080231B06ED184B4B0393FC
:106090004B4A4C4B200029000FF072FE071E0ED019
:1060A00022002B000020484910F016FA80231B061E
:1060B000CD18012304000293444A454B25E0454A8C
:1060C000454B200029000FF051FE00281AD1002274
:1060D0003D4B2000290011F09DF8002206000F0022
:1060E000394B200029000FF0CBFE02000B003000DE
:1060F000390010F0F1F90223040002930D00334A35
:10610000364B02E000220023029700920193200008
:1061100022002B00290010F003FE314A0423103224
:106120000F000600F8F714FF02000B0030003900E2
:1061300010F0F6FD2A4A0490059138320523390003
:106140003000F8F7F1FE02000B000498059910F0FA
:10615000C3F922002B0010F0E3FD0B000200290020
:1061600020000FF08DFE6B460827DF5F022F02D163
:106170001C4A1D4B03E0012F03D11A4A1B4B0FF0A1
:106180007FFE02000B00009801990FF079FE6A462D
:1061900004000C20125E013208D180231B06C918AE
:1061A00004E00A4C0A4901E0084C1149200007B0FC
:1061B000F0BDC046FFFFEF7FFFFFEFFFFFFF0000D6
:1061C000E69D3F334F5003400000F03F182D4454EC
:1061D000FB21F93F1F85EB51B81EE53FFB21E93F4D
:1061E000289E0300075C143326A6813C26A6913C1A
:1061F000FB21F9BFF7B505000C00100019001700CE
:106200001E0011F05BFB002800D0F2E02A00230002
:106210002800210011F052FB002800D007E10022E5
:106220000023280021000FF091FD00220023002808
:1062300027D038003100002C11DA0FF0A1FD002822
:1062400000D0F4E000220023380031000FF084FD7C
:10625000002800D088E0002E00DBE8E084E00FF0AA
:1062600075FD051E04D0F50FED0700D187E07DE038
:1062700000220023380031000FF082FD00287ED17B
:1062800074E0380031000FF061FD002809D02800CB
:106290000022002321000FF073FD674D002879D103
:1062A0007BE00122654B5242380031000FF068FD5F
:1062B0000122524200281BD0604B280021000FF021
:1062C0005FFD002855D101225D4B5242280021007C
:1062D0000FF042FD061E4FD12800002200232100AE
:1062E0000FF03AFD3500002800D08EE0050046E0B2
:1062F000534B380031000FF02FFD01224F4B52421B
:10630000002818D0280021000FF03AFD002838D1CD
:1063100001224B4B5242280021000FF01DFD0028A6
:1063200032D128000022002321000FF033FD424D1E
:1063300000281CD12BE0280021000FF021FD0028AF
:1063400027D101223E4B5242280021000FF004FDCC
:10635000002821D100220023380031000FF0FCFC7E
:106360000090002857D01AE0334D10E0324D354CE4
:106370005DE0314D344C5AE02F4D344C57E02C0049
:1063800055E0334D334C52E0314D334C4FE0334CFC
:106390004DE0294D324C4AE0274D324C47E0002277
:1063A0000023280021000FF0D7FC002830D0022263
:1063B000012313431BB2022B2AD0032B34D11E4AD4
:1063C000264B0092019328003A003300210010F080
:1063D00083F8FFF72FFE02000B00009801990FF0E1
:1063E0004FFD0022002307000E000FF0AFFC002835
:1063F00002D13D0034001AE00022002328002100D1
:106400000FF0AAFC0028F4D00025802424060EE01A
:10641000094A0C4BD5E700220023280021000FF089
:106420009BFC009A0028C3D100220023C9E7280062
:10643000210003B0F0BDC046182D4454FFFFEF7F8C
:10644000FFFFEFFFFB210940FB21E93FFB21E9BFF3
:10645000D221337F7CD902407CD902C0FB2109C004
:10646000FB21F93FFB21F9BFF0B5002285B00023E5
:1064700004000F000FF06AFC002800D08EE000221C
:106480000023200039000FF067FC002805D080238E
:106490001B06FD1801235B4201E03D00012301932F
:1064A0000022404B200029000FF06AFC00281ED07B
:1064B00001223D4B5242200029000FF061FC0028D0
:1064C0006CD120002900F8F71BFF040001980D0093
:1064D00011F04AFA354A06000F00354B200029001A
:1064E0000FF0CEFC02000B003000390052E0220019
:1064F0002B002000290010F013FC002206000F00E2
:106500002C4B200029000FF027FC00282BD02A4A12
:106510000423603230003900F8F71AFD274A029050
:1065200003910423083230003900F8F7FDFC020023
:106530000B00029803990FF0CFFF32003B0010F0E0
:10654000EFFB22002B0010F0EBFB02000B00200001
:1065500029000FF095FC019A040001321FD180231D
:106560001B06C9181BE00022154B300039000FF044
:1065700087FCF8F731FC02000B00200029000FF027
:106580007FFCF8F7BDFE04000D00019811F0ECF956
:1065900022002B0010F0C4FB040000E039002000B2
:1065A00005B0F0BD84D79741FFFFEF7FEF39FAFECA
:1065B000422EE63F0000E03F289E0300A89E030015
:1065C0000000F03FF0B5002287B0002304000E0069
:1065D0000FF0D6FB002804D180231B06F518514B81
:1065E00001E035000123019300224F4B20002900D8
:1065F0000FF0C6FB002800D08EE000224B4B20009D
:1066000029000FF0BDFB002847D022002B000020FE
:10661000454910F0FFFD464E0423320028320400A5
:106620000D00F8F795FC02000B002000290010F087
:1066300077FB32000490059150320423200029009A
:10664000F8F772FC22002B00029003912000290031
:106650000FF016FCF8F7C0FB02000B0006000F005D
:106660003448354910F0D6FD029A039B04000D0012
:10667000049805990FF030FF32003B0010F050FBFA
:106680002E4A2F4B10F0C6FD02000B0020002900FF
:1066900010F0C0FD274A284B31E02A4A2A4B20003F
:1066A00029000FF059FB002838D122002B002000D0
:1066B000290010F035FB1E4A0523703206000F003A
:1066C000F8F746FC02000B003000390010F028FB00
:1066D0001E4A029003910523203230003900F8F75A
:1066E00023FC02000B00029803990FF0F5FE220034
:1066F0002B0010F015FB02000B00200029000FF00A
:10670000BFFB6B4604229B5E04000E00013305D1E3
:1067100080231B06CE1801E000240D4E200031001E
:1067200007B0F0BDFFFF00000000F03F0000E43FB5
:10673000A89E0300182D4454FB21E93F075C143345
:1067400026A6913C3A8C30E28E79453E289F030084
:106750000000F87F70B500221F4B04000D000FF001
:10676000FBFA002835D100221C4B200029000FF035
:1067700007FB00282DD10022194B200029000FF023
:10678000FFFA002812D00022154B2000290010F03B
:10679000C7FA02000B000020114910F03BFDF8F78A
:1067A0001BFBFFF70FFF02000B000FE0200029008A
:1067B000FFF708FF02000B000A480B4910F02AFD02
:1067C0000A4A0B4B0FF05CFB064A074B0FF058FBD5
:1067D00001E00020074970BD0000F0BF0000F03F5D
:1067E0000000E03F182D4454FB21E93F075C1433BF
:1067F00026A6913C0000F87FF7B5364B0022040036
:106800000D000FF0A9FA00285DD10022324B2000C4
:1068100029000FF0B5FA002811D001222F4B524267
:10682000200029000FF0ACFA00284FD120002900E9
:10683000F8F766FD2A4A2B4B0FF022FB48E00022B6
:10684000244B2000290010F0E5FC0022264B060016
:106850000F000FF081FA002820D030003900F8F73F
:10686000BBFA224A04000D004832042330003900EC
:10687000F8F76EFB1D4A009001917032052330003D
:106880003900F8F751FB02000B00009801990FF056
:1068900023FE22002B0010F043FA19E000220D4BDA
:1068A000200029000FF0ECFA32003B0010F038FA1B
:1068B000F8F792FA02000B00200029000FF0E0FA2E
:1068C000F8F71EFD04E00020094901E00020094915
:1068D00003B0F0BD0000F03F84D79741FFFFEF7F8A
:1068E000EF39FAFE422EE63F0000E03F289F03000A
:1068F0000000F87F0000F07FF0B585B0039301231E
:1069000005000C005B4202920093002C26D02F78E9
:106910006B1C01930399029B38009847009B661EED
:10692000BB4217D10222FF3201239446E918E61A2E
:10693000581E01919C4208D0E95C009A8A4205D118
:1069400001336345F2D1FF2000E00026C0B2039975
:10695000029B984700973400019DD6E705B0F0BD33
:1069600070B50400F6F759FA2A4B00284FD12000E1
:10697000F6F71CFA051E09D02279274B142A46D0B7
:10698000264B412A43D0264B042A40D02000F6F75C
:106990001CFC244B00283AD1002D03D02279224B35
:1069A000812A34D02000F6F72DFA204B00282ED172
:1069B000002D09D022791E4B012A28D01D4B022A16
:1069C00025D01D4B282A22D02000F6F733FA1B4B86
:1069D00000281CD1002D03D02279194B112A16D082
:1069E0002000F6F704FA174B002810D1002D06D02E
:1069F0002279154B122A0AD0144B242A07D02000E2
:106A0000F6F762FB421E9041114B404203401800D2
:106A100070BDC0461FA90300C09F0300CB9F0300A9
:106A2000DD9F0300E99F0300ED9F03003989030008
:106A30003BA003002FA0030022A003001BA0030023
:106A400011A0030000A0030006A00300F99F0300AB
:106A5000CDA5030070B57149040011F022F901259C
:106A6000002800D1D7E06E49200011F01AF9002863
:106A700000D1D0E06B49200011F013F9002800D1BB
:106A8000C9E06949200011F00CF9002800D1C2E0EA
:106A90006649200011F005F9002800D1BBE06449E7
:106AA000200011F0FEF8002800D1B4E06149200078
:106AB00011F0F7F8002800D1ADE05F49200011F097
:106AC000F0F8002800D1A6E05C49200011F0E9F8B8
:106AD000002800D19FE05A49200011F0E2F8002878
:106AE00000D198E05749200011F0DBF8002800D1D0
:106AF00091E05549200011F0D4F8002800D18AE037
:106B00005249200011F0CDF8002800D183E050490F
:106B1000200011F0C6F800287DD04E49200011F069
:106B2000C0F8002877D04C49200011F0BAF80028AE
:106B300071D04A49200011F0B4F800286BD04849C0
:106B4000200011F0AEF8002865D04649200011F071
:106B5000A8F800285FD04449200011F0A2F80028CE
:106B600059D04249200011F09CF8002853D04049E8
:106B7000200011F096F800284DD03E49200011F079
:106B800090F8002847D03C49200011F08AF80028EE
:106B900041D03A49200011F084F800283BD0384910
:106BA000200011F07EF8002835D03649200011F081
:106BB00078F800282FD03449200011F072F800280E
:106BC00029D03249200011F06CF8002823D0304938
:106BD000200011F066F800281DD02E49200011F089
:106BE00060F8002817D02C49200011F05AF800282E
:106BF00011D02A49200011F054F800280BD0284960
:106C0000200011F04EF8002805D02649200011F090
:106C100048F845424541280070BDC04600A0030029
:106C2000ED9F030094AA03003BA00300CB9F030049
:106C300011A003002FA0030006A00300DD9F0300A6
:106C4000C09F0300F99F030022A0030046A0030099
:106C500078A003004BA0030057A0030061A003002D
:106C60006FA00300C0A703001FA903007EA00300BC
:106C700086A003008BA00300E99F03001BA0030074
:106C80003989030093A003009BA00300A3A0030085
:106C90004D9A030076B203005E9A0300CDA503006F
:106CA000ABA00300B0A0030070B5134C2821A0686E
:106CB000F7F754F8282500281CD0A38E2B4211D1B9
:106CC000A36802229B5E292B0CD0FEF745F8F6F74D
:106CD00057FBA0680222835E292BEED02C21F7F708
:106CE0003DF8E8E72823A28E1A4203D12921A068A3
:106CF000F7F734F8002070BD8C5A0020282170B5B9
:106D00001B4D0600A868F7F729F8002801D10020DC
:106D10002CE0A8680223C15E292925D0002E15D0B9
:106D200003000021020064331B782032C3180133B2
:106D3000D977300001F009F9041E02D10DF068FD89
:106D4000E5E704F031FF2000F6F71AFB8021A86880
:106D50004900F7F703F80028D9D0A8680222835E1B
:106D6000292BD6D02C21CEE7F6F7F8FF70BDC04610
:106D70008C5A0020F7B505000E00170005F0EAFD5B
:106D8000041E0BD131002800FCF7D2F8041E05D1F7
:106D90002800F6F742F8002817D133E0002F40D042
:106DA000200001F08BF901903000F7F78DF8019A7F
:106DB00001000700280001F096FD01990400380049
:106DC000F6F712FB002C2CD1E2E7174C3000210023
:106DD00010F067FF002815D10530F5F720FF0600F9
:106DE0002A00124901F08AFB22003100280001F03C
:106DF000ACF8010004002800FDF7EAFC3000F6F7CB
:106E0000BFFA0EE00A49300010F04BFF0024A04208
:106E100007D12800FFF7A4FDA04202D0FAF7CAF973
:106E200004002000FEBDC046908803005BAA03005A
:106E300052880300F8B505000E001700F6F7F3F9C5
:106E4000002807D13A0031002800FFF793FF041E05
:106E500020D107E000223100280001F076FA041E5C
:106E600018D1EFE72800F5F7D8FF002812D00C4919
:106E7000300010F016FF00280CD10530F5F7CFFEDA
:106E8000074A06000100280001F05FF80400300006
:106E9000F6F776FA2000002F01D101F00FF9F8BDC6
:106EA000908803000023F0B585B002900391019310
:106EB000594CA0680222835E2E2B51D1F6F78BFB32
:106EC0001F22A38E1340012B42D1A7680222BB5E72
:106ED00080225200934202D01C32934238DD3B00A4
:106EE000002264331B780298FB180133DA7701F033
:106EF0008DF82037061E12D13000F6F794F9051EE2
:106F000014D0A068F7F730F8002207000100300025
:106F100001F0E9FC05003800F6F732FA0CE0012236
:106F20003900FFF787FF051E06D1E5E733003A0079
:106F30003A49012006F072F9A068F6F74CFB019877
:106F4000F6F71EFA0298F6F71BFA01960295AFE7DC
:106F50008021A0684900F6F701FF0028A8D158E079
:106F60005B2B4DD1F6F737FBFDF7F6FE01F0A6F8E7
:106F70005D210500A068F6F7F1FE002804D1290084
:106F80000198F6F731FA44E01F22A38E1340012B3B
:106F900032D1280004F0FAFC0500029801F036F81E
:106FA000041E0BD12000F6F73EF9061E0CD000227D
:106FB0002900200001F097FC06000BE029000DF0ED
:106FC00031FC061E06D1EDE723002A0014490120FA
:106FD00006F024F90198F6F7D3F9002C04D08022AA
:106FE000638992009B1863810298F6F7C9F9200023
:106FF000F6F7C6F9019402962800F6F7C1F957E7AB
:10700000039B002B02D0019A1A6002E00198F6F768
:10701000B7F9029805B0F0BD8C5A0020B4A0030067
:10702000FBA00300F8B51F23264D0600AA8E0024FE
:107030001340012B14D1EB6A5F1E002F0ADBBB004B
:10704000EB1800223100D86801F07FF9041E07D147
:10705000013FF2E700223100286801F076F90400D0
:107060001F23AA8E1340012B29D1002C27D13000D9
:10707000FFF7F0FC310000280BD02000FBF758FF91
:10708000071E13D131002000FBF752FF071E0DD160
:1070900015E02000FBF74CFF041E10D13000F6F77E
:1070A00013FF210004F0A8FC040008E032003900BE
:1070B000286800F04AFF04003800F6F761F9200064
:1070C000F8BDC0468C5A0020F0B5B7B002AF7B6166
:1070D0001F23C54D3862B961FA60A88E1840012897
:1070E0000CD13B6A002B09D1002902D00A00BF490C
:1070F00001E0BA69BE4906F091F8C4E31F23AA8EE5
:107100001340012B06D01F23AE8E1E40012E00D04F
:10711000B4E304E006F0DAF80028F4D1B3E33B6A04
:10712000002B00D1AAE31800F5F777FE041E05D165
:107130003A6AB049300006F071F89DE37B69002B94
:107140001CD1386AF5F71FFE002800D143E128233F
:10715000FA18D018396A03F0E6FD2823FA18D01877
:1071600003F0D8FD2822C023BA18D3181B680500E5
:107170009B007B620023FB611C002CE02821A86897
:10718000F6F7ECFD0028DCD17DE32822C423BA18F1
:10719000D3181B688E0028009E1900F037FF2822A4
:1071A000C023BA18D3181A68306001321A60FB691C
:1071B00028000133FB61F6F7E3F82823FA18D0180A
:1071C00003F08DFD2823FA18D01803F0A3FD050065
:1071D0007B6A04337B622800F5F7BFFF002842D0AA
:1071E0002822C023BA18D3181B689C4218D8002C38
:1071F00001D0A40000E010246A46A3000833D31A8B
:1072000028219D46C4237918CB1802AE7A6A1968E2
:10721000300010F030FD2822C423BA18D3181E60A5
:107220002822C023BA18D3181B6828215A1EC42349
:107230007918CB181B68796A5B18F969043B91428D
:10724000A3DC1968013A5960F7E72800F6F798F8C7
:107250002823FA18D01803F042FD2823FA18D01872
:1072600003F058FD0500002D0AD06349280001F005
:1072700067F80028E9D0280000F0C8FE786201E035
:10728000FB687B622800F6F77BF82823FA18D018F1
:1072900003F020FD7B69002B6AD02822C023BA1896
:1072A000D3181B689D0028204F4B998E1A0001426D
:1072B0000CD090682921F6F751FD2822C023BA1876
:1072C000D3181B68FB61002852D1DCE29B685B8805
:1072D000292BEED0002BECD02822C023BA18D318CB
:1072E0001B689C4218D8002C01D0A40000E0102498
:1072F0006A46A3000833D31A28219D46C42379186F
:10730000CB1802AE2A001968300010F0B4FC282215
:10731000C423BA18D3181E602822C023BA18D31861
:107320001A68282101321A60C4237918CB181B6807
:107330005E19FDF711FD00F0C1FE2B4B306098681F
:107340000222835E292B11D02C21F6F707FD00289D
:107350000CD12822C423BA18D31828221968C023B4
:10736000BA18D3181868F6F727F88CE204359AE7AC
:10737000386A03F0B5FE1C4B7A6A1D6B002A05D0F3
:10738000127A796A01320A720A000EE01B4A9042B0
:1073900007D1002D00D178E22A7A01322A721D63CA
:1073A00073E21A68117A013111721A63002800D051
:1073B0006BE22822C423BA18D31819680400F869AC
:1073C000F5F7FAFF084B1A6B002A02D0117A01393F
:1073D00011721D6348E20620F5F721FCF8610028D0
:1073E0000ED10DF015FA4EE28C5A002075A1030063
:1073F0008CA10300A0A10300C5A10300999B02007A
:107400002C23396AF81803F08EFC2C23F81803F0AB
:1074100081FC2C230500F81803F075FC04002800FB
:10742000F5F79BFE00281FD0002C1DD0280001F08E
:107430000DF9061E0DD004F0B7FB2100300000F05E
:10744000DEFFF869310000F0D9FC3000F5F798FF55
:1074500001E00DF0DDF920002900F5F7C5FF2C2330
:10746000F81803F03CFCD0E729002000F5F7BCFF3A
:107470007B691D1E00D196E02823BE4EB48E1C40B1
:107480003300002C51D1B2680221525E292A4CD01F
:107490002C23F81803F03EFC0500F5F75EFEB368F8
:1074A000786202229B5E292B0CD100280DD1280086
:1074B000F5F766FF7B6A002BDED02C23F81803F06B
:1074C0000EFCD9E7FDF748FC00E0200000F0F6FDD7
:1074D0007B6A0600002B05D001220021280001F064
:1074E0004FF801E009F043FE041E0DD004F05CFBF0
:1074F0003100200000F083FFF869210000F07EFCDD
:107500002000F5F73DFF01E00DF082F93000F5F7BE
:1075100037FF984B98680222835E292BC7D02C2115
:10752000F6F71CFC0028C2D1ADE129219868F6F7D6
:1075300015FC002800D1A6E1FB687B620023BB603C
:107540001E007B611D004AE02C23F81803F0E2FBCB
:107550000600F5F702FE786200282CD001220021F7
:10756000300001F00DF8041E28D004F01DFB282186
:10757000C42279188A181268AB00D158200000F094
:107580003EFFF869210000F039FC2000F5F7F8FE15
:107590003000F5F7F5FE7B6A0135002B03D02C2374
:1075A000F81803F09CFB2822C023BA18D3181B68D4
:1075B0009D42C9DBC0E709F0DAFDD4E70DF028F9F8
:1075C000E6E703F0A7FB0400F5F77EFD00280CD1E9
:1075D0002000F5F7D5FE2C23F81803F080FB2C23B0
:1075E000FC6AF818002CECD14CE06349200000F054
:1075F000A7FE002804D0200000F008FD0500E7E702
:107600005E49200000F09CFE002804D0200000F01D
:10761000FDFC7861DCE75A49200000F091FE00286B
:1076200004D0200000F0F2FC0600D1E7554920000C
:1076300000F086FE002804D0200000F0E7FC78620D
:10764000C6E75149200000F07BFE002807D020004B
:1076500000F0DCFCF5F725FF83B2BB60B8E7200043
:10766000F5F77BFD0028B3D0200000F0EFFF386174
:107670000028ADD00100F86900F0C0FB3869F5F7CB
:107680007FFEA5E703F026FB002E10D03F4A210025
:10769000300003F0BFFE396A04F0AEF904000100C7
:1076A000F86900F0ABFB31002000F5F79DFE3823B0
:1076B0000024304A918E0B40A34200D0CEE014004B
:1076C000D16A39613A69934209DA9A00A1182826E9
:1076D000C8680821BE19711850500133F2E7002D17
:1076E00034D000232800E362F5F781FB002821D085
:1076F0002823FA182900D01803F015FB3B6D002B46
:1077000012D01C4EF46A631CF3622823FA18D018B6
:1077100003F0F9FA28230234A4003619FA1870602D
:10772000D01803F0DCFAE9E72833FA18D01803F090
:10773000D1FA07E001238022E3626B8992009B1853
:107740006B81E5602800F5F71BFE00E0E562F86953
:1077500005F0F2FD0024A04265D0064B1A6B7A605A
:107760007A6AA24214D0127A796A01320A720A0045
:1077700012E0C0468C5A0020CAA10300CFA103002A
:10778000D4A10300C5A10300D9A10300FFFFFF7F1F
:107790001A68117A013111721A637B691C1E37D085
:1077A0002823FA18D41879692000F6F760FB2822FC
:1077B0008E230121BA18D3183A895E4E1A805E4A88
:1077C00093689460BB60938E3B60938E33400B4311
:1077D00093863B6A5A893F231340072B6ED10222BE
:1077E000A35E00243B2B61D1534D3968AB8EAA8E2A
:1077F0001E40524B1340524A0A401343AB86282383
:10780000FA18D018F5F7CAFEBB68AB60002E68D135
:10781000494B1A6B002A02D0117A013911727A6829
:107820001A6305F06FFD0025434BDA6A954206DACC
:10783000AA00D318D868F5F7A3FD0135F4E70022B4
:1078400039698A4209DA28260825BE199100751976
:10785000581849590132C160F2E7D9627869F5F7E1
:107860008FFDF869F5F78CFD7B6AFA68200093427A
:107870005CD01800F5F784FD200057E07B69002BF1
:1078800001D0FFF711FA002050E03B6A28229988C6
:10789000C023BA18D3181B6828220093C423BA182F
:1078A000D3181B687A6A05F0F9FD82E57D2B9BD021
:1078B000FDF75DFA00F002FC040095E7214A002183
:1078C000F86900F042FB0500FCF7FEFE280000F01E
:1078D000F5FB0400002D87D00021280000F08FFD6B
:1078E00082E7AB8E68681E431A221749AE8600F005
:1078F0001AFE051E8CD0B869F5F7E6FB134900287F
:1079000000D11349BA69280003F036FB0A4B9B6883
:10791000002B03D0280005F0B6FB03E00D4928003A
:1079200003F02AFB2800F5F72BFD71E7BD4635B0C3
:10793000F0BDC046380C00008C5A0020C0FCFFFF90
:107940003F030000BD810300A182030040A10300AA
:107950005CA10300DEA103001F23F0B5BF4C93B070
:10796000A78E06001F4000230193012F03D106209C
:10797000F5F755F90190002303939E4210D0A068BB
:107980000223C25E80235B009A4209D1019B0393CC
:10799000002B02D0F6F7E8FA0390A068F5F71BFE7B
:1079A0000198FFF7ABF9051E04D101990398F5F78B
:1079B0001BFD08E07B21A068F6F7D0F9051E04D175
:1079C0000198F5F7DDFC280045E1019B002B11D063
:1079D000A36802229A5E2623FF339A420AD13F22ED
:1079E000019B5B899343383A1343019A5381A06802
:1079F000F5F7F1FD00230493012F15D1A0680300D2
:107A000066331B88002B0FD0C3684268806E9918BC
:107A100001390CAB07AA03F086FCA368079A66330A
:107A20001B889B18013B04938C4E0CADB368280057
:107A3000191DF6F73BFA012300245B420293B0685C
:107A40004388002B03D1012F00D0F1E016E01BB2D8
:107A5000002C0FD07B2B01D1013403E07D3B594238
:107A60005941641A436FC26E9B18013B0293F5F7AC
:107A7000B2FDE4E77D2B00D0E9E0E4E7029B002BB8
:107A800000DCD5E00E9B0C9A0CAE9B18FF1A029BF3
:107A9000FB180293102B25D91800F5F7E6F9041E00
:107AA00020D003F09FFA0500337D3100037007A852
:107AB0000AF021FE029B6E1CED18089B0293029AAD
:107AC000079B93420AD2B54208D007A809F048FBA9
:107AD000307007A80AF04EFD0136EEE70A98F5F778
:107AE0004FFC4FE009F043FB0700041E4AD0802200
:107AF000438992009B1843812B7D2900037007A8BE
:107B00000AF0F9FD0125089B0593059A079B93420E
:107B10000CD30A98F5F734FC200029000A300AF04B
:107B20008BFB2000F5F72CFC3C002BE0029B013B7B
:107B30000293002BEDD007A809F012FB059020005E
:107B4000F9F73FFFA84214D8200029000A300AF0B4
:107B500073FB2420F5F763F8061EDAD0F4F7CCFFA8
:107B600001002000F4F7D8FF2000F5F709FC3400ED
:107B700000256B461B7D6E1C635507A80AF0FAFCB6
:107B80003500C0E7364A2100019800F0DEF92100F7
:107B9000F5F72AFC314BDA6A1F00002A30D0012A9F
:107BA00006D18022DC68920063899B1863811FE004
:107BB0000320F5F734F800250400FB6A9D4215DA2E
:107BC000280003F0B9FAAB00FB18D96803F014FFE2
:107BD000061E02D10CF01CFE08E00100200000F09F
:107BE0000DF93000F5F7CCFB0135E6E7002C07D0A6
:107BF00021001C4A019800F0A8F92100F5F7F4FBD8
:107C0000049B002B0CD0180003F096FA041E07D03A
:107C10000100154A019800F098F92100F5F7E4FBFE
:107C2000039B002B04D01A001049019800F075FC4A
:107C30000CA8F6F744F9094B7D219868F6F78EF801
:107C4000041E019807D1F5F79BFB200003E07B2B76
:107C500000D007E700E713B0F0BDC0468C5A002003
:107C6000CFA10300CAA10300D9A10300D4A103003E
:107C700030B58BB0040003F0B1FD05002000F5F72E
:107C800013F8F4F72BFF2A000100040068460AF0FD
:107C9000FEFB68460AF099FD050068460AF002FB03
:107CA0002000F5F76DFB28000BB030BD70B5F4F780
:107CB000FBFF00240500002D0BD02800F4F70EFF79
:107CC0000600F4F7A4FF050030000134F5F758FB77
:107CD000F1E7200070BD10B50400F5F788F8002822
:107CE00003D0201E20D020681EE02000F5F75EF8AB
:107CF000002801D0608817E02000F5F7E5F900289A
:107D000003D0200003F0B6FB0EE02000F5F77AF870
:107D1000002806D12000F5F780F803000120002B91
:107D200002D02000FFF7C2FF10BDF8B50600080022
:107D30000C00F4F7E1FE07003000F4F7B5FF002572
:107D4000874207D12000F4F762FF01003000F4F70A
:107D50004FFF01353000F4F7EBFE874207D12000DA
:107D6000F4F74FFF01003000F4F7D6FE01252000A4
:107D7000F4F747FF00280DD0F4F7B0FE050020000F
:107D8000F4F745FF01002800F4F717FF2800F5F786
:107D9000F7FA01252000F4F73AFF00280DD0F4F798
:107DA0009DFE05002000F4F72CFF01002800F4F7E9
:107DB000FBFE2800F5F7E4FA012500212000F4F786
:107DC000F3FE00212000F4F7F8FE002D02D0237A04
:107DD000013B2372F8BD70B504002000F4F764FF86
:107DE00000280AD0F4F77AFE050001002000FFF712
:107DF0009CFF2800F5F7C4FAEFE770BDF8B50B7AE1
:107E0000050001330B720C00F4F7F1FF00280CD0D1
:107E10002000F5F7CAF9002807D023682A1E00D0F1
:107E20002A68934201DB01332B602800F4F780FEBF
:107E300000287DD0F4F752FE06002800F4F7D7FFA3
:107E4000002823D0002E56D02000F5F7AEF90028E8
:107E50001ED03000F5F7A9F900280DD13000F4F755
:107E6000D0FE07003000F5F78BFA002F43D0380022
:107E7000F4F734FE0600E5E7200003F0AFFC07004E
:107E8000300003F0ABFC3F1AE8D401E0002E32D002
:107E90003000F4F7BCFE002814D0F4F71FFE0500F4
:107EA0002000F4F729FE01002800F4F77DFE2800E9
:107EB000F4F722FE01002000F4F77FFE2800F5F71A
:107EC0005FFA06E02000F4F717FE01002800F4F73F
:107ED00023FE2000F4F710FE01003000F4F76DFEE1
:107EE0003000F4F709FE01002000F4F75DFE3000D9
:107EF000F5F746FA28E02800F4F7D6FEF4F7EEFD91
:107F000007002000F4F7F8FD010006003800F4F740
:107F10004BFE3800F5F734FA2800F4F7C5FE0100EF
:107F20002000F4F74AFE31002800F4F761FE0BE070
:107F30002000F4F7E1FD040001002800F4F758FEEA
:107F400021002800F4F7E8FDF8BD70B50C0005002D
:107F50001000F5F7B9FF210003F04EFD041E03D019
:107F600001002800FFF74AFF200070BD70B5040033
:107F7000051E46D0F4F70FFF002803D02000FFF7BE
:107F800077FE3DE02000F4F7A3FE002805D0200096
:107F9000F4F792FE03F0D0F832E03F23628920002C
:107FA00013400F2B07D1F4F77FFE431E9841C0B258
:107FB00003F0B9F824E0F4F7ABFE00281AD0200053
:107FC000F4F772FE00280FD1267A0500002E18D192
:107FD0002000F4F7ADFE3500002812D122000A4936
:107FE000053005F01BF90CE0F4F778FD050084423C
:107FF00007D100E020008022438992009B18438132
:108000000500280070BDC046E6A1030070B5051E3E
:1080100001D100204EE0F4F7BEFE002803D0280076
:10802000FFF726FE46E02800F4F752FE002805D0B0
:108030002800F4F741FE03F07FF83BE03F236A8914
:108040002C0013400F2B2DD02000F4F761FE0028E8
:108050001FD02000F4F728FE0600A54202D0200021
:10806000F5F78EF9002E0FD1A542D2D12B7A002B35
:10807000CFD12800F4F75CFE0028CAD12A000E49AF
:10808000053005F0CBF8C4E73000F4F727FD040015
:10809000DAE72000A5420DD18022638992009B1867
:1080A000638107E02800F4F7FFFD431E9841C0B24A
:1080B00003F039F870BDC046E6A1030070B50400B6
:1080C000FFF7A4FF05002000F5F75AF9280070BD5E
:1080D00037B504000320F4F7A2FD051E21D02100CE
:1080E00001A8F5F7BBF9019C002C17D08022638909
:1080F00092009B1863812000F5F72FF8002806D026
:108100002000FFF733FF01002800FAF711FA2000E2
:10811000F5F736F901A8F5F78DF9E4E701A802F0C3
:10812000D9FD28003EBD30B5040091B0002804D12F
:10813000002200231000190040E0F5F72BF800287A
:1081400001D003CC52E02000F5F74AF8051E03D019
:1081500020680FF009FC49E02000F4F748FE0028F1
:108160000DD02068002840D0012808D12900200027
:10817000FAF721FAFFF7A2FFF5F787F936E02000BA
:10818000F4F7A2FF0028D3D040226946200003F074
:10819000A7FA402804D116493F3805F03FF8C7E751
:1081A0006B461878002820D0124968460FF079FDF8
:1081B000002806D10022002300200F490EF08CF980
:1081C00014E00E4968460FF06CFD002809D1002329
:1081D0000022002008490EF07FF980231B06C918F1
:1081E00004E068460CF0E0FD00E0010011B030BD95
:1081F000F8A103001DA203000000F03F1CA2030031
:1082000010B590B00400F4F7D0FF002804D120008E
:10821000F4F7C0FF002806D08022638992009B18E3
:108220006381200046E02000F4F7A5FF00280ED16E
:108230002000F4F7CAFF002809D12000F4F78DFDD3
:10824000002804D12000F4F7A6FD002805D0200066
:1082500003F0C4FA02F070FF2CE02000F4F734FFC2
:10826000002822D0200003F0B8FB011E11D04022CC
:108270006946200003F034FA402810D10E4901204D
:1082800004F0CCFF00220023100019000EF024F9A6
:108290000EE0200002F075FF0028E8D105E06846F6
:1082A00005F046FA02F05DFF04E02000FFF73BFF17
:1082B00002F02EFF10B010BD26A2030070B588B0EA
:1082C00006000C001500F4F70FFF002836D000223E
:1082D000310003A80AF08EF8039B0093049B0193DE
:1082E000019A009B934211D22678002E22D003A837
:1082F00008F036FFB04204D00698F5F741F80020A8
:108300001CE003A801340AF035F9E5E7002D07D198
:1083100003A808F025FF2378181A4342584103E0C8
:108320002378002BF4D1012004000698F5F728F8F3
:10833000200003E00120002DF6D1E9E708B070BD70
:1083400010B50022FFF7BAFF10BDF0B585B001925D
:108350000A7803AB07000E001A70002A09D04A7889
:108360005A70002A06D08A789A70002A03D0CA78F8
:1083700001E05A709A703800DA70F4F795FC051E27
:1083800018D00C23013D5D43144C039B2C1922682B
:1083900093420BD131002000FFF7D2FF002805D017
:1083A0008022638992009B18638114E02000F4F717
:1083B0002EFCE4E7019C002C0DD03000F5F784FD85
:1083C000290003F019FB2C00061E04D00100380020
:1083D000FFF714FD3400200005B0F0BDBC260020DE
:1083E00070B500220500FFF7B0FF041E06D00100A3
:1083F0002800FFF79AFC2000F4F7C2FF70BD70B5AB
:1084000004000D00F4F774FC002817D02000F4F7E6
:108410005BFE6689002807D02000F9F7B9FA3F23F0
:1084200015309E43064303E03F239E43323B1E43E9
:10843000668100212000F4F7DBFB06E02000F4F762
:1084400033FC002801D0F4F7ADFF291E4ED02000E8
:10845000F4F7ABFE002821D02800F4F7A6FE061E94
:1084600004D12800F4F787FE002838D02800F4F75C
:10847000ACFE002833D1802329689B00CA181E4B0C
:108480009A422CD83F23608989B298430300701E1A
:1084900086410F20801B1843608127E02000F4F7FD
:1084A00013FE00281BD02800F4F77FFE002816D00A
:1084B0002800F4F78AFE002811D180232E689B0043
:1084C000F2180D4B9A420AD82000F9F761FA3F22C0
:1084D00063891030934318436081B1B206E02B7A70
:1084E000280001332B72F4F707FB01002000F4F79A
:1084F0007FFB200070BDC046FF03000070B5150073
:108500000122FFF722FF041E06D02900FFF777FFA4
:108510002000F4F735FF280070BD10B5FFF7EEFF1F
:10852000F4F72EFF10BD70B503001600002819D017
:10853000531E9A41D2B2FFF708FF0500FFF766FD10
:10854000041E0BD1002E09D0002D07D03000F4F707
:1085500066FB040001002800FFF751FF2800F4F734
:108560000FFF2300180070BD10B50C001100012290
:10857000FFF7EBFE002802D02100FFF740FF10BDFF
:10858000F7B50191050017004489002A1DD13F2647
:10859000230033400D3B022B03D80820B44304438F
:1085A00013E0F4F7C5FA002808D0274A390028005C
:1085B00002F030FF041E18D1002443E02800F9F730
:1085C000E7F9B4431A300443A4B27F202040F4F703
:1085D00026FB041EF0D00422290020000FF04BFBE4
:1085E0002800F4F781FD002813D1019B002B29D02E
:1085F0002800F4F759FB051E24D0F4F76FFA037A2C
:1086000001330372F4F7BCFE29002000F4F7F0FAFE
:1086100018E02800F4F78CFA0028E6D0F4F75EFAA8
:10862000070000F013F8061E08D0F4F765FA010001
:108630002000F4F771FA3000F4F7A2FE3800F4F7E6
:108640009FFED2E72000FEBDFFFFFF7FF8B50400CC
:10865000F4F700FC002806D0434A0021200002F075
:10866000D9FE03007EE07F2360891840F4F7D7FA33
:108670000500031E76D02000F4F716FD092200281D
:1086800007D13F236289134007221A3B934200D946
:10869000033A210028000FF0EEFA2000F4F738FB2F
:1086A00000281AD02000F4F7FFFA002815D0F4F7BC
:1086B00015FA0700FFF7CAFF0600037A01330372B9
:1086C0003800F4F75DFE3000F4F716FA01002800D8
:1086D000F4F78EFA3000F4F753FE2000F4F704FDAF
:1086E000002819D02000F4F723FA2B00002839D0F5
:1086F000F4F7F4F90600FFF7A9FF041E08D0F4F719
:10870000FBF901002800F4F707FA2000F4F738FE1F
:108710003000F4F735FE24E02000F4F784FD2B0050
:1087200000281FD02000F4F7BFFA0400002C18D056
:108730002000F4F7D3F9012211000600FFF720FF13
:10874000041E06D001002800FFF758FB2000F4F7B4
:1087500017FE3000F4F75BFA04003000F4F710FE67
:10876000E4E72B001800F8BDFFFFFF7F10B5037A88
:108770000400002B0ED1F4F7CBFA011E03D1200028
:1087800003F03AF904008022638992009B18638108
:10879000200004E0FFF75AFF002103F02DF910BD7F
:1087A000F0B58FB001900E000292F4F77DFA05004B
:1087B000002D00D185E02800F4F790F9041EB442A2
:1087C00000D18BE0002807D12000F4F720FA050043
:1087D0002000F4F7D5FDEBE7002EF5D0F4F72AFBE7
:1087E000002837D03000F4F725FB002832D02000D5
:1087F000F4F7F6FC002812D03000F4F7F1FC002862
:1088000006D0236832689D1A6A426A41D5B255E0A3
:1088100020680FF0A9F801253268736813E0300072
:10882000F4F7DEFC636827680393002806D03068FD
:108830000FF09AF8012502000B0002E001253268D2
:108840007368380003990DF081FA002800D1051CE7
:10885000EDB233E02000F4F737FC0028B4D030004C
:10886000F4F732FC051EAFD00022210004A809F065
:10887000C1FD0022310009A809F0BCFD04A808F0E0
:108880006FFC070009A808F06BFC874206D0079828
:10889000F4F776FD0C98F4F773FD95E7002F06D1F9
:1088A0000798F4F76DFD0C98F4F76AFD06E004A84C
:1088B00009F060FE09A809F05DFEDFE7002D83D016
:1088C0000EE0029800280CD0301E0AD0FFF74EFFB1
:1088D000040001000198FFF791FA01E0300000E088
:1088E00020000FB0F0BD70B5050008001600FFF7BE
:1088F0003DFF0400002E02D03100FFF780FD2B7AEF
:10890000280002332B72F4F7F7F80500010020006D
:10891000F4F753F929002000F4F746F9200070BD60
:10892000704700DF704713DF704711DF704744DF87
:108930007047F0B5060097B008000D001700F4F777
:10894000C3FB00280FD12800F4F751FA00280AD100
:108950002800F4F72BFA002805D12A00224901301B
:1089600004F05CFC3DE029000BA801AC09F0D0FD4F
:1089700031003A00200009F08AFD237D01269B0684
:1089800018D52800F4F7A0FB060013E0200009F03A
:10899000A5FC00281FD00BA8002E11D009F041FF24
:1089A0000100200009F076FE200009F012FE0BA85D
:1089B00009F028FE0BA809F0A3FC0028E6D10AE084
:1089C00009F057FF05000100200009F02FFE2800E4
:1089D000F4F7D6FCE8E7200009F064FC0BA809F0E6
:1089E00069FC17B0F0BDC0465CA20300114B70B526
:1089F000041E9C4205D901200F4904F00FFC002001
:108A000016E0102807DC200003F0DCF80500002049
:108A100085420DD003E0F4F728FA051EF3D02100BB
:108A2000280002F0BDFF04002800F4F7A9FC200094
:108A300070BDC046FFFF00008CA20300F0B58FB0F0
:108A400001900F001500FFF746F906000400002D05
:108A500003D0280002F0C2FE04000320F4F7DFF880
:108A6000009000283ED0002F04DAF519EB43DB1705
:108A70001D4003E0351EBD4200DD3D00002C04DA40
:108A8000A419E343DB171C4002E0B44200DD3400CC
:108A9000019903A809F03CFD002603A809F030FC69
:108AA00000281CD0002E1AD103A809F0DFFBF4F730
:108AB000F8FC854203DD03A809F0A4FDEDE7A5421B
:108AC0000BDA03A809F0D5FE01000098F9F730FD94
:108AD00003A809F097FD0135DFE70126DDE703A8CC
:108AE00009F0E8FB00980FB0F0BDF0B599B0059320
:108AF0001EAB1B78050002931FAB1B78080009937F
:108B000020AB1B78049108920693F4F7FBFA041E3D
:108B100002D12A004E4906E00898F4F77EF9041EB7
:108B200006D12A004B49012004F078FB20008DE09B
:108B3000059B002B07D01800F4F764F9041E02D13E
:108B40002A004549EFE70024029BA34206D00320F8
:108B5000F4F765F804000020844277D004990DA84A
:108B600009F0D6FC00270DA809F0CAFB002858D050
:108B7000002F56D10DA809F079FB0390F4F715FBEF
:108B8000002847D0039802F029FE07900DA809F0AD
:108B900070FE0A90079802F0CFFA049B0AAEB36009
:108BA000032370603900009301963B00059A0898F2
:108BB000FEF78AFA310005000220F4F7FDFB002DD4
:108BC00028D0099B002B10D0280002F076FC029BD5
:108BD000002B35D0069B984219D10DA809F049FE0B
:108BE00001002000F9F7A4FC11E0029B002B0ED03D
:108BF000079802F0A1FA061E09D0290002F0FCFE37
:108C000020003100FFF7FAF83000F4F7B9FB280034
:108C1000F4F7B6FB0398F4F7B3FB0DA809F0F2FCE8
:108C2000A1E70DA809F046FB029B2000002B0DD107
:108C3000099B002B0AD00698784002F074FA05E0F0
:108C4000069BC01A431E9841C7B2E0E719B0F0BDB9
:108C5000ACA20300DEA203000DA303001FB51300A6
:108C6000012400220294009201940A0001000248AB
:108C7000FFF73BFF04B010BD4AA303001FB513006C
:108C8000002401220294019200940A00010002488B
:108C9000FFF72BFF04B010BD50A303001FB5012444
:108CA000130002940A000194010000940248FFF7A7
:108CB0001CFF04B010BDC04655A303001FB500241F
:108CC000130002940A000194010000940148FFF788
:108CD0000CFF1FBD5CA303001FB51300002401227D
:108CE0000294009201940A0001000248FFF7FDFE81
:108CF00004B010BD64A3030070B504000D00F4F7C8
:108D000001FA002801D1002014E0002D03D10A4807
:108D1000F5F7DAF803E00021280002F02DFC051E2B
:108D2000F1D001002000F9F713FD04002800F4F74A
:108D300027FB200070BDC04668A3030070B5002269
:108D4000F9F700FC051E04D10120404202F0F4F9BD
:108D500008E000221100FFF713FC04002800F4F7DC
:108D60000FFB200070BDF8B5041E35D00368012B41
:108D700032D10021F9F71FFCFFF7A0F90500F4F745
:108D800059F8002825D02800FFF7CDF90600280063
:108D90000F0002F023FD04002800F4F7F1FA200090
:108DA0000EF0E2FD02000B00300039000CF0CEFFA7
:108DB000002801D0002C05DA01200B4904F02EFA1E
:108DC00000200FE00320F3F72AFF00280AD00460F8
:108DD00008E02800F4F7D4FA80222000638992008A
:108DE0009B186381F8BDC0466AA30300F0B51D005F
:108DF000424B93B01B68019000911700002B7BD071
:108E0000189B602B78D8FF22002403AB5A709A700D
:108E1000DA701C70189B06AE34700B950A93A0B2E2
:108E200004A90BF041FF002809D1082204A90198E8
:108E30000EF012FF002802D103AB9C7002E0013457
:108E4000072CECD103ACA178FF2955D0009B032B54
:108E50000AD1189A06AB602A01D1403A00E04022BC
:108E60001A701A78032139E0254BEB1AC32B10D85E
:108E7000244B002F04D101228A40186810423BD0B5
:108E800001228A40196891432022196006AB1A70AA
:108E90001EE01D4BEB1A1B2B08D820233370002338
:108EA00063700CAB0B9318230A9311E017482D1A2B
:108EB000232D21D830233370002363700133E370F6
:108EC000134B997A0223194002D12422F2F770F948
:108ED000009A06AB022A0CD101211A780A431A70B3
:108EE00009AB7360054B3A001B68310020009847BE
:108EF00002E01A780221F1E713B0F0BDB42500209A
:108F0000D4250020A02400203C2500209826002005
:108F1000C025002010B50AF0D9FC10BDF0B589B00D
:108F200000900F0015001C00F3F761FF002800D12E
:108F3000F4E0009B0193002B01D01B680193002FEC
:108F400004DA019BFF18FB43DB171F40019B9F4284
:108F500000DD1F002800F4F728F9031E019802D055
:108F6000280002F03BFC019B0290DB1B984200DDD5
:108F70000293231E00D02368029A03209B1A0593B4
:108F8000F3F74DFE0099049007A801F0CCFE0023F2
:108F90000393079B07A8002B3BD0039B002B38D1E2
:108FA00001F0B8FE051E01D1012629E0F4F7FDF815
:108FB0000028F9D0280002F011FCB842F4DB029B33
:108FC000DB19984219DA049B002B06D007A801F0A0
:108FD0009AFE01000498F9F7ABFA07A801F09AFE8F
:108FE000060007A801F07BFE31000098FEF79DFE09
:108FF0003000F4F7C5F9002602E00123039E039335
:109000002800F4F7BDF9002EC3D007A801F067FED1
:10901000BFE701F07FFE2100050006A801F083FEF6
:10902000069B06A8002B52D001F06DFE0290002D89
:1090300042D0002002F080F8029902F0DDFC041E0C
:109040003ED0037A01330372F3F756FD03902800F4
:10905000F3F7D7FD071E15D0F3F740FD037A06009E
:109060000133037202F0BAFB013003992060300033
:10907000F3F7A3FD3000F4F783F939002000F3F78C
:1090800093FD07E001002000F3F78EFD039900989F
:10909000F3F7AEFD03992800F3F786FD2B7A28003D
:1090A00001332B72F3F728FD01002000F3F785FD53
:1090B0002000F4F765F903E002990098F9F719FA2E
:1090C0000298F4F75DF906A801F009FEA8E701F09F
:1090D00001FE2800F4F754F9079B07A8002B14D0D1
:1090E00001F018FE041E09D0F4F75FF8002805D03F
:1090F000200002F073FB059B181820602000F4F795
:109100003FF907A801F0EBFDE6E701F0E3FD019A66
:10911000059B9446009A63440498136009B0F0BD1F
:1091200073B505000C00F3F762FE002820D0210083
:1091300001A8012401F0F7FD6442019B01A8002B66
:109140000ED001F0E0FD010006002800F9F7D1F98A
:1091500004003000F4F714F901A801F0C0FDECE7B9
:1091600001F0B8FD201E05DA281E03D0286801E0B2
:109170000120404276BDF0B59BB0019008000C0084
:1091800003921F00F3F712FE051E0BD02379812BEB
:1091900008D18022638992009B18638100232600F6
:1091A000029330E02000F3F745FE00280CD02000A9
:1091B00002F014FB07000F20019B18407843FFF7D3
:1091C00015FC0023060019E02000F3F710FE00282C
:1091D00008D1002D06D101202200374904F01EF8E5
:1091E000002067E02000FEF776FD07000F20019BBE
:1091F00018407843FFF7FAFB012306000293002E84
:10920000E9D000230393002F06D10F21019B708822
:1092100019400CF009FC07000420F3F700FD051EBF
:1092200044D06B461B79478003716B469B89038052
:10923000337A300001333372F3F75EFC010028000B
:10924000F3F7D6FC029B002B30D021000FA809F0C9
:109250005FF90FA809F054F8002824D00FA809F0EE
:1092600005F80400F3F7A1FF002815D00FA809F0B6
:1092700000FB0700200002F0B1FA2900020005A857
:1092800009F005F9390005A809F0D0F905A809F099
:1092900009F83800F4F774F82000F4F771F80FA813
:1092A00009F0B0F9D5E70FA809F004F83000F4F799
:1092B00067F828001BB0F0BD7FA30300AADF70474A
:1092C00063DF7047A8DF7047A6DF7047F0B5050081
:1092D00087B014000E20002D20D02A88104B0638AD
:1092E0009A421BD00F4B1A79002A17D010225E1D0C
:1092F00099715A716B469F1D0323B47002AC002113
:1093000020003B80F1F754FF2B8A2888238001231B
:109310002100A370A760E660FFF7D6FF07B0F0BD9D
:10932000FFFF0000A0240020F0B50B788DB0002BCB
:1093300000D0DEE0774C02AB9A1C210008230588A0
:1093400013804031073B2800FFF7B8FF724B1B68C2
:109350009847B120FFF7EBFA002801D008F0E4FDB0
:10936000FFF7E3FA002801D008F0DEFD6B4E7069CC
:10937000FFF7D9FA0196002801D008F0D5FD2600A4
:1093800048363278002A00D085E0654B1B68002BF8
:1093900000D180E0FF23B370624B1989A9427AD1D2
:1093A0007270D87A604BB0701B78002B43D00628BF
:1093B00041D81C2545435D4B5D19AB7EFF2B3AD050
:1093C00080B203A90BF070FC00280DD11C2303A967
:1093D0001A0005A806F092FA002805D11C23B578DA
:1093E0005D43524BED1801E0002824D126002900EE
:1093F0000C361031072230000EF03DFC2000102208
:10940000290013300EF037FC2000112205A924306A
:109410000EF031FC20001E2102AB36300A22C918A2
:109420000EF029FC3000FFF77CFA002801D008F08C
:109430007BFD3F482DE03C4B1B78002B62D035482C
:10944000030048331A78002A5CD1354A1268002A92
:1094500058D09978FF290AD15978FF2954D00C2384
:109460005943304B59188B7A9B074DD507E01C2385
:1094700059432E4B59188B7E9B0745D410310C3025
:1094800007220EF0F8FB20000C30FFF74AFA002804
:1094900001D008F049FD8021C022264BC9035200AB
:1094A0009950196801200023234C02009A40114270
:1094B00000D0E2670133202BF7D1019B5B6918686C
:1094C00080F308885868FF2464B2EFF30585002D07
:1094D00001D1A6460047251C061C21273FBAF0B43F
:1094E0000024002500260027F0B4F92040B20047F0
:1094F0000EE003220121FFF7E9FE002808D008F062
:1095000013FD05E00D4800E00D4808F00DFDBAE739
:109510000DB0F0BDA02400206C1F00200010001032
:10952000B4250020C0250020B0250020D42500202F
:109530009180000000E100E004E100E0088000000C
:1095400005800000A5DF7047A2DF7047A0DF7047ED
:1095500013B50400694680780BF0A6FB002810D1F3
:109560001C226078074B50436946C018130006F070
:10957000C5F9054B054A9B7A21009B009B5868461C
:10958000984713BD3C250020B42500204CA20300C1
:1095900010B50022084B0DF0C3FB0022074B0DF065
:1095A000BFFB054B00220CF097FF0CF01BFC044B9B
:1095B0001860596010BDC04600408F400000E04078
:1095C000F0240020044B01211A89002801D08A438D
:1095D00000E00A431A817047F0240020044B042164
:1095E0001A89002801D00A4300E08A431A81704793
:1095F000F0240020F8B506000D00F7F7DBFC00288A
:1096000002D1304901304CE02800F3F75DFD7409C8
:109610002D4F002838D02D492800FEF791FE062155
:10962000002841D12A492800FEF78AFE032100289C
:109630003AD128492800FEF783FE0421002833D1BF
:1096400025492800FEF77CFE052100282CD123495E
:109650002800FEF775FE0121002825D120492800A9
:10966000FEF76EFE022100281ED11E492800FEF7DB
:1096700067FE0721002817D11B492800FEF760FE6E
:10968000002801D008210FE01F2301201E40030005
:10969000B340A4003F19FA689A43FA60002D10D035
:1096A000124903F0BBFD0CE01F220123324093401E
:1096B000A4003F19FA6830009A431343FB600AF094
:1096C000EBFFF8BDA6A30300F0240020B2A3030023
:1096D000B9A30300BFA30300CCA30300DEA30300D0
:1096E000E8A30300DBA30300E5A30300F2A3030048
:1096F00070B50A4C2578F7F73AFC207085420BD0FC
:10970000FF2D03D000212800F7F760FC2078FF2808
:1097100002D00121F7F75AFC70BDC046701F00202F
:1097200070B50A4C6578F7F722FC607085420BD063
:10973000FF2D03D000212800F7F748FC6078FF28B0
:1097400002D00121F7F742FC70BDC046701F002017
:10975000F8B505000C00F3F74AFB00281FD02800DD
:10976000F3F7E6F901270500002D20D02800F3F7D4
:10977000B5F90600FEF74AFC0500F7F7F8FB2100F3
:109780003940F7F723FC2800F3F7FAFD3000F3F730
:1097900038FA05003000F3F7F3FD6410E4E7611ECA
:1097A0008C412800F7F7E3FBE1B2F7F70FFCF8BDB7
:1097B000F0B585B005000A9802920393F3F722FBF7
:1097C000002818D0002226490A98FEF7ACFEF3F7CD
:1097D0005CFE002206000F000A982249FEF7A3FE55
:1097E000F3F749FE021E08D11F490A98FEF79BFEB7
:1097F000F3F741FE01E0002600272800F7F724FBDD
:109800006C0900280ED10121184AA300D3181F2289
:1098100008002A409040020018699043186128000F
:109820000AF03AFF1F2201232A4093400F4AA40066
:109830001419226930009A43134323610022002344
:1098400039000CF093FA002801D00026084F00954B
:10985000029A039B3000390009F0E8FB05B0F0BD27
:1098600003A4030008A4030012A40300F0240020B2
:1098700000004940F7B52C4C0500A08A16001F00D7
:10988000F3F72CF9294A0190294B300039000CF0EC
:1098900063FA002801D0254E254F2800F3F74FFC2E
:1098A000002838D0002229000198FEF779FF00280F
:1098B00031D0FEF703FC002200901E4B390030002F
:1098C0000DF02EFA1C4B00220CF006FE0CF08AFA6A
:1098D000050001F031FC0700184A01000098FEF76E
:1098E00043FE3900F3F780FD154A164BD058236824
:1098F000C01A401901F020FC05000100124A00982E
:10990000FEF732FE009A2900F3F762FD0822238950
:109910001343238103E00D49012003F07FFC0198EC
:10992000F3F72EFDF7BDC046F02400209A999999CF
:109930009999B93F0000E04000408F40787E0300D5
:1099400000B0004004050000287E030017A40300B7
:10995000F0B585B01F000AAB20CB02901B78160033
:109960000393F3F75AFA00280AD10298F3F7ACFBF5
:10997000041E05D13049012003F050FC250058E0B9
:109980000520F3F74CF92D4A04002D4B3000390027
:109990000CF0E2F9002801D0284E294F0022294B73
:1099A000390030000DF0BCF90022274B0CF094FD7B
:1099B0000CF018FA00900191244A254B0021D3584D
:1099C000244F18003A687B68801A9941009A019BDD
:1099D0008018594101F0C5FB1F4902002000FEF725
:1099E0009CFD039B002B08D10098019901F0B9FB65
:1099F0001A4902002000FEF790FD029A1849200043
:109A0000FEF77CFD002D07D02B68002B04D02A0028
:109A100014492000FEF772FD2000F4F755FB01F019
:109A20008BFB05002000F3F7ABFC08223B891343B6
:109A30003B81280005B0F0BD28A403009A999999AC
:109A40009999B93F0000E04000408F4000B00040CD
:109A500004050000F0240020287E0300787E030027
:109A6000337E0300817E030007B501210191049933
:109A70000091FFF76DFF0EBD07B50021019104991C
:109A80000091FFF765FF0EBD00B593B0422201A91A
:109A900001F026FE422808D11549413803F0BEFBEB
:109AA000002200231000190009E0124901A80EF05D
:109AB000F8F8002806D10022002300200E490CF0FF
:109AC0000BFD12E00D4901A80EF0EBF8002809D1BA
:109AD00000230022002008490CF0FEFC80231B0616
:109AE000C91802E001A80BF05FF913B000BDC04631
:109AF000F8A103001DA203000000F03F1CA2030018
:109B000070B5060092B008000C000025F3F792F93A
:109B1000A84203D0200001F061FE05003000F3F7F9
:109B200039FB002806D03000FEF7FDFAF5F720FFDC
:109B300000280BD001AC42222100300001F0D0FD02
:109B400042280CD11349413803F068FB002200235E
:109B5000100019000CF0C0FC01F0DAFA17E06B46B7
:109B6000DE1C002333709D4207D12378302B04D1B3
:109B70006378303B092B00D80A25320029002000E9
:109B800003F078FD3378002BE0D101F0EAFA12B04F
:109B900070BDC04626A2030070B5031E0DD0002183
:109BA00001F0EAFC064B0022196B0500F7F78CFA6E
:109BB00004002800F3F7E4FB2300180070BDC04642
:109BC0008C5A002070B500250B4AD36AAB4203DDE6
:109BD00001339B00D3185D682800F3F71EF9041EBB
:109BE00005D10120054903F019FB200002E02800FF
:109BF000FEF76EFA70BDC0468C5A002049A40300DF
:109C00008023F0B55B051A6E8BB000925B6E02AEDE
:109C1000019300236A46D25C9A550133202BF9D177
:109C200007F0A5FA051E1AD0002403273C4205D1EF
:109C3000002C03D00B49280001F0BCF98023305DD3
:109C40005B0018430122F03B694603F08BF86B463A
:109C50002800591C013401F0ADF9202CE6D1280070
:109C60000BB0F0BD7DA40300F7B50400F3F72CFAA8
:109C70003B4F031E0ED08022638992009B186381A4
:109C8000210000223868FEF78BFDFEF717FA260048
:109C9000040005E0022221003868F8F72FFB0600D7
:109CA0003000F3F711FA002851D02000F3F7B5F88F
:109CB00000284AD000222B492000FEF746FB012253
:109CC000050021003868F8F73DFC002301939D4210
:109CD00003D10200531E9A4101922900F3F784FB3D
:109CE00007F045FA051E36D00021200001F044FCA3
:109CF000019B0700002B0ED028001B4901F05AF9E8
:109D00003100280001F0D1FA184B0922390028004F
:109D100001F09BFA0FE03100280001F0C6FA144967
:109D2000280001F047F93900280001F0BEFA114976
:109D3000280001F03FF93800F3F722FB2800F4F780
:109D4000BDFA2800F3F71CFB05E00B4900E00B49C6
:109D5000012003F063FA31002000F3F745FBF7BD63
:109D60008C5A0020CAA103007FA40300FFFFFF7FDD
:109D700089A40300C388030097A40300C9A40300B7
:109D800070B504008CB008000E001500F3F752F80F
:109D900000280ED0300001F021FD012D01D12070EE
:109DA0002BE0022D01D1208027E0042D25D1206059
:109DB00023E03000F3F7A6F900281ED0310001A8F7
:109DC00008F0A6FB01A808F09BFA002812D001A811
:109DD00008F027FD012D01D1207006E0022D01D1F0
:109DE000208002E0042D00D1206001A8641908F051
:109DF00009FCE7E701A808F05DFA0CB070BD70B58A
:109E000004008AB01500012912DC012A01D1007872
:109E10000AE0022A04D1407823780002184303E0C4
:109E20000020042A00D12068002101F09AF92FE0D7
:109E3000101E022803D00420824200D00338F8F715
:109E4000D0F8061E24D001000022684608F01FFB4F
:109E5000684608F043FA002816D0012D01D1217878
:109E60000AE0022D04D1617823780902194303E046
:109E70000021042D00D12168684608F00BFC6846DB
:109E8000641908F0A6FBE3E7684608F00BFA300017
:109E90000AB070BDF8B5056804000F00002D11D0A0
:109EA0002800F2F7B4FE290006003800FDF73DFF58
:109EB0002068F3F765FA0020864202D03000F2F7FE
:109EC0000DFE2060F8BD73B50400F2F790FF002886
:109ED00021D00025210001A800F025FF2E00019CC3
:109EE00001A8002C10D000F00EFF0400F7F73FF897
:109EF000F7F7A2F86D0005432000F3F741FA01A837
:109F000000F0EDFE0136EAE700F0E4FE2000002E4E
:109F100006D0280004E02000F7F729F8F7F78CF8BE
:109F200076BDF7B5284C0600A08A0F00F2F7D6FDE3
:109F30000500002E20D1010001A800F0F4FE019BD5
:109F400001A8002B15D000F0DEFE00221F490700FB
:109F5000FEF7E9FA061E04D1290001A8FFF79AFFCF
:109F600002E001A800F0BBFE39003000F3F73CFA34
:109F7000E5E700F0AFFE1EE03000F3F7E0F8002860
:109F800012D0310000222800FEF70AFC061E0BD07A
:109F9000A08AF2F7A3FD07003100FDF7C6FE3900E5
:109FA0003000F3F721FA06E00949002F00D10949F2
:109FB000012003F033F92800F3F7E2F9082223899E
:109FC00013432381F7BDC046F02400202D7E0300FB
:109FD00007A5030017A4030010B50121FFF7A1FF97
:109FE00010BD10B50021FFF79CFF10BD13B5040094
:109FF000F6F7B2FE210001A800F095FE019B01A832
:10A00000002B1ED000F07FFE0400F3F75DF8031E66
:10A0100005D0002220001100F7F704FC04E00C4AF0
:10A020000321200004F0D8FD2000F3F7A9F901A8CE
:10A0300000F055FE019B002BE0D00648F6F760FDCE
:10A04000DCE700F047FE0448F6F75AFD13BDC046B2
:10A05000010B020076830300A87F0300F7B505001B
:10A060000620F2F7DCFD041E33D0290001A800F021
:10A070005AFE01A800F047FE050001A800F02FFEDF
:10A08000019B002B1DD00021280001F075FA071E4E
:10A0900013D0114A002101F0BDF906003800F3F792
:10A0A0006FF9002E09D0300001F07EFD2000310054
:10A0B000FDF7A4FE3000F3F763F92800F3F760F929
:10A0C000D7E701A800F006FE2A0004492000FEF7A9
:10A0D00024FA2000FEBDC046FFFFFF7FCFA1030092
:10A0E000F0B58FB0019010000F001400F2F7A2FE3F
:10A0F00000281ED02000FEF716F8002200230400DE
:10A100000D000BF029FE002807D122002B002000B3
:10A1100029000DF0D3FB002804D03249012003F0C0
:10A120007DF85CE022002B00390001980AF0EEF97E
:10A1300055E02000F2F7E6FF00284BD003AE2100E7
:10A14000300008F0E5F9300008F0DAF800283DD0DA
:10A150003378012B04D0002B08D0022B0CD014E054
:10A1600004A800F0D0FDF3F790F90BE004A806F086
:10A17000F7FF0DF03BFC05E0337E002B18D004A860
:10A1800008F0E7FA04000D0001E000240025002299
:10A190000023200029000BF0FDFD002810D0220034
:10A1A0002B00200029000DF089FB002802D007E0D9
:10A1B0000024002522002B00390001980AF0A6F99E
:10A1C000012330005F4008F01DFABCE7300008F0C2
:10A1D00071F804E022000449012003F01FF80FB0D9
:10A1E000F0BDC04617A5030059A5030070B50400D3
:10A1F00088B0002801D1012049E0F2F703FE051ED6
:10A20000F9D12000F2F7C6FF00280FD12000F2F7A5
:10A21000EEFD00280AD12000F2F756FF002836D0C4
:10A220000022210003A808F0E5F813E02000FDF764
:10A230007AFF02000B000DF041FB0028EBD0DAE7BB
:10A2400003A806F08DFF07F0E1F800280CD003A862
:10A2500008F090F9039B0093049B0193019A009BE3
:10A260009342EDD3012600E006000698F3F788F844
:10A27000002E0BD12000FDF756FF02000B00012538
:10A280000DF01CFB002800D1351CEDB2280008B0F1
:10A2900070BDC04670B50C000500002300222800E8
:10A2A00021000BF059FD80231B06E318002800D184
:10A2B00023002800190070BD10B507F035FE10BD51
:10A2C00070B50D0016000C00631B9E4205D9217865
:10A2D000152009F0D5F80134F6E770BD70B50022FD
:10A2E000002304000D000BF055FD00280AD02000CB
:10A2F0002900F5F705F80022064B0CF011FDFBF7DD
:10A3000035FA05E000220023100019000CF0E4F8F3
:10A3100070BDC0460000E03FF8B505000C00F5F741
:10A3200027FB002805D0002D06D180231B069C4268
:10A3300002D12800210021E0002200232800210072
:10A340000BF00AFD002802D11048114901E00F4826
:10A35000104923002A000BF093FD06000F000DF0BA
:10A36000CDFA041E0DD100220023300039000BF07D
:10A37000F3FC002805D080210020090600F0C8FE6B
:10A3800002E0200000F0D8FEF8BDC0462083E4FFC4
:10A39000FFFFDF3FFFFFDFBFF0B5214B214E1B88E2
:10A3A00087B0B34205D000201F4D2C78844235D1B0
:10A3B00009E0152009F0D0F80028FADAF3E70134B3
:10A3C0002855142C06D0152009F0C6F80028F6DA16
:10A3D000002C20D06B46DC80AF8DB7421BD02B0009
:10A3E0002E331B78002B16D002AE00211022300035
:10A3F000F0F7DEFEAB8C310033806B1CF3606B46F4
:10A400000633B36001233800B370FEF75DFF002808
:10A4100001D101232B70E017001BC00F07B0F0BD66
:10A42000741F0020FFFF000008250020A9DF7047EF
:10A4300087DF704786DF70477CDF70477ADF7047C1
:10A4400076DF704710B50378002B08D1044B3B2111
:10A450001888FFF7F5FF002801D007F065FD10BD53
:10A46000741F002074DF704710B5104B1888104B14
:10A47000984203D01321FFF7E3FF01E0FFF7F2FF5B
:10A48000002801D007F050FD0AF032FC002801D06E
:10A4900007F04AFDFA20400007F00CFBF7F73EF901
:10A4A000F6F758FE642007F005FB10BD741F00206E
:10A4B000FFFF000073DF70477FB518220021684658
:10A4C000F0F776FEB4236A4668465382743B1382E3
:10A4D000FFF7F0FF002801D007F026FD07B000BD10
:10A4E000F0B5038893B00400A74F112B1DD002D8FC
:10A4F000102B05D041E0122B37D0502B1FD03CE061
:10A500003B0082882100380050331A8052300822E4
:10A5100016310DF0B0FB3B0000225A331A703B009D
:10A520005C33DB89934228D125E03B000122503384
:10A5300052421A803B0000225A331A700CE03A0053
:10A540005C32C188D289914224D1C38B022B21D1A4
:10A55000431CDB7FDB070ED40AF0CAFB00280CD0BB
:10A560007B6F002B09D0984707E03800A11D5230BF
:10A5700008220DF080FB09F04DFC2388112B05D03B
:10A58000502B07D0102B29D1A38801E001235B4277
:10A59000BB8523E0E388398DA21D994212D1118B2E
:10A5A00002290FD1A31CDB7F621CD27F1B02134345
:10A5B0003A0001390B402E32002B01D011700DE012
:10A5C00013700BE0B98B994208D13B6B002B05D07F
:10A5D00038002100128B1830203198473B00A033FF
:10A5E0001A68002A00D1DEE02388112B1DD006D87E
:10A5F000102B00D0D7E03800A388783019E0502B1A
:10A6000002D0512B17D0CEE038007830E188038992
:10A61000994200D059E108230CA90B70E38B0B720F
:10A62000230020334B609047BDE038000123783091
:10A630005B420380B7E0A579022D00D045E1534B82
:10A6400022891B8A9A4200D03FE1A37A043B022B65
:10A6500000D83AE128222E2102AB9B181D70063249
:10A6600002AB9B181B782D3A134302AA52181370A1
:10A67000E38B02AA1386238C09AE5386230008229B
:10A680002233002130000F93F0F792FD08AB736086
:10A690003E4B3580998A18883200FEF753FF3A4DB9
:10A6A000002806D03B00A4331B68002B0AD0984733
:10A6B00008E002AB5B7E02AA127E1B02134301225A
:10A6C00013420AD1FE2302AAFF3393852B0078336D
:10A6D00018880CA9FEF7F6FD5EE02F0000237837FE
:10A6E00002AA38880CA99385FEF7ECFD002853D107
:10A6F000E31CD97F481E07284AD80BF081F90410C3
:10A700001F212325422700233370238C012B04D8DB
:10A7100028000622783001213CE0012309E00123D2
:10A720003370228C9A4204D8280006227830022105
:10A7300030E033722300233373601BE0022318E000
:10A74000032316E0042314E0052312E0238C022BDC
:10A7500004D828000322783008211BE0631DDB7F2A
:10A76000221DD27F1B021343B38001D1073300E0C7
:10A77000062333702800A03578302B6831009847C5
:10A7800011E00923F5E7C0460825002080250020B8
:10A7900003223800FEF79AFD002804D0A4352B6868
:10A7A000002B00D098472388112B16D00ED8012BF0
:10A7B00029D0102B00D088E0A288CD4B15201A801C
:10A7C0000022CC4B1A70F6F7EBFA7EE01B2B20D060
:10A7D000522B0CD0192B78D106E00122C44B5242E7
:10A7E00016201A80F6F7DCFAFFF766FE6DE0C04B24
:10A7F000188800231A001900FFF718FE002864D0FB
:10A8000007F092FB61E00022BA4B1A70FFF7C4FD1B
:10A810005BE00520F2F703FA061E099055D00720E9
:10A82000A51D285600F088FCB34902003000FDF752
:10A8300074FEA879EB78AA78697802906879099E05
:10A84000019028790090AD4800F0F3FDAC4902007A
:10A850003000FDF762FE287AC00801F0B3F9061E49
:10A860002AD02B7A0100DB0800220CA8059307F000
:10A87000C1FD23000F331F000493049B059AFB1AAC
:10A880009A4208D939780CA803F0BAFC0CA807F052
:10A8900071FE0137F1E70F98F2F772FD297A300067
:10A8A000C90801F07DF805003000F2F769FD2A00C3
:10A8B00094490998FDF731FE934B09AA186893490A
:10A8C0000AF0E8F80998F2F75BFD914DFF232A00A2
:10A8D000283212780793002A00D1EEE1EA6A002AB2
:10A8E00000D1EAE108AE09AF7370B370F370231DB5
:10A8F0007B602A23002228003B8123883270383075
:10A90000102B0CD0827A049292073FD5A2888149FD
:10A910008A4209D0A91CC98F914237D104E0012194
:10A92000837A0B4207D1C8E12A003832D27AB2705A
:10A93000002272702AE0022383720F333B70727020
:10A94000A288AB1CA61DDA87310007220DF093F90F
:10A95000637D01241C4007D02A005B084432D35C8D
:10A96000FF2B46D0079344E01C27380060436A4B16
:10A9700010301818072231000DF06EF9002801D1AF
:10A98000079436E00134072CEFD117E0172B00D0E5
:10A9900086E02A0001210426280014272C32537A4D
:10A9A00038308B435372049A09ABB24382721F70E2
:10A9B000A379002B29D1E37933423CD1002209ACA1
:10A9C000EB6A210008A898472378122B00D074E185
:10A9D00028003830837A012B00D16EE10123023543
:10A9E0008372023BEB87C37207220021F0F7E0FB82
:10A9F00063E12A000A21079B3832DBB208A8D37230
:10AA000091728370FEF7A4FDD8E7C77A0CA9B8B29B
:10AA10000AF04AF900280CD1404B1B68334208D099
:10AA200060210CA804F0D4FF002802D1380009F0FE
:10AA3000BDF8A279C3E708AEB378FF2BBED00827D4
:10AA40003A438272E27A920707D51C2228005A43C1
:10AA50004C308218907E8843907629003831CA7A2B
:10AA6000FF2AABD01C242F000A784C375C43022A03
:10AA700008D0281907225C300DF0FDF83B199A7EAA
:10AA8000022106E001211B4A3B190832D28F1A83AA
:10AA90009A7E8A439A760121300009F02DF88DE7DD
:10AAA000172B00D9CBE0132B76D13B700423049AEB
:10AAB00013431B4A9372D37AFF2B43D12A000027FA
:10AAC0001C214C32049208007843049B1B189A7E88
:10AAD000FF2A32D1290038310A78022A22D0FD22F9
:10AAE00028189A765C30F63A0DF0C5F81CE0C0469E
:10AAF000741F00200825002090A5030095A50300E1
:10AB0000B3A50300DDB103008C5A0020B8A50300F3
:10AB100088250020FFFF0000D4250020E45A0020F3
:10AB2000C0250020FE229A762A0007AB1F70079BE3
:10AB30003832DBB2B370D37211E00137072FC2D1C4
:10AB40005F4E0DE016235F481A22002118303B703B
:10AB5000F0F72EFB4423049A13435B4A93720026BA
:10AB600000212B001C2228000F913833DB7A4C3057
:10AB700053432A00C3181093544B119134330C9350
:10AB80000D910E913032A0880CAB09F033F80028FB
:10AB900000D092E0320012E7142B2FD12B00383373
:10ABA000DB7AFF2B1BD1280000231C27E1894C30C6
:10ABB0003A005A438218128B8A420DD1290008228A
:10ABC0000498383102430793DBB2CB728A723000AB
:10ABD000B370FEF7BDFC02E00133072BE8D12B0078
:10ABE0003833DB7A0021FF2B01D0384934312A0079
:10ABF000A0884C32002308F0FBFF5EE0112B5CD1F3
:10AC00000223049A9A4313002A0038329372049A5A
:10AC1000120707D55BB2002B0BDA0021300008F0D9
:10AC20006BFF06E0B078FF2803D008F0BFFFFF23DA
:10AC3000B3702B00102238339A72122302E01C2BBF
:10AC400002D113233B70B9E6522B07D12C35AB7AD6
:10AC50001F4A9B009B58300098472EE0182B2CD1A0
:10AC6000A379112B17D1049B1B0714D515481A2261
:10AC700000211830F0F79CFA16232A0004993B7043
:10AC80004A330B43383293722A0002212C32537A12
:10AC90000B43537292E680232A0004995B420B43D4
:10ACA0003832937215233B702B002C339B7A084A61
:10ACB0009B009B583000984780E613B0F0BDC0461B
:10ACC0004380000088260020C025002008250020A1
:10ACD00080A5030010B50068F2F752FB10BD70B5F7
:10ACE00004680500002C0DD02000F1F790FF06004D
:10ACF0002000F2F745FB0020864202D03000F1F739
:10AD0000EDFE286070BD10B50068002801D0FDF789
:10AD10007DF910BD0068002804D08022438992008C
:10AD20009B184381704710B504000800F1F7BCFF81
:10AD30000023984202D0F1F7D1FE0300236010BD3A
:10AD4000F0B587B0009003910098039916001F009A
:10AD5000F4F70EFE002807D032003B003000390027
:10AD60000CF0ACFD002808D00022002310001900D0
:10AD70000BF0B2FB04000D006BE0002200230098F2
:10AD800003990AF0E9FF009C039D002803D080226C
:10AD9000039B12069D1800220023300039000AF0A0
:10ADA000DBFF002802D080231B06FF1800220023AF
:10ADB000300039000AF0CAFF00283BD10122274B9E
:10ADC0005242300039000AF0D1FF002834D001226D
:10ADD000224B5242009829000AF0C8FF00282BD0CD
:10ADE00022002B00300039000AF0C0FF002825D0D7
:10ADF00000221B4B200029000BF092FF04900591CC
:10AE000001960297019A029B049805990AF0C2FFE5
:10AE1000019A029B002806D0019802990BF030F8A5
:10AE200001900291EEE7200029000CF0F3F90400F4
:10AE30000D00D5E7002400E00400250000220023D7
:10AE4000009803990AF088FF002802D080231B068F
:10AE5000ED182000290007B0F0BDC046FFFFEF7FCE
:10AE60000000E03FF7B50500019110001900160041
:10AE70001F000CF043FD041E092C15D80CF074FDC6
:10AE800002000B00300039000AF060FF00280BD0F0
:10AE9000002C5ED028000199012C5CD02A00019B77
:10AEA0000BF03EFF013CF7E7002200232800019948
:10AEB0000AF052FF002200282FD0284B3000390022
:10AEC000FFF73EFF002200230AF040FF002833D0A6
:10AED00080230022DB0530003900FFF731FF00221C
:10AEE00000230AF033FF802212069446019B63443C
:10AEF000002802D02800190020E019002800F4F7EB
:10AF0000FFF90B000200390030000BF009FFFAF7DF
:10AF10002DFC80231B06C9181DE000232800019981
:10AF20000AF014FF002807D0390000220023300067
:10AF30000AF01CFF011E0ED028000199F4F7E0F979
:10AF400002000B00300039000BF0EAFEFAF70EFCAD
:10AF500001E02000014903B0F0BDC0460000F03F11
:10AF600070B504000D002178002904D028000134B8
:10AF700007F0E8F9F7E770BD0EB430B586B009AC5C
:10AF800020CC0100002201A807F034FA01A807F044
:10AF900012FA23002A0001A90548009401F012FFCB
:10AFA0000498F2F7EDF906B030BC08BC03B01847BE
:10AFB00061AF020010B586B00C000022010001A8AC
:10AFC00007F018FA01A807F0F6F92178002904D053
:10AFD00001A8013407F0B6F9F7E70498F2F7D0F9C1
:10AFE00006B010BD10B50400F1F734FF031E01D008
:10AFF00023000C33180010BD37B50400F1F702FF31
:10B00000002807D1201E25D08022638992009B183A
:10B0100063811FE0002210492000FBF70BFF0500B1
:10B02000F1F7FBFE002808D12800F2F7A9F98022E9
:10B03000638992009B1863810BE00021220001913B
:10B0400000910B002800FCF73FF804002800F2F7FD
:10B0500097F920003EBDC046ECAC030070B5041E5D
:10B06000184D2CD0F1F779FE174D002827D120007C
:10B07000F1F7C8FE002822D12000F1F7B8FE002821
:10B080001DD12000F1F792FE002818D12000F1F721
:10B09000C4FE0E4D002812D12000F2F715F80C4D19
:10B0A00000280CD12000F2F766F80A4D002806D1DE
:10B0B0002000F1F7BFFE084D002800D1074D280001
:10B0C00070BDC04673B003001FAB0300D5AA0300D8
:10B0D00025AE0300C3A5030052A50300F3810300BE
:10B0E00070B5002209490500FDF72FF900280BD0A3
:10B0F000FCF7E4FF0600FFF775FF2B68C41830006B
:10B10000F2F73EF9200000E0286870BDCFA10300EF
:10B1100070B5050009200C00F1F781FD002801D071
:10B120000560446070BD10B504000A20F1F777FD9A
:10B13000002800D0046010BD10B504000820F1F70D
:10B140006EFD002800D0046010BD10B5FFF7F4FFBD
:10B15000002805D03F2243899343343A1343438167
:10B1600010BD80220023120612184B4110B5002B8F
:10B1700002D1FFF7E1FF03E00AF06CFEFFF7C8FF22
:10B1800010BD70B588B00E000022010003A807F0C2
:10B1900031F9039B0093049B0193019A009B934216
:10B1A00030D203A805F0DCFF050006F02FF9041EDD
:10B1B00003D003A807F0DEF9EBE7FD232B3D1D428A
:10B1C00002D103A807F0D6F90025039B0093049B46
:10B1D0000193019A009B934215D203A8013505F013
:10B1E000BFFF2E2801D1002E07D13038C0B2092868
:10B1F00004D90698F2F7C4F80BE0002603A807F07C
:10B20000B9F9E2E700250698F2F7BAF8EC17641BE3
:10B21000E40F200008B070BD30B587B004000D0009
:10B22000F1F752FF0300002083420CD021002A00D6
:10B2300001A807F0DFF801A805F092FF04000498C8
:10B24000F2F79EF8200007B030BD70B50D00160073
:10B250008CB00100002207A81C0007F0CBF807A85B
:10B2600007F0A9F83200290002A807F0C3F8029BF2
:10B270000093039B0193019A009B93420DD2002CF3
:10B280000BD002A805F06CFF010007A807F05AF8E0
:10B2900002A807F06FF9013CE9E70598F2F770F8AA
:10B2A0000A98F2F76DF80CB070BD10B5024B002291
:10B2B000FFF7CBFF10BDC046FFFFFF7FF0B50124B5
:10B2C0008BB001920F000022010005A807F092F850
:10B2D00000252600069B0293059B0393039A029B7D
:10B2E00093421AD905A805F03BFFBC4209D1019B46
:10B2F0009E4208D30898F2F743F8681EA74210D37D
:10B300000EE0BC42F6D801360A2801D101260134EC
:10B3100005A8013507F02EF9DCE70898F2F730F8B8
:10B3200028000BB0F0BDF0B501258BB002911700DD
:10B330000100002205A81E0007F05CF800232C0085
:10B340000193069B059A0393934212D905A805F031
:10B3500007FF019B029A93420BD001340A2801D1C6
:10B3600001240135019B05A80133019307F002F97F
:10B37000E7E70898F2F704F83D6034600BB0F0BDE1
:10B3800070B588B00E000022010003A807F032F863
:10B3900000250124039B0093049B0193019A009BC9
:10B3A000934210D203A805F0DBFE0A2803D1013432
:10B3B000A64204D207E0A31B5A425341ED1803A84A
:10B3C00007F0D8F8E6E70698F1F7DAFF280008B0AA
:10B3D00070BD10B588B00100002203A807F00AF87C
:10B3E0000124039B0093049B0193019A009B9342C9
:10B3F0000AD203A805F0B4FE0A384342434103A829
:10B40000E41807F0B7F8ECE70698F1F7B9FF200069
:10B4100008B010BDF8B505000E00170005F0A7FE36
:10B42000041E04D03B0032002900FFF70EFF20006D
:10B43000F8BD0FB410B586B005F099FE041E11D00A
:10B440000100002201A806F0D5FF01A806F0B3FF15
:10B4500009AB0748089A01A9009301F0B3FC0498CE
:10B46000F1F78EFF200006B010BC08BC04B01847EE
:10B4700061AF0200F8B505000024F1F735FE2600A3
:10B48000A04218D0002D13D02800F1F751FB07007F
:10B490002800F6F77DFA002524183000F1F770FF38
:10B4A000AF4203D03800F1F719FB05002E00E9E7A1
:10B4B0003000F1F765FF2000F8BDF8B50500F1F7A1
:10B4C00003FE002803D02800FFF7D4FF2FE0280058
:10B4D000F1F7A3FC041E2DD12800F1F788FC041E0F
:10B4E00028D12800F1F78EFC041E23D12800F1F7A3
:10B4F00051FE002818D02800FCF715FE02000B00B2
:10B5000006000F000CF0DAF900280AD1002200230F
:10B51000300039000AF01AFC4442444160420124E0
:10B5200004400120044005E0280000F057F9441EC3
:10B53000A041C4B22000F8BD10B50B4B041E10D0C2
:10B54000F1F70BFC094B00280BD12000F1F713FE9B
:10B55000031E06D02000FFF7B0FF054B002800D1E6
:10B56000044B180010BDC04673B00300B88103003F
:10B57000D181030094810300F0B595B004000E0062
:10B58000F1F7B2FD00280AD02000F1F7C1FB002836
:10B5900005D04D4A00212000FFF73CFF38E0200095
:10B5A000F1F792FD071E06D08022638992009B1856
:10B5B0006381250080E02000F1F724FC002820D0E2
:10B5C0003A0042492000FBF735FC051E11D0404BE4
:10B5D00002689A420DD021003B003A00F5F748FD81
:10B5E00004002800F1F7CCFE01212000FFF7C4FF82
:10B5F00005E02800F1F7C4FE3648F2F765FC0500C7
:10B600005FE02000FFF798FF002803D0F2F75CFC12
:10B61000050051E02000F1F7D8FD002804D0217882
:10B6200003A8F5F71DFC0AE02000F1F7BEFD002895
:10B6300007D00A23012203A9206801F093FB03A885
:10B64000E4E72000F1F7A6FD00280BD001235B42C0
:10B6500001930B33009303AA38332068616801F02B
:10B660005DFAECE72000F1F7C2FB002804D12000CE
:10B67000F1F79CFB00280CD01748F2F725FC0700D7
:10B6800001002000F7F764F805003800F1F778FEB4
:10B6900012E02000F1F7C1FB051E09D005F067FD9F
:10B6A000051E09D001000022200004F0EFFF03E096
:10B6B0000A49042001F0B2FD002E02D02000F1F76B
:10B6C0005FFE280015B0F0BDFFFFFF7FCBA5030094
:10B6D00029030300D4A5030068A30300E4A5030025
:10B6E000F0B58BB004000D001600FFF725FF071E14
:10B6F00006D00100320028000CF0F8FA38001EE0F5
:10B700002000F1F752FD002806D00A23012229006B
:10B71000206801F027FB11E02000F1F73BFD071E38
:10B7200010D0012327685B42646801930B330093B8
:10B730002A0033003800210001F0F0F928000CF055
:10B74000BAFA44E02000F1F7CFFC011E27D0210017
:10B750003A0005A806F04EFE3400059B0293069BB6
:10B760000393039A029B934212D2012C06D8002322
:10B7700008982B70F1F704FE300028E005A805F0CA
:10B78000EFFC287005A806F0F5FE013C0135E4E762
:10B790000898F1F7F5FD0023301B2B7017E020000F
:10B7A000FFF7EAFE3200041E08D02900FFF798FFD9
:10B7B00005002000F1F7E4FD280008E00549280015
:10B7C0000CF094FA0420044901F028FD20000BB08D
:10B7D000F0BDC046A97F0300E4A5030030B5040016
:10B7E00089B0002801D100204CE0F1F7B6FA00281A
:10B7F000F9D12000F1F7F4FC002804D12000F1F782
:10B80000CAFA051E01D020683CE02000F1F7EFFAEB
:10B8100000280BD02368012B08D129002000F6F75F
:10B82000CAFEFCF74BFCF1F73CFE2BE02000F1F7E1
:10B83000B1FC00280CD02568646828002100F4F7CA
:10B8400097F80028CFD0280021000AF0CBFA19E0A1
:10B850002000F1F739FC0028C5D001212000FFF7B6
:10B8600090FC0028BFD0202269462000FFF738FF57
:10B87000202804D104491F3801F0D0FCB3E7684602
:10B8800001F056FF09B030BD26A2030010B5040038
:10B89000F1F78BFC002804D02000FFF79FFFC117B1
:10B8A00004E02000FCF73FFC0AF09CFA10BDF0B564
:10B8B000040089B0002804D03F2243891A40082A96
:10B8C0005ED02000F1F700FC002838D000250022CF
:10B8D000210003A806F08EFD2E002F00039B00938D
:10B8E000049B0193019A009B934217D203A805F091
:10B8F00037FC0300303BDBB20135092B03D9069836
:10B90000F1F73EFD37E0002F04D1302801D0013798
:10B9100000E0012603A806F02DFEDFE70698F1F708
:10B920002FFD2A1E05D00122002E02D0013D6A42C1
:10B930006A41D3071FD52000FFF750FF18E0200011
:10B94000F1F728FC002816D02000FCF7ECFB0600DD
:10B9500020000F00FFF742FF05000CF005F8020081
:10B960000B00300039000AF0F1F9002803D028005C
:10B97000FFF7E2FB08E000212000FFF7FDFD03E0F8
:10B98000802292009B18438109B0F0BD70B504007D
:10B99000FFF78DFF05002000F1F7F2FC280070BDD5
:10B9A00070B5050004200E00F1F739F9041E12D01D
:10B9B0002B7A280001332B72F1F79EF8010020004A
:10B9C000F1F716F981232371002E03D12800FFF728
:10B9D00051FD06006680200070BD10B50400F1F72F
:10B9E00083FB03000120002B05D02000F5F7D0FFDA
:10B9F00043425841C0B210BDF0B504008BB00D00F9
:10BA0000002800D1CAE03F2342891340082B26D1E9
:10BA10000800F1F7CAFB061E05D12800F1F7ABFBC1
:10BA20000D27002816D02800F1F7CFFB0D27019035
:10BA300000280FD1802329689B00CA18594B9A42CD
:10BA400008D8731E9E410F2389B220009F1BF1F777
:10BA5000CFF8019D3F2366899E433E4391E01A0043
:10BA60001A3A072A00D98DE01E2B6AD90100042258
:10BA700005A806F0BFFC2420F1F7D1F8071E36D048
:10BA80008022438992009B18438106000023019382
:10BA9000069B0293059B0393039A029B934228D92A
:10BAA000019B082B16D9300019000A3006F0C4FBA0
:10BAB0002420F1F7B4F80190002805D0F1F71CF824
:10BAC00001003000F1F728F83000F1F759FC0023AD
:10BAD000019E0193019B05A80133029305F040FBF1
:10BAE000019BF05405A806F045FD029BCFE7060038
:10BAF00001900898F1F744FC002E07D0300001991E
:10BB00000A3006F099FB3000F1F73AFC20000421DE
:10BB10000A3006F091FB3800F0F7EEFF010020003C
:10BB2000F0F7FAFF00212000F1F747F8002120008C
:10BB3000F1F73AF820000021F1F75AF83800F1F750
:10BB40001FFC2800F1F731FB1526002811D0280032
:10BB5000F1F73BFB071E0CD1802329689B00CA1814
:10BB6000104B9A4205D889B22000F1F741F83D0008
:10BB7000053E2000F5F70CFF3F22638986199343A9
:10BB80001E436681002D09D02B7A280001332B72C9
:10BB9000F0F7B2FF01002000F1F72AF820000BB007
:10BBA000F0BDC046FF03000010B50400F1F7B0F887
:10BBB000011E02D12000FFF71FFF402263891343BB
:10BBC000638110BDF8B507001A20F1F728F8051EAB
:10BBD00003D11E4801F026FC35E080220400438991
:10BBE00092009B1843812000F1F75EFA0926002895
:10BBF00006D12000F1F78CF8053E002800D103366D
:10BC000020000A30B74203D8390006F015FB17E0D0
:10BC1000310006F011FB2420F1F701F8BF1B061ECE
:10BC200003D10B4801F0FEFB0AE0F0F765FF0100CD
:10BC30002000F0F771FF2000F1F7A2FB3400D2E7FB
:10BC40002000F1F79DFB2800F8BDC04615820300D7
:10BC50004282030070B50C00043123680500984748
:10BC6000002D02DB63690133636100280BDB2500D3
:10BC70001835C1B2280006F05CFB280006F0A9FCCC
:10BC800023690133236170BDF0B585B00E00050056
:10BC9000F5F7CEF801AC07003100200007F019F8E5
:10BCA000002826D03B00223BDBB2022B13D9002F09
:10BCB0001FD16079FF2802D0012108F0EDFCA079A6
:10BCC000FF2802D0032108F0E7FCE079FF2802D02A
:10BCD000012108F0E1FC084A002E06D031002800BE
:10BCE000FCF742FCF1F74CFB03E011002800FCF7E5
:10BCF00077FB05B0F0BDC046A97D030010B5F6F78F
:10BD00006DFE10BD10B5024801F08CFB10BDC046A1
:10BD100010A603000B0010B5C1B2187807F078FC2C
:10BD200010BDF7B51F000D001600F5F781F86B4642
:10BD3000DC1D207011380A281AD8002E04D02800E3
:10BD40000021FFF719FC050022000A49280006F02F
:10BD5000C2FD002E02D02800F1F712FB002F07D001
:10BD600021000D20FFF7D6FF21000A20FFF7D2FFA8
:10BD7000F7BDC04615BD0200002310B51A00FFF73D
:10BD8000D0FF10BD012310B51A00FFF7CAFF10BD88
:10BD900010B500230122FFF7C4FF10BDF0B59DB020
:10BDA000070000911600F5F743F80300113BDBB2E2
:10BDB00001900A2B00D9E2E096239B010493FF2314
:10BDC00004AD2B716B71AB71F73BEB71012200235A
:10BDD0006A722B72AB729E4206D1320069493800FA
:10BDE000FCF7A1FB060004E08022738992009B18F7
:10BDF0007381002307AC05AA03930293624BA260F0
:10BE0000624A07930B23E2600D2202A9A3802382DA
:10BE1000A383033352185B18626123625C4A5D4B53
:10BE2000A26163620F22082352182385A386093377
:10BE30005B18E262584AA363584B22631622E363FD
:10BE400005235218D38703AA6264554A2165A26468
:10BE50001AAA1380009B002B0DD01800FFF7BEFC20
:10BE60000200504B653A9A4204D94F49012001F033
:10BE7000D5F900E02860210007223000F6F7C4F869
:10BE80000124002842D00023039C2B722000F1F7EC
:10BE90001BF900281DD045492000FCF751FA002865
:10BEA00001D001230CE042490398FCF749FA00282D
:10BEB000F7D140490398FCF743FA002802D0022347
:10BEC0002B720FE03C490398FCF73AFA0028F6D1B0
:10BED00008E02000F1F769F900280CD02000FFF7F6
:10BEE0007DFC28722A7A022A05D93449012001F002
:10BEF00095F900240AE0029C002C04D02000F0F701
:10BF00002CFF002826D000230124AB720398F1F700
:10BF100037FA0298F1F734FA002C03D13000F1F728
:10BF20002FFA2CE02900019808F0E0F80498FFF7B8
:10BF300003F9234902003800FCF7EFFA1149002EFB
:10BF400004D032003800FCF7E8FA18E03800FCF7BB
:10BF500047FA14E01B492000FCF7F2F90028D2D17F
:10BF600019490298FCF7ECF9041E02D00124AC72C6
:10BF7000CCE7029A1549012001F050F9C6E71DB03F
:10BF8000F0BDC046A97D030058A603005BA60300D0
:10BF9000397E0300B27D03005EA603000A7E030023
:10BFA0007BA803001B96980067A6030004B4030057
:10BFB00083A60300A682030087A603008CA60300C5
:10BFC000A78803009EA60300A3A60300A7A603005C
:10BFD000F7B5F6F7BBF80520F0F721FE041E00D1F7
:10BFE0007EE0404E404B002231005868FCF79BFA3F
:10BFF0000196051E00900AD00021F6F72EFB0121C4
:10C0000000902800F6F729FB2800F1F7B9F900277E
:10C0100001250C233F226E1E5E43344B9819438941
:10C0200013420CD00137F0F715FF002807D02F4B33
:10C030000C21F0580B3009F0F7FC2D183F18FF26A3
:10C040000135B600B542E4D9009BFD1A701BFFF71D
:10C0500073F8274902002000FCF75FFA2800FFF779
:10C060006BF8244902002000FCF757FA3000FFF774
:10C0700063F8214902002000FCF74FFA0098FFF70F
:10C080005BF8019902002000FCF747FA1B48FFF714
:10C0900053F81B4902002000FCF73FFA0020FFF78D
:10C0A0004BF8184902002000FCF737FA1648FFF752
:10C0B00043F8164902002000FCF72FFAFD20800209
:10C0C000FFF73AF8124902002000FCF726FA802018
:10C0D000C002FFF731F80F4902002000FCF71DFAFB
:10C0E0002000FEBD698203008C5A0020BC2600207F
:10C0F000C0A60300C5A60300CBA60300905C0020E9
:10C10000D1A60300E1A603001CB50300EDA60300C1
:10C11000FEA603000FA7030010B50520F0F77FFD72
:10C1200004002F48F1F7D0FE2E4902002000FCF752
:10C13000F4F92D48F1F7C8FE2C4902002000FCF765
:10C14000ECF92B48F1F7C0FE2A4902002000FCF769
:10C15000E4F92948F1F7B8FE284902002000FCF76D
:10C16000DCF92748F1F7B0FE264902002000FCF771
:10C17000D4F92548F1F7A8FE244902002000FCF775
:10C18000CCF92348F1F7A0FE224902002000FCF779
:10C19000C4F98020C002FEF7CFFF1F490200200033
:10C1A000FCF7BBF980200002FEF7C6FF1B49020026
:10C1B0002000FCF7B2F9FDF723FD19490200200029
:10C1C000FCF7ABF9174B187807F0E6F8F1F77CFEAF
:10C1D000154902002000FCF7A0F9200010BDC04660
:10C1E000979A03001CA7030024A7030030A70300AD
:10C1F0003BA7030044A703004FA7030078A7030051
:10C200009E7D030083A7030089A7030092A7030074
:10C2100097A703009DA70300A9A70300AFA70300EA
:10C22000B3A70300721F0020BAA7030070B5084926
:10C2300005000020F4F7EEFF041E07D02800FEF7EB
:10C2400084FF044902002000FCF767F9200070BD5C
:10C250009BA00300AEA30300F7B50C00022105006C
:10C2600000920193012608F017FA0027002C27DD21
:10C27000019B00993B40314019430ED072B600211A
:10C28000280008F06FFA0A2005F0AEFE0121280010
:10C2900008F068FA62B637200CE072B6280008F0A1
:10C2A00061FA412005F0A0FE0121280008F05AFAA9
:10C2B00062B6052005F098FEB6197F41013CD5E72E
:10C2C000F7BD10B50200002308780821FFF7C4FF6E
:10C2D00010BDF8B50C0002210500012708F0DCF9BB
:10C2E0000026002C1BDD72B60021280008F03AFA67
:10C2F000032005F079FE0121280008F033FA0A2016
:10C3000005F072FE280008F01DFA002800D03E4318
:10C3100062B6352005F068FE7F00013CE1E73000A1
:10C32000F8BD10B50400022108F0B6F90021200084
:10C3300008F018FAFA20400005F056FE012120000E
:10C3400008F010FA502005F04FFE200008F0FAF92E
:10C350000400D220400005F047FE01204440E0B236
:10C3600010BD10B500220349FCF7DDF8F4F718FE04
:10C3700010BDC046AEA30300F0B58FB00391FFF728
:10C38000F0FF0700F4F716FE002800D18BE0032031
:10C39000F0F745FC0290002800D184E0039B013BAC
:10C3A000FE2B01D9F0230393002338000593FFF7F8
:10C3B000B8FF002879D001250026039B039ADB17DC
:10C3C00008213800FFF748FF049601950121380045
:10C3D000FFF77FFF0121C4B23800FFF77AFFC0B238
:10C3E000012C02D1012814D130E0844219D1019BE3
:10C3F000059A934205DA07AB9C5D2C40601E844190
:10C4000004E0019B059A9C1A60424441E4B2002C6E
:10C4100005D007AA935D01242B43935505E0019BAA
:10C42000049307AA935DAB43935500232200012197
:10C430003800FFF711FF019B6D000133EDB201934E
:10C44000002D01D101360135072EBFDD019B402BA8
:10C450002BDD07A90B78002B27D0002209A88B5CC5
:10C460001C0925005735092C01D83034250054000B
:10C4700025540F252B401D005735092B01D830338B
:10C480001D00041901326570082AE8D100230374E5
:10C49000F1F71AFD01000298F6F74AF8049B002B09
:10C4A00003D0049B81E7002000E002980FB0F0BDAC
:10C4B00070B58AB00C00FFF754FF0600F4F77AFD60
:10C4C00000282DD02000F0F7B5FC002822D0200055
:10C4D000FFF784F9010004000120F5F782FD051E35
:10C4E0001ED001000022684605F0D1FF002C0CD0C0
:10C4F00008213000FFF7EDFEC1B2684605F019FFD4
:10C50000684606F066F8013CF0E7684605F0CAFEAA
:10C51000280005E008213000FFF7DBFEFEF70CFEE7
:10C520000AB070BD73B50E001500FFF71AFF6B4619
:10C53000DC1D2070F4F73EFD002816D022000B49C8
:10C54000300006F0C8F92078002D07D0012108F04E
:10C5500009F92078012108F09FF806E0032108F08E
:10C560009BF82078012108F0FDF873BDC3C20200DA
:10C5700010B5FFF7F6FE0400F4F71CFD002805D007
:10C58000CC22002308212000FFF766FE10BD10B565
:10C59000FFF7E7FE0400F4F70DFD002802D02000AD
:10C5A000FFF7BFFE10BDF0B587B00C00FFF7D9FE56
:10C5B0000500F4F7FFFC002846D02000F0F784FDCA
:10C5C000002803D1214800F02DFF3DE02000FEF7B8
:10C5D00051FF1028F6D12800FFF7A3FE2100002408
:10C5E000002201A805F006FF2700260001A804F09C
:10C5F000B7FD6B46187001A805F0BCFF01A804F058
:10C60000AFFD6B46587001A805F0B4FF00226B46E1
:10C61000102168469A7001F02DF8220009F07AFB8B
:10C62000083407430E43402CE0D10498F0F7A8FEED
:10C630005522002308212800FFF70EFE3A003300A0
:10C6400021002800FFF708FE07B0F0BDC2A70300D5
:10C65000F0B599B00D00160008A909AA06F0BAFBBA
:10C66000041E00D194E0FF2E03D000213000F4F727
:10C67000ADFC2800F0F7DEFB0090002811D0280068
:10C68000089CFFF7ABF809A9C0B2A047002804DA5C
:10C69000012009A94042089B9847FEF74DFD040080
:10C6A00070E02800F0F710FD071E40D004F05FFD99
:10C6B00029000400009A03A805F09CFE009D2F00AD
:10C6C000049B0093009A039B934203D30698F0F7D0
:10C6D00057FE29E000F01AFA0028F7D103A804F069
:10C6E0003FFD089B09A9013700939847002806DB06
:10C6F00002ABD91C08702000013508F00FF903A81F
:10C7000005F038FFDCE700F001FA00283AD10120FB
:10C71000089B09A940420093984702ABD91C0870B6
:10C720002000013508F0FAF8AF42ECDC2AE02800DE
:10C7300006F0A0F901000120F5F753FC041E21D0FA
:10C7400001003A000EA80D970C9705F0A0FE08AA6C
:10C750001149280006F0BFF80C9B00930D9B019334
:10C76000019A009B934203DB0EA805F09BFD09E0B4
:10C7700000F0CCF90028F7D1012008A94042FFF7CA
:10C7800069FAE9E7FF2E03D001213000F4F71EFC1F
:10C79000200019B0F0BDC04655BC0200F0B587B00E
:10C7A000050002910392F0F738FB002805D12A001A
:10C7B0006249032000F032FD0BE02800F0F7D8FAC0
:10C7C00000280BD046202F68AE88F0F728FA041E08
:10C7D00001D10020B0E0076086800CE00620002D2B
:10C7E00005D03F2368891840072800D00620F0F7BD
:10C7F00016FA041EEDD0290005A8FEF794FA059B51
:10C80000002B27D005A8FEF785FA050005A8FEF73E
:10C810007AFA06002800F0F7A0FC00230193984262
:10C8200011D03200531E9A410192002E0BD02800E5
:10C83000FBF70CFF071E06D001002000FBF7DEFA15
:10C840003800F0F79DFD31002800F0F7CDFD019B89
:10C85000002B04D1039904A8FEF765FA1DE005A892
:10C86000FEF73DFACBE7012200212800FBF788FE06
:10C8700007003100FBF7C3FD39002000FBF7BEFACB
:10C8800028003900F0F7B0FD05A8FEF728FA3000BF
:10C89000F0F776FD04A8FEF722FA049B04A8002B0B
:10C8A00011D0FEF730FA059B0600002B31D005A809
:10C8B000FEF730FA0500F0F750FC0028D3D128002D
:10C8C000F0F75EFD25E0FEF705FA059B05A8002BB5
:10C8D00016D0FEF71FFA012211000600FBF750FEEA
:10C8E000051E06D001002000FBF788FA2800F0F7AB
:10C8F00047FD3000F0F744FD05A8FEF7F0F9E4E746
:10C90000FEF7E8F9029A0E492000FBF7F7FD200038
:10C9100012E004F02CFC051EB9D02800FFF744F902
:10C9200031002800FBF76BFD20002900FBF766FAB9
:10C930002800F0F725FDAAE707B0F0BDE1A7030046
:10C94000C5A103001F21024A938E8B439386704733
:10C950008C5A0020F7B505000191F0F753FA002832
:10C9600030D0002251492800FBF7DDFD041E12D112
:10C970004F4B02004F491868FBF7D5FD061E1CD02F
:10C9800022004D49FBF7CFFD07003000F0F7F8FC1F
:10C99000002F12D03C00A5420FD0002201992000A8
:10C9A000FBF7D3FC071E04D101992000FFF7D2FF4B
:10C9B00007002000F0F7E4FC75E02000F0F7E0FC51
:10C9C000002071E02800F9F7CBFF0400002C68D0AC
:10C9D000374B002221001868FBF7B7FC002806D16E
:10C9E000364920000BF05DF900281ED157E0FBF717
:10C9F00065FB0500F0F717FC002801D100270EE0C9
:10CA000000222D492800FBF78EFD061EF6D00022DD
:10CA10000199FBF79AFC07003000F0F7B1FC280001
:10CA2000F0F7AEFC002FDBD03DE0254920000BF0F5
:10CA300038F9002833D0234920000BF032F90028C0
:10CA40002DD0214920000BF02CF9002827D01F49B8
:10CA500020000BF026F9002821D01D4920000BF002
:10CA600020F900281BD01B4920000BF01AF90028E0
:10CA700015D0194920000BF014F900280FD01749E0
:10CA800020000BF00EF9002809D00A4D20002900E3
:10CA90000BF007F9441EA04144422C4096E7104C8D
:10CAA00096E7200000E03800FEBDC0465288030033
:10CAB0008C5A002039890300908803003BA00300B2
:10CAC000CB9F030011A003002FA0030006A00300CA
:10CAD000DD9F0300C09F0300F99F030022A0030015
:10CAE00094AA030010B5084C0A00E36A002B05DD88
:10CAF00001339B00E3180100586801E00100206841
:10CB0000FBF723FC10BDC0468C5A0020024B988EC8
:10CB10000007C00F7047C0468C5A0020F0B589B09E
:10CB20001600009302000B0005000C000AF0C6FE80
:10CB3000002802D0009A814910E028002100F2F775
:10CB400017FF0022002300280CD12100280009F043
:10CB500003F9009A7A49002800D07A4930000BF096
:10CB6000C5F8E8E02800210009F0F6F800280DD00B
:10CB7000009B013B0093002B02D16B461B78D9E050
:10CB80002D23337080231B06E41801366E4A6F4B49
:10CB90002800210009F074F90AF0B0FE2100070016
:10CBA00028000AF0ABFE0130874204D138000AF0B9
:10CBB000DBFE05000C000022654B0E9802920393E9
:10CBC0000AF0D2FE029A039B049005910AF0A8F89D
:10CBD0002A0023000690079109F0C8F8002802D027
:10CBE000069A079BE9E73700029803990022584B01
:10CBF0003E0009F0CFF8002831D0029A039B2800AC
